:020000040000FA
:1000000000A10020FD2F0000B9B20000E92F000080
:10001000E92F0000E92F0000E92F00000000000098
:100020000000000000000000000000005930000047
:10003000E92F00000000000029320000E92F000035
:100040009532000095320000953200009532000094
:100050009532000095320000953200009532000084
:100060009532000095320000953200009532000074
:100070009532000095320000953200009532000064
:100080009532000095320000953200009532000054
:100090009532000095320000953200009532000044
:1000A0009532000095320000953200009532000034
:1000B0009532000095320000953200009532000024
:1000C0009532000095320000953200009532000014
:1000D0009532000095320000953200009532000004
:1000E00095320000953200009532000095320000F4
:1000F00095320000953200009532000095320000E4
:100100007BB972B90029BEBF00204FF0004106E064
:1001100008BF00281CBF6FF000414FF0FF3000F017
:1001200057B8ADF1080C6DE904CE002909DB002BAE
:100130001ADB00F057F8DDF804E0DDE9022304B033
:100140007047404261EB4101002B1BDB00F04AF895
:10015000DDF804E0DDE9022304B0404261EB410137
:10016000524263EB43037047524263EB430300F098
:1001700039F8DDF804E0DDE9022304B0404261EB28
:1001800041017047524263EB430300F02BF8DDF866
:1001900004E0DDE9022304B0524263EB43037047FD
:1001A00053B94AB9002908BF00281CBF4FF0FF31DE
:1001B0004FF0FF3000F00CB8ADF1080C6DE904CE43
:1001C00000F010F8DDF804E0DDE9022304B0704728
:1001D000704700BF034613F8012B002AFBD1181A01
:1001E000013870472DE9F0478C468E46089E15462B
:1001F00004461946002B40F0D080724547D9B2FA28
:1002000082F74FB1C7F120030EFA07FC20FA03F37F
:10021000BD4043EA0C0CBC404FEA154EA8B2BCFBF3
:10022000FEF8230C0EFB18CC08FB00F943EA0C4344
:10023000994528D9EB1808F1FF3204D2994502D923
:10024000A8F102022B44A3EB0903A4B2B3FBFEFC0A
:100250000EFB1C330CFB00F044EA0344A04214D90B
:100260002C190CF1FF3304D2A04202D9ACF10203E5
:100270002C44241A43EA02401EB1FC40002334609F
:100280007360BDE8F0874246DDE76346F1E7002A88
:1002900079D0B2FA82F3002B3FD01946C1F1200386
:1002A00002FA01F52EFA03F20EFA01FE20FA03F328
:1002B00043EA0E034FEA154E00FA01F4B2FBFEFCCE
:1002C000AFB20EFB1C201A0C0CFB07F842EA0042EE
:1002D00090455AD9AA180CF1FF3004D2904502D9A2
:1002E000ACF102002A44A2EB08029BB2B2FBFEFC76
:1002F0000EFB1C220CFB07F743EA02439F4246D940
:10030000EB180CF1FF3204D29F4202D9ACF1020289
:100310002B44DB1B42EA004202E0AEEB0203012267
:100320004FEA154EAFB2B3FBFEFC200C0EFB1C33A4
:100330000CFB07F840EA034398452AD9EB180CF167
:10034000FF3004D2984502D9ACF102002B44A3EB54
:100350000803A4B2B3FBFEFC0EFB1C330CFB07F737
:1003600044EA0344A74216D92C190CF1FF3304D2F6
:10037000A74202D9ACF102032C44E41B43EA00403B
:100380000F46114678E71F2188E76046ABE76246D3
:10039000BFE76046DBE76346EFE7734506D916B96A
:1003A000002108466DE7C6E9000EF9E7B3FA83F7C6
:1003B00087B9734501D3824207D8841A6EEB0303D1
:1003C00001209C461EB900215BE73846FAE7C6E9E2
:1003D000004CF8E7C7F1200CBB4022FA0CF51D4396
:1003E00020FA0CF12EFA0CF30EFA07FE41EA0E0188
:1003F0004FEA154900FA07F4B3FBF9F81FFA85FE36
:1004000009FB18300B0C08FB0EFA43EA00439A452F
:1004100002FA07F240D9EB1808F1FF3004D29A45EE
:1004200002D9A8F102002B44A3EB0A0389B2B3FB63
:10043000F9F809FB183308FB0EFE41EA03418E452B
:100440002CD9691808F1FF3304D28E4502D9A8F1DE
:100450000203294443EA0040A0FB0298A1EB0E01ED
:100460004145CE46434602D306D14C4504D2B9EBB2
:10047000020E68EB05030138002EA4D0B4EB0E0287
:1004800061EB030101FA0CFC22FA07F34CEA0303C7
:10049000F940C6E9003196E74046C5E74346D9E74B
:1004A00030B587B00AF065F800F0E2F83448492129
:1004B0000AF0AEFB00F078F800F0D2F800F09AF8FD
:1004C000A8B14FF08043D3F800340BB1DB070ED551
:1004D000012000F087F82B4849210AF099FB01F030
:1004E000BBFF00B1FEE7284802F080FBFEE703A84F
:1004F00001F0E0FE254B1B68834204D024484521CF
:100500000AF086FBFEE7059A224849210AF080FBA3
:10051000039921484B7D0A7DC98A009149210AF03F
:1005200077FB1E4849210AF073FB9DF8100002A9D1
:1005300000F088F8044600B1FEE7029A059B184DCA
:100540001344039A128913442B6006F0E3F900F078
:1005500037FE02F095FB02F06DFD2B681B6883F3FC
:10056000088884F31488BFF36F8FBFF36F8F2B68F5
:100570005B6898470B4845210AF04AFBFEE700BF3D
:1005800092E80000ABE80000F8E50000F41000205D
:10059000CFE80000F2E8000021E900003FE9000098
:1005A000D807002064E9000008B50B480CF071FA88
:1005B00028B9BDE80840094845210AF029BB084A86
:1005C00005481E2109F087FFBDE8084002480022C7
:1005D0001E2109F09BBF00BF3CE2000087E900003C
:1005E0000100020002461E21014809F08FBF00BF32
:1005F0003CE2000037B5114C20460CF04AFA10B925
:10060000002003B030BD0E4A1121204609F063FFDF
:100610000028F5D12569A36801A95B6820469847A1
:10062000002804D0ECDB003818BF0120E9E72B6874
:1006300001985840C0F34040F5E700BF3CE200009D
:100640001100010008B5024608B9086008BD03485A
:1006500045210AF0DDFA6FF01500F7E7BEE900006A
:1006600002484FF4C05109F0A5BC00BFB8450020B6
:10067000094B0A4AC3F80026C3F80426C3F8082623
:10068000C3F80C26C3F81026C3F81426C3F818269E
:10069000C3F81C26704700BF000001403546526E6B
:1006A00008B502480AF0F0F8002008BDD7E90000BC
:1006B000014B1B68184700BF5001002030B50446AD
:1006C00085B00D461022002168460DF005FD02237D
:1006D0008DF802302A46044B01932146684609F002
:1006E000B3FD05B030BD00BFB106000008B504463B
:1006F000EFF31183202383F31288BFF36F8F06F08B
:1007000009F9204602F05AFF02480AF0BDF80AF043
:10071000E8FDFCE710EA00002DE9F043079D15B95C
:100720001560002012E00324B5FBF4F404EB440749
:10073000BD4218BF0134B4F1804F09D2A400013486
:100740008C4200D838B914606FF00B00BDE8F0831C
:100750004FF0FF34F7E7DFF8BCE004460021B94270
:1007600003F1030C04F104062CD3A942274624D23A
:100770001F7801F1010CAC45264938BF5B784FEA80
:10078000A70E28BF002311F80EE084F800E0AC4566
:1007900001EB131E3CBF9B0003F03C034FEA07171D
:1007A00007F0300738BFCB5C1EF80770677028BFB2
:1007B0003D23A3703D23E3703746381A00231060B1
:1007C0003B70AEE71CF8034C1CF8023C1CF8018C93
:1007D0004FEAA40924011EF8099006F8049C04F0CD
:1007E00030040EEB13199B0019F8044006F8034C73
:1007F00003F03C030EEB981408F03F08E35C06F8A6
:10080000023C1EF8083006F8013C033134466346CA
:10081000A5E700BF29EE00002DE9F043DDF81CE05C
:10082000DFF8208100273C463E46764526D3D4BBE0
:1008300014600020BDE8F0830135754531D013F810
:1008400005C0BCF1200FF7D0AEEB0509B9F1010FDF
:1008500016D0BCF10D0F13D103EB050999F80190E7
:10086000B9F10A0F1BD0B54205D1BCF13D0F0AD139
:100870000137022F0AD96FF01500DBE73546DCE7B8
:10088000BCF10A0FEEE71CF0800FF4D118F80C60F1
:100890007F2EF0D03F2E01D8002FECD101346E1CFA
:1008A000C3E72E46C3E704F007054FF0060CE40843
:1008B0000CFB05F50CFB04F40735E41B04EBD50435
:1008C00070B18C420CD80027DFF878E0DFF8788030
:1008D0001E44014603253C46B34205D10C1AA7E746
:1008E00014606FF00B00A5E713F8019BA9F10A0C47
:1008F0005FFA8CFCBCF1160F04D828FA0CFC1CF033
:10090000010FE9D11EF809C00134BCF1400F08BF46
:10091000013D0CF03F0C042C4CEA8717DCD17DB173
:100920003C0C012D0C7002D101310024D4E7022DC2
:100930004FEA17244C7016BF8F7002310331F4E771
:100940002C46C9E7A9ED0000090040002DE9F04759
:10095000058B0446280717460CD501290CBF45F026
:10096000100545F02005258387F31188BFF36F8FAD
:10097000BDE8F087022905F0070540F09480204685
:1009800009F0AAFF052864D801A353F820F000BF9E
:1009900069090000A70A0000530A0000150A0000B8
:1009A0002F0A0000410A000001F007035A1F012A24
:1009B0001FD8002221F00701062BD4F8008089B24D
:1009C000C4E9002209D1434603E0628B013262830D
:1009D0001B68002BF9D141F002012183204609F068
:1009E0007BFF4FF0000900286DD041F020012183EA
:1009F00069E0042B0AD121F0070189B22183204646
:100A000009F06AFF10B141F0200121834FF0000886
:100A1000C14658E02369D3F80090238B23F00703E5
:100A200043F0060323834FF0000846464BE023695A
:100A3000D3F80490238B23F0070343F00403F1E77A
:100A40002369D3F80890238B23F0070343F00503B1
:100A5000E8E74FF00008C146E7E7012243F008034A
:100A6000238387F31188BFF36F8F002A3BD1B8F13E
:100A7000000F4AD1B9F1000F02D02D492046C847D6
:100A8000EFF31187202383F31288BFF36F8F238B3B
:100A900023F008039BB22383D9063FD523F010022D
:100AA000228303F007056669218B002EBFF67CAF19
:100AB0000023D4F8008021F00701C4E9003341F09D
:100AC000010121839946238B03F0070AAA4502D02E
:100AD000A268002AC1D1B8F1000F02D1B9F1000F0C
:100AE000DAD00022BAE7A1680029C0D00D68002939
:100AF000BDD04F68334652462046B8471DB12B68DB
:100B000029461D46F3E72B46FAE74146334652464F
:100B10002046D8F8008009F00BFFA8E79A067FF579
:100B200023AF23F02002228303F0070527E700BF4D
:100B30005DA90000014B03600020704710E6000033
:100B400070B5104B1C680D46B4B10F4B19680023EB
:100B50008B4202DB6FF0010070BD224612F8106B71
:100B6000864202D001331446F2E7E0680BF091FFB1
:100B700028B12C600020EFE76FF00C00ECE76FF07D
:100B80001200E9E75401002010E6000010B588B01B
:100B9000436802938368C068CDE903320A68002382
:100BA000CDE906230C4601AA044905930AF01FFD6E
:100BB000079808B9059B236008B010BDDFAC0000A2
:100BC000F0B40D4B0D4E5F6A0D4BB34203D36FF083
:100BD0008500F0BC70475C68BC420AD31D6945B112
:100BE00094F802C08488E4B2A44502D12B46F0BC3C
:100BF00018472433E9E700BFDC0700201004002079
:100C0000EC0300202DE9F047144CDFF85480DFF8A6
:100C1000549005460E461746444503D36FF08500B1
:100C2000BDE8F0876268D9F824309A4213D3A369EB
:100C30008BB1A9889078C9B2884205D13A4631462D
:100C40002846BDE8F04718475279012A03D13A46B1
:100C50003146284698472434DEE700BFEC030020E5
:100C600010040020DC0700202DE9F0410B4CDFF8D8
:100C7000308005460E461746444502D36FF0850086
:100C800009E063690BB92434F6E73A463146284651
:100C900098470028F7D1BDE8F08100BFEC030020A1
:100CA0001004002010B504460AF08FFB10F1780FF5
:100CB00000D050B9054A20460AF047F8D2F8C430AF
:100CC00023EA0003C2F8C430002010BDDC07002076
:100CD000024B00221A605A60704700BF970800203C
:100CE00070B50B4B0B4CA34201D3002070BD196AA9
:100CF0001E7F00220439D5B2AE4201D82433F2E778
:100D0000013211F832508542F5D10120EEE700BFE3
:100D1000EC0300201004002073B58488E4B263065D
:100D20000D468DF8074007D02046FFF7D9FF78B170
:100D30000D4B93F8BA0058B10B4E204655B103F055
:100D400043F8F3691BB10DF1070108209847012012
:100D500002B070BD03F060F8F369002BF7D00DF11D
:100D600007010920F2E700BFDC07002008B50948A9
:100D70000378C3F341130A3350F823303BB100F139
:100D8000080200F110019847C043C00F08BD184683
:100D9000FCE700BFDC07002004282DE9F14FDFF855
:100DA000989004460F4616D001282DD1DFF88C808C
:100DB00098F8B93043B300F009FE214D4D4520D2DB
:100DC000D5F820B04FF0000A2B7F5FFA8AF6B342C5
:100DD00004D82435F2E7FFF77BFFE7E70BEBC60605
:100DE0000AF1010A30790AF0F0FA0246307909F086
:100DF000ACFFD8F8C430002A23EA0003C8F8C43096
:100E0000E2DA002388F8B9300D4D4D4508D30B4B7D
:100E10001B6A6BB13946204601B0BDE8F04F184758
:100E2000EB681BB13A462146284698472435ECE743
:100E300001B0BDE8F08F00BF10040020DC070020E7
:100E4000EC03002073B586788DF800600379427951
:100E50001C4C43EA0223ADF80230C378304603F05D
:100E600003038DF8043009F070FFD4F8C430184241
:100E700005460BD0304600F08BFD3046FFF712FFE1
:100E80000BF098FF10B9962007F0C8FE684602F0F4
:100E900077FF10F1780F03D010B1002002B070BDC1
:100EA0009DF8000002F0F4FF10F1780F01D0002847
:100EB000F3D1D4F8C43001202B4384F8B900C4F82E
:100EC000C430EBE7DC0700202DE9F047A94EB369F9
:100ED00004460F4690466BB9237803F01F03012B9D
:100EE00000F0A280022B00F0078143B16FF01500E3
:100EF000BDE8F08798470028EED10020F8E794F984
:100F000000206178002A2FDA062910D00829D8F8A5
:100F1000002024D00029E9D101231370517096F8E4
:100F2000C3305B0043F001031370022320E16288A9
:100F3000100A011F01290546D8D90728D6D8D1B2F1
:100F4000726A1478002CD1D05678AE4203D19942FF
:100F500000F0088101332244F3E7137808E196F8A2
:100F6000BA301370012303E101390829BED801A367
:100F700053F821F00F100000ED0E00001F100000CC
:100F8000ED0E0000990F0000ED0E0000ED0E0000C8
:100F9000ED0E0000A70F00006088C0B202F0DEFE78
:100FA0000028AAD0A2E763883BB1FF27756A00201A
:100FB000B8462B786BB9002898D0FFF789FE638874
:100FC00086F8BA30F369002B97D06B490320984715
:100FD00093E76B78042B0DD0052B0ED0022B06D196
:100FE0006F796388BB4208BF40F00100C0B22B7824
:100FF0001D44DEE795F80380F9E76388BB42F6D12C
:10100000B8F1000FF3D12846FFF71CFFEFE7638824
:10101000012B7FF46BAF002386F8C3306DE7638844
:10102000012B7FF463AFF7E796F8BA30002B3FF45B
:101030005DAFA388756A5FFA83FC2A4611780029A0
:101040003FF454AF5078022804D192F804E0E6450A
:1010500000F294800A44F1E70A704A7038604CE765
:10106000154499E00B2A7FF441AF00274FF0FF08A9
:10107000C146BA4606E06B78042B0FD0052B21D071
:101080002B781D442B78002BF5D1F36913B1514611
:1010900007209847002F7FF430AF27E795F80280AC
:1010A000A38895F803909845EAD163889945E7D1DC
:1010B000B8F1070F1DD806EB0803AA4683F8BB90CA
:1010C0000127DDE7A3884345DAD16388DBB24B45CE
:1010D0000AD0AF78384600F05BFC3846FFF7E2FDF7
:1010E000B0FA80F77F09CBE72846FFF7ABFE07464B
:1010F000C6E7AA460027C3E794F900206378002AD0
:101100001ADA002B7FF4F2AEA388DDB25B060AD0B8
:101110002846FFF7E5FD00283FF4E8AE96F8BA3020
:10112000002B3FF4E3AED8F800402846214602F0F9
:1011300093FE00236370F8E6012B08D0032B7FF4A5
:10114000D5AE6388002B7FF4D1AE012103E0618826
:1011500000297FF4CBAE2046FFF7DEFD00287FF4A8
:10116000CCAEC3E60228C8F800207FF4F6AE538860
:101170003B60C2E6DC0700209608002094F90010CE
:1011800062780029BFF66EAFD8F80010002A3FF44D
:1011900063AF0A2A7FF4AAAE2A78002A3FF4A6AEEB
:1011A000687804287FF45CAFA87883427FF458AF56
:1011B000072B96BF9B19002393F8BB300B70D1E629
:1011C00070B5164D95F8B830FBB102F0A7FD0028B8
:1011D00022DB00F0FBFB0024D5F8C430E340DA0743
:1011E000E6B214D4D5F8C43004F11002D340DB07C2
:1011F00005D546F08000FFF755FD00280CDB0134D3
:10120000102CE9D1002385F8B830002004E03046E6
:10121000FFF748FD0028E5DA70BD00BFDC070020BD
:1012200013B5164C237DF3B9E268A168019201ABB6
:10123000802009F098FD019AA3681344A360E36835
:101240009B1AE3606BB962B12369E2889A4208DDB8
:1012500094F8C82093FBF2F102FB11330BB9012380
:10126000237502B010BD00231A461946802023754D
:1012700002B0BDE8104002F035BE00BFDC07002020
:1012800030B585B0002302460D460193002858D1A1
:10129000002935D108220B460DEB02010AF0AEF809
:1012A000002804DA802002F08FFD05B030BD2A4C02
:1012B000029A2260039A626004F13802A2609DF9EA
:1012C0000820BDF80E302575002AC4E903550ADB55
:1012D000802B04D9802002F077FD0020E3E713B1D2
:1012E000C4E90333E1E7FFF741FD0028DAD0E288E3
:1012F00023699A42D4BFE260E360FFF791FFD4E72D
:10130000154CD4E90215002D01AB04DC0AF076F887
:101310000028CADAC6E72A460AF070F80028D9DBA6
:10132000019AA3681344A360E3689B1AE360002B4F
:10133000BBD104F13803A360FFF718FD0028DCD10E
:10134000B0E78028B1D1044BDA68002AD5D11B7DE3
:10135000002BD2D1A9E700BFDC070020054B064ACD
:101360009A62064ADA62064A1A63064A58629A6123
:1013700000207047DC070020C90E0000C10B0000F0
:10138000690C0000050C00002DE9F3410446454DB1
:1013900045484FF0FF334FF0FF3206F025FE95F839
:1013A000B830002B78D16E6A76B900F0CBF8FFF731
:1013B000D5FF6E6A46B94FF0FF343B4806F086FE13
:1013C000204602B0BDE8F08138482C62E86102F0A6
:1013D0009DFE02F075FC041EEFDB00F019FB041EFD
:1013E000EBDB7378012B5AD1F379002B57D0002611
:1013F000684685F8C830ADF802308DF804608DF885
:10140000006002F0BDFC041ED7DB802768468DF823
:10141000007002F0B5FC041ECFDB2549304602F017
:1014200061FE041EC9DB2249384602F05BFE041E41
:10143000C3DB204CDFF8808044451AD3002002F043
:1014400027FD041EB9DBD5F8C430802043F001032A
:10145000C5F8C43002F01CFD041EAEDBD5F8C43064
:1014600043F48033C5F8C430012385F8B830002434
:10147000A3E7276A0026227FF3B29A4201D82434D8
:10148000DAE707EBC30257F83310107902F02AFEAF
:1014900001360028EFD08EE76FF077048DE76FF00C
:1014A00015048AE7DC070020FC020020990D0000EB
:1014B00081120000EC0300201004002030B51F4B07
:1014C0008BB005AA03F1100518685968144603C4C7
:1014D0000833AB422246F7D11B78237001AC1022AF
:1014E000002120460CF0F8FD1222002114480CF0D7
:1014F000F3FD102120460AF02CF900281ADD0828F7
:10150000B8BF082009380E4A0444002114F8013FEE
:101510000AA800EB131003F00F0328336B440131CA
:1015200010F8140C13F8143C10700829537002F1D1
:101530000202EBD102480BB030BD00BF39EA000017
:10154000B95D00202DE9F04F724B93F800B087B0E1
:10155000BBF1000F03D0704807B0BDE8F08F6E4CB0
:1015600000264FF0011AB0463546B14623783BB904
:101570006A4B02349C42F3D1664A01231370EAE7B6
:101580006378052B05D8DFE803F08F07038F1F3B37
:10159000A14623781C44E9E7402304A88DF810B045
:1015A000ADF812308DF814B009F0FBFE40B10823FD
:1015B00004A8ADF8123009F0F4FE08B1ADF812B08D
:1015C000BDF81230E371E4E7E378002BE1D1A378B2
:1015D0006BB108F101085FFA88F8DAE76B689C42A2
:1015E00007D024354E4B9D42F8D30020B4E74D4D33
:1015F000F8E7AB68002BECD0414620469847E8E777
:10160000002DF2D000222B7F9A42EED2296AA078D8
:1016100001EBC2010B79984244D10127E07800F038
:1016200003008DF81400207994F805C040EA0C20DE
:10163000ADF8120094F902000028FBB228DA07F195
:1016400010004FF0010C0CFA00F010EA0A0F26D13E
:1016500043F080008DF8100004A8CDE90213019238
:1016600009F09FFEDDE90121039BC0B99DF8102020
:10167000A27012F0800F18BF10330A7118BFDBB2CE
:101680004FF0010214BF9A40BA404AEA020A80E7CA
:101690000120B84010EA0A0F01D11846DAE70137F5
:1016A000102FBBD10132AEE7032E1AD1FFF706FF90
:1016B000074650B1FEF78EFD024630B11028A8BF94
:1016C00010223946A01C0CF0E0FC23786FF00201D8
:1016D0001A19091B04EB5303D14213D50136F6B294
:1016E00057E7002EF1D1B9F1000F3FF47EAFA4EB24
:1016F000090389F80230C3F3072389F8033089F816
:101700000480EBE702F801BC13F8010902F8020DAE
:10171000E2E700BFB85D002030030020EB030020AB
:1017200010040020EC03002010B5094B00211A46DC
:101730001C78844204D15C6814B102EB811010BDA6
:101740000131042903F14003F2D10020F7E700BF83
:10175000A80800202DE9F34150F8283C10F82C6C23
:10176000103304460AD1036950F8202C980736D567
:10177000D2B9590715D5002344F8283C54F8283C21
:1017800010330BD054E9077554F8148C0BF012FB8E
:1017900000284FD02E4821460BF0F0FA02B0BDE8E9
:1017A000F08143F00403236154F8241C01AB30465C
:1017B00009F0D9FA10B16FF01503DDE7019A54F87A
:1017C000243C134444F8243C54F8203C9B1A44F82D
:1017D000203C54F81C3C134444F81C3CCEE754F81D
:1017E000241C01AB304602F0F3FB0028E3D1019D3D
:1017F00054F8243C2B4444F8243C54F8203C5B1B14
:1018000044F8203C54F81C3C2B4444F81C3C002D6C
:10181000B1D0304602F080FCB5FBF0F303FB10556D
:10182000002DA8D154F8203C002BA4D0304602F063
:1018300017FCA3E744F8180CA4F1100006F0C8FC4C
:10184000002DABD0424639463046A847A6E700BF38
:10185000100400204B1E012B73B506460D460FD811
:10186000FFF762FF044668B9012D09D101AB0122DF
:101870000DF10301304602F0ABFB019B002BF5D1CB
:1018800002B070BD0BF096FA04F12C0108B1012DE5
:1018900005D1084602B0BDE87040FFF75BBF0348C2
:1018A00002B0BDE870400BF069BA00BF1004002020
:1018B0002DE9F74F064601911546984609F09BFA27
:1018C000044600285BD1EFF3118A202383F31288AA
:1018D000BFF36F8FDFF8ACB000220023584606F04C
:1018E000ABFC70B9DFF8A090A70109EB8414636822
:1018F00013F1100F14D10193584606F069FC019BB7
:1019000006E00134042C0BF1400BE5D16FF00B0322
:101910008AF31188BFF36F8F184603B0BDE8F08FCC
:10192000019B2061C4E902350C9B63610D9BA3619F
:1019300030466FF00F0309F80760C4F83C8063601D
:1019400002F0EAFB58B1304602F0E6FBB5FBF0F3DB
:1019500003FB10551DB1E36B43F00403E36318F080
:10196000020F07D007F12C01084849440BF006FA92
:101970000023CDE7304602F073FB0346C8E76FF063
:101980000F03C9E7C4080020A808002010040020A5
:1019900010B5EFF31184202383F31288BFF36F8F08
:1019A000FFF7C2FE50B14368103307D16FF08B03CD
:1019B000436000F12C0104480BF0E0F984F3118836
:1019C000BFF36F8F10BD00BF10040020F8B50E4CA0
:1019D00004252027EFF3118687F31288BFF36F8F5A
:1019E0006368103307D16FF08B030848636004F11C
:1019F0002C010BF0C3F986F31188BFF36F8F013D03
:101A000004F14004E6D1F8BDA8080020100400202D
:101A100038B5094C0025094920460BF093F90122FD
:101A2000A4F11000114601350BF047F9042D04F123
:101A30004004F0D1002038BDD40800205517000024
:101A40000169012381F84B300B6833B191F84930BB
:101A50001BB1024808310BF091B970471004002007
:101A60000169012381F84A300B6833B191F848309D
:101A70001BB1024808310BF081B9704710040020F7
:101A800070B50569EFF31186202383F31288BFF345
:101A90006F8FD5F8900009F078F8044686F3118826
:101AA000BFF36F8F30B104480022002305F1180105
:101AB00006F030FD204670BD1004002070B50123F3
:101AC00082F8483013680D4614463BB192F84A300C
:101AD00023B10E4802F108010BF050F9D4F8903010
:101AE000DA885B899A4205D17DB904F1180140F684
:101AF000CD4204E004F11801002DF8D00022BDE829
:101B000070400248002306F005BD70BD100400209F
:101B100070B50E4681880446C9B21548154609F0CD
:101B200046F910B394F900206378002A16DB202BC5
:101B300004D0222B0ED06FF085000AE02B681A68C3
:101B400040F8102C9A8820F80C2C9B7900F80A3C5D
:101B5000002070BD638800F8093CF9E7212BEAD129
:101B60001038072328603360F2E76FF01200F0E7C7
:101B7000AC09002008B50146034809F026F910B168
:101B8000012300F8073C08BDAC0900200D4A0346BC
:101B90000021A0F848101068C3F89400908892794A
:101BA000A3F8980083F89A2083F89C1083F89B1080
:101BB000A3F89E1083F8A010402203F14C000CF013
:101BC0008BBA00BFE0E5000010B504690023C4F83B
:101BD000A8300C4BC4F8A400596804F1A80269B9F4
:101BE000C3E9002204F1080007490BF0ABF804F147
:101BF000180006490BF0D2F8002010BD0A605A60A8
:101C0000F0E700BFAC09002021AE0000951C0000E9
:101C100073B504698DF80710002384F84830202537
:101C2000EFF3118685F31288BFF36F8F0122D4F88A
:101C300090000DF1070108F0A8FF86F31188BFF3AB
:101C40006F8F012810D00BF0B5F8B0B10F4BBFF378
:101C50005B8F012253E8001F002903D143E80020D5
:101C60000028F7D1BFF35B8F2122002304F1180174
:101C7000074806F04FFC02B070BD94F8A130002B6D
:101C8000E4D0002121200BF060F9C9E7A809002069
:101C900010040020F0B5D0F88C305B681B6A1F7D03
:101CA00085B00546384609F0A6F8064650BB95F8BB
:101CB00086303BB3A86F0146C38831F80A2F9B1AC0
:101CC0009BB2B3F5806F28BF4FF4806303AA08F07E
:101CD0000DFF0446B0B18306A5F1180308BF00F15B
:101CE000FF3485F830600193074B03990093224637
:101CF00002233846FFF7DCFDA86F224600F10A01F7
:101D000008F02AFF05B0F0BDBD1A000037B5144633
:101D10000A1E054621DDD4F88C0004F14C0108F0C0
:101D200034FF012384F8493023683BB194F84B30E9
:101D300023B1114804F108010BF020F8D4F88C20ED
:101D40009388918912695B1A9BB2D31A3F2B04D8EE
:101D5000012384F8A03003B030BD94F89E30002BEE
:101D6000F9D0064B009301940123402204F14C0169
:101D70002846FFF79DFDEEE7100400200D1D000032
:101D800073B50D4601461D4809F005F8044610B329
:101D9000691EA0F1A40605291DD8DFE801F01E1C6C
:101DA000031E242810F8061CA9B903685D680123E6
:101DB00000F8063C2B6A3246187BFFF7A7FF14F8A1
:101DC0005C2C42B92B6A187D0D4B009301960223BF
:101DD0001146FFF76DFD02B070BD304602B0BDE8A0
:101DE0007040FFF7D3BE012304F8053CF3E710F879
:101DF000053C002BEFD00023F6E700BFAC09002024
:101E0000BD1A000013B500240749084800944FF09C
:101E1000FF334FF4806206F03DFB054903480AF0AA
:101E2000CFFF204602B010BDC06700201004002084
:101E300057EA000080B505460E461746984606F05C
:101E400037FF034601F038FADFF81890044649F8E6
:101E50000030424630463946A84754F8090001F0A0
:101E6000CDF900BF080000002DE9F04FD7B0DFF832
:101E700070A1DDF888C1DAF80050CDF80CC0DDF8AB
:101E800084C1CDF808C00DF1380BDDF880C1CDF864
:101E900004B0CDF800C0639C07468846164609F09A
:101EA00039F828B1DAF80050284657B0BDE8F08F6D
:101EB0006CB1A1465A4616AC134603CBA342C9F8EF
:101EC0000000C9F804101A4609F10809F4D10023EA
:101ED000009332464FF6FF73414608A809F05FF8B9
:101EE00005900028DED1314638460D9C09F00DF9E9
:101EF000A042D7D34FF0FF3416E03F88202FD1D136
:101F0000D9F800103B4616AA304608F09BFE002880
:101F1000C8D13A4616A9584609F0E8F8314B1B6873
:101F20008342BFD10123059306AF0DF11C090DF1CA
:101F30001A033A46494608A809F07FF80028B1DBA1
:101F400048D1D9F8001008A809F0C2F8BDF81A80E5
:101F500040B9254A4FF6FF7132F8023B8B42A1D0BF
:101F60004345F9D1B8F1100FC7D0B8F1200F13D005
:101F7000B8F1010FD8D13B88202B93D8D9F80010A5
:101F800016AA304608F05EFE00288BD1397816A8D4
:101F900000F02EF80446C7E7002CABDB134B1B68A0
:101FA0009C42A7DA3B88B3F5807F7FF47BAFD9F8FA
:101FB000001016AA304608F045FE00287FF472AFE4
:101FC000E4B200943B8816AA4146584600F0E2F875
:101FD00005468FE7059B012B7FF464AF64E700BFE4
:101FE00098010020F410002074E8000000E60000D2
:101FF0002DE9F0412029A2B080460D4605D94FF0C9
:10200000FF34204622B0BDE8F081124B124E1F680B
:102010000024BC42F3DA08A80BF02BFF002108A82B
:1020200007F03AFE736856F8081B1A6808A80BF008
:1020300029FF694608A80BF065FF08A80BF01DFFF3
:102040002A46414668460CF056F80028D9D001349B
:10205000DFE700BF00E6000004E600002DE9F04FD6
:102060008A46ADF27C5D1946484B1F68DDF8A03505
:10207000B3F5807F40F08480202A40F081805EADFF
:102080002A460BF086FE0446002879D195F8FF30E9
:10209000BC2B75D10DF198090DF10C0B4FF0DF0839
:1020A0004E46CBF800000CA80BF0E3FE00210CA874
:1020B00007F0F2FD20220DF257210CA80BF0E2FEF2
:1020C000042259460CA80BF0DDFE04A90CA80BF065
:1020D00019FF0CA80BF0D1FE42469BF80330202AD2
:1020E000A8BF20220133484604A901928BF803308F
:1020F0000BF0CBFF019AA8EB0208B8F1000F914456
:10210000D1DC30463246DF23117815F801CB013B94
:1021100081EA0C0102F8011BF6D1337803F07F034A
:10212000337010F8015B5DBB0134BE2CF9D196F819
:10213000BE30012B24D10CA80BF09BFE29460CA825
:1021400007F0AAFD124908220CA80BF09BFE51468D
:1021500020220CA80BF096FE20220DF257110CA89D
:102160000BF090FE04A90CA80BF0CCFE0CA80BF011
:1021700084FE20220DF2572104A808F0B7FF07467D
:1021800038460DF27C5DBDE8F08F00BF980100205D
:1021900069EE00002DE9F0479946A2B0294B9DF861
:1021A000A8A01D68064605A80F4690460BF0D7FD6F
:1021B0000922012105A80BF0D6FD234B53F83A4024
:1021C000039403EBCA0304AA5B681B681C44214602
:1021D000302303A80BF019FF60BBDDE90332134481
:1021E0009C4227D106AA214603A80BF06BFB08BB33
:1021F00008AA214603A80BF065FBD8B906A80BF086
:1022000061F8039B05909C4214D105A807F084FC5B
:1022100080B906A80BF056F8059005A80BF0B7FD9D
:10222000484507D1009043463A46314605A8FFF796
:1022300015FF054605A80BF0E4FD284622B0BDE8D1
:10224000F08700BF9801002004E6000038B5094B74
:10225000002918BF0B4643620121054608F058FFCC
:10226000044628B9286A08F02CFD2863204638BDAA
:102270000124FBE7B409002000487047F810002053
:102280001FB50B6913F00C0F18BF23F00C030246A7
:1022900018BF0B6100204FF480730093CDE902005A
:1022A000034B0190FFF7E0FD05B05DF804FB00BFB4
:1022B000CB5D0020F8B5104E104B054630461C682B
:1022C00008F082FFB0B90E4F306A394605F0B4FC11
:1022D00080B9306A3946FFF7D3FF0446094B1B68C3
:1022E000984207D1306A08F027F92871336A5B6891
:1022F000AB602F602046F8BDF81000209801002048
:10230000CB5E0020F4100020F7B5254E30688368BE
:10231000DB6B03B1984730688368DB6A002B31D1EF
:10232000204C214D306883681B69002B2DD0012281
:102330000DF107019847012827D1236843B92B687D
:102340002BB369681A682A608B4200D16A602360E7
:10235000164A9DF8070011887F2904D823680B448A
:102360004F1C178018720A28DCD123681188596025
:1023700000200F4918604D6875B9C1E9003310801D
:102380002060CEE798470028CAD103B0F0BD0948C5
:10239000452108F03DFCF8E72B604B60EFE700BFFC
:1023A000841500202C1100203C110020B445002091
:1023B0003411002060EA000010B5044B0446186890
:1023C0008368E1B25B689847204610BD8415002001
:1023D000F8B5054616460846EFF3118C202383F323
:1023E0001288BFF36F8F19490B684BB1184C6268A4
:1023F0009A4205D000221A6062689AB9C4E9003393
:10240000144A13682BB157681C681460BB4208BF9C
:1024100054608CF31188BFF36F8F0B602BB9184693
:102420003360F8BD13606360EAE75C68A042D8BF20
:1024300000F1FF3403F10801224628460BF025FE87
:1024400000232B55601C0123EAE700BF3011002058
:102450003C1100203411002037B52449244A0023C0
:10246000C1E90033C2E90033224A1C4648681460BF
:1024700088B9C1E900220133082B02F18802F5D1A5
:102480001D4D1E4828600AF004FB38B94FF0FF3498
:10249000204603B030BD02604A60ECE70020FEF742
:1024A00073FF04460028F1D12868836823B11B6CB0
:1024B00013B113492246984728688368DB6A0BB139
:1024C000984748B1286883681B69002BFAD001221D
:1024D0000DF107019847F4E70A4B286800221A809B
:1024E00083681B6A002BD3D09847D1E73C110020AA
:1024F00034110020441100208415002058E200000F
:1025000009230000B44500202DE9F04FEFB0DFF8BB
:10251000DC90DFF8DC80D9F8001041F20443ADF81C
:102520000C3040F60613ADF81030324B1E680B78B5
:102530005A1CA6EB080662F302030B7073BA4B80B9
:102540008B8800245BBA8B804C700822204608F0F0
:10255000FDFEB5B23246414608F0F8FE05F10A0329
:10256000D9F800101FFA83FB5BBAADF818300B687E
:10257000CDF81A3007460DF1180A4B68CDF81E3019
:10258000324641467FBA0DF122000C350BF07DFD3D
:10259000ADB22AF80B7032AE05AF009553463A46FD
:1025A000ED213046FEF7B8F8134DBDF81480A04574
:1025B00002DC6FB0BDE8F08F2B6802215B6894B934
:1025C00004A8A8EB040798472B687C2FA8BF7C279A
:1025D000301939465B6898472B6808485B680121C9
:1025E0003C449847E3E703A8EBE700BFE015002071
:1025F000EB5E002098150020E4150020BCE90000E7
:1026000010B50A2104460A480AF013FA02220949C1
:1026100007480AF001FA214605480AF0DAF90448A9
:102620000A210AF00EFABDE81040FFF76DBF00BFA7
:10263000981500209EEA00002DE9F04FD7B00DF16B
:102640001C0A0DF124094FF0FF34CAF80040C9F804
:10265000004008940AAC00250B4601210246256083
:1026600032A80091CDE901550421CDE90C550B9517
:102670000AF026F94022294622A80BF02DFD8F4BA7
:102680001E9305231F938E4B8E4808AECDE920364E
:102690008D4B23938D4B0DF13008CDE925388C4BB4
:1026A00028938C4B0321CDE92D01CDE92A39CDE9C1
:1026B0002F3A042229910BAB1EA932A8249208F0CC
:1026C00097FD002842D1DAF800305A1C3ED00C9F0A
:1026D000002F3BD0DDF834807F4A2BB90899B1F147
:1026E000FF3F18BF0B4613601068002107F01EFF64
:1026F0002146C0B2FEF724FA064638BBDAF80010CD
:10270000764DD9B9236828609A68D9F80030934289
:102710001CD8734A1060734A41461360D4F800B065
:10272000DFF8BCA1DBF80830DAF8009001399942F3
:102730000ED36FF01503CAF8003007E02B689942FA
:1027400065D1684B1B6841449942E7D903265EE096
:10275000894519DC0EAA584607F0F0FE034600280A
:10276000E7D1DDE90E128A1805924946A2EB09026B
:10277000584608F0E2FC024620B15B48452108F0CB
:1027800047FAD6E7DDF81490CAF80090B9F1000FC7
:10279000DCDB206808F095FAB8FBF0F303FB00FBE4
:1027A0002B682068A8EB0B0A98444E4B1B68984591
:1027B00038BF4FF0000A08F084FA0128D94605D93D
:1027C000206808F07EFA0138074254D12968206851
:1027D0005B463A4608F04BFA0028B7D143E0C845BB
:1027E000206828BFC84608F073FA402201460EA8A8
:1027F0000BF072FC424639460EA80BF046FC2968E5
:10280000206843460EAA08F032FA08B306460A21A9
:1028100036480AF00EF93649344802220AF0FCF82C
:10282000324831460AF0D5F84EB926492F480322DE
:102830000AF0F2F8294B2D4819680AF0D4F80A2159
:102840002A480AF0FEF8FFF75FFE57B0BDE8F08FA8
:102850002B6843442B604744A9EB0809206808F023
:1028600030FA4845BBD9BAF1000F07D12B68534461
:102870004B442B60CBE74FF04008EFE7206808F0AF
:1028800027FA082201460EA80BF026FC524607EB59
:1028900009010EA80BF0F9FB27682968384609EBF7
:1028A000010408F00EFA0EAA03462146384608F045
:1028B000DEF900287FF44AAFD8E700BFA1EA0000A4
:1028C000EFC60000B0EA0000A7EA0000F9C6000069
:1028D000ACEA0000F5C60000941500209015002019
:1028E0008C15002088150020B4EA000098150020FF
:1028F0009EEA0000F0B50C68164F174B85B0023801
:102900000D46C4F58061009003AA38190131FDF726
:1029100083FF0446D0B92B68039A1344022B2B6023
:1029200011D93E8876BAB6B2023B9E420BD13246EE
:10293000B91C08F00BFD30B9022E04D92B689A1E81
:102940002A60FC540124204605B0F0BD4FF0FF344E
:10295000F9E700BF905F00209363002007B50023D4
:102960000093044A0448A42302210AF06CF803B03F
:102970005DF804FBEB5E002098150020F0B50729F8
:10298000ADB0044640F21681037813F0050F40F015
:10299000118143885BBAA1F108059BB2AB42C0F03C
:1029A0000981854B186083885BBA8380FFF7D6FF67
:1029B000A688012E40F0E480E37923B1012B00F0DA
:1029C000D7800820F1E02778FFF756FC054608F08D
:1029D000F7FB284608F0F8FB07F00707024680B12E
:1029E0007648452108F014F93446284608F0A2FB41
:1029F00014B12046FFF704FE2DB0BDE8F040FFF70C
:102A0000ADBF01462846FFF721FC044648B1024607
:102A100045216B4808F0FCF83446284608F0D9FBFD
:102A2000E3E7002F40F0A280314666480AF001F843
:102A300065496448062209F0EFFF6248052109F064
:102A4000F4FF2E6A002E6BD0604B0CAA1F68214643
:102A50002023304608F0F6F85D4B0C9A9A420CD1D0
:102A60000023CDE9023301934023009332461CAB8F
:102A70000CA92846FFF7F8F90746564B1B68BB42DE
:102A80004ED10023009332464FF6FF730CA906A8DF
:102A900008F085FA00284ED04FF0FF36142149483F
:102AA00009F0C7FF4C494748042209F0B5FF4548E3
:102AB000002109F098FF4EB948494248042209F024
:102AC000ABFF4048202214A909F09DFF44493D482E
:102AD000072209F0A1FFBDF8463001931CAE9DF816
:102AE000453000933F4A9DF844304021304607F07E
:102AF00081FB129B43B1421E3E2A05D8C0F1400122
:102B0000394A304407F076FB3046FDF763FB314627
:102B100002462C4809F080FF2A48142109F091FF51
:102B20000521284809F089FF0121264809F089FF7D
:102B3000FFF7EAFC71E70DF1120304AA05A906A844
:102B400008F07BFA0028A7D1BDF81230102BF2D183
:102B5000BDF81030202B9FD13046059914AA08F0FB
:102B600071F8061E18BF0126764297E7082454E73D
:102B7000294604F108002DB0BDE8F040FFF75CBD28
:102B8000002E7FF41EAFE379012B0DD0052B7FF4CF
:102B900018AF3046FFF734FD4FF4005000210AF023
:102BA000D4F90120FDF7A2FD30462DB0BDE8F0407C
:102BB000FFF726BD2DB0F0BDE0150020D6EA0000DD
:102BC000FAEA0000981500201AEB00009801002096
:102BD0003DB8F396F410002021EB000026EB000036
:102BE0002BEB000033EB00003FEB00002DE9F3413D
:102BF0001F4F204E01233B701F4B002405460094BD
:102C000018603B7813B902B0BDE8F08140F201488A
:102C1000FDF72EFD2B6801AAA8EB04013019984797
:102C20000028019B0FDC002BEBD004443378062BEB
:102C300010D17378092B12D1002300936946A01E8E
:102C4000FFF758FE0BE00444002BEFD14445D8D1E8
:102C50000024D6E7042B02D17378142BEED0012880
:102C6000F6D1009905480239FFF788FEF0E700BF6A
:102C70008F5F002091630020E4150020925F002008
:102C8000BFF36F8F72B6124B4FF0FF32C3F8802044
:102C9000C3F88420C3F88820C3F88C20C3F89020A0
:102CA000C3F89420C3F89820C3F89C20C3F880216F
:102CB000C3F88421C3F88821C3F88C21C3F890217C
:102CC000C3F89421C3F89821C3F89C21704700BF32
:102CD00000E100E008B50348034A0021121A08F099
:102CE000DDFA08BD10040020C06700200748084A2C
:102CF000084908B5121A08F0D3FA0748074A0849E4
:102D0000BDE80840121A08F0CBBA00BF000000204E
:102D100010040020D0EE0000000000200000002081
:102D2000D0EE000030BFFFF7FDBF00BF2DE9F0413E
:102D30000B4EDFF8308006EB0807CC1B0546324609
:102D4000094920460BF0A1F9A01942460021083C90
:102D50000BF0C2F92C6707F10800BDE8F08100BF55
:102D60000000000008000000D8E50000134B9A6A3C
:102D700012F0007F9A6A14BF1E201D2012F0807F7F
:102D80009A6A18BF1F2012F4002F9A6A18BF2120D8
:102D900012F4802F9A6A18BF222012F4003F9A6A18
:102DA00018BF232012F4803F9A6A6FEA02426FEA4A
:102DB00012429A6218BF2420704700BF00ED00E065
:102DC00010B5194B0246986A9C6A10F4805F14BFD4
:102DD0001720162014F4006F9C6A18BF1820A40551
:102DE00009D5986B986A000404D51AB19A6A22F43E
:102DF00000429A6219200C4B9A6A12F4806F9A6A08
:102E000018BF1A20D2050CD49B6A13F4005F18BFB8
:102E10001C20054A936A43F47F43936200230B709E
:102E200010BD1B20F5E700BF00ED00E010B51C4B06
:102E30000246986A9C6A10F0100F14BF11201020EF
:102E400014F0080F9C6A18BF1220A40709D5586B0C
:102E5000986A000604D51AB19A6A22F080029A6232
:102E600013200F4B9A6A12F0010F9A6A18BF1420B0
:102E700012F0200F9A6A18BF1520D40658BF9B6A1B
:102E8000074B9A6A920642BF5A6A22F400525A626B
:102E90009A6A42F0FF029A6200230B7010BD00BFD5
:102EA00000ED00E0F0B5494B5B688BB00446C3F31E
:102EB0000803002585F31188BFF36F8F02F07F4070
:102EC000B0F17F4F11D102F00C0008280DD010078F
:102ED0004CBF0C4601250022033B8DF80720032B35
:102EE00005D8DFE803F024676B642C46F3E7002382
:102EF0009DF80720CAB902AE04F120072068616876
:102F0000324603C20834BC421646F7D1099A002D56
:102F100058D0C2F3080121B96FEA52226FEA422267
:102F2000099202A9184608F0BDF90BB0F0BD274B75
:102F3000DA6A9107DBD4DA6A002AD8DBDA6A52004F
:102F4000D5D55A69A16942F480725A61BFF34F8F97
:102F5000BFF36F8F31F8022C596921F480715961E8
:102F6000BFF34F8FBFF36F8F02F47F43B3F55F4F13
:102F700004D1D2B2022A01D12368B9E7134B9A6A6D
:102F8000D2B232B10DF107010120FFF74FFF034626
:102F9000AEE79A6A12F47F4F05D00DF107010120C8
:102FA000FFF70EFFF3E79B6AB3F5803F9FD3FFF770
:102FB000DDFEECE70DF107010020E6E70DF107016A
:102FC0000020EDE76FF30802AAE700BF00ED00E084
:102FD000044B5A6942F010025A615A6922F0080201
:102FE0005A61704700ED00E0EFF30880EFF30981CC
:102FF00001B57246FFF756FF01BD00BF0B4880F3D5
:10300000088803F0B9FC202080F3118808484FF4A9
:103010000061401880F30988EFF31480022108430F
:1030200080F31488BFF36F8F00F07EF800A10020BA
:10303000C06F00200749D1F890200023C2F3072277
:103040001846934200DB7047C1F89830C1F8A000E1
:103050000133F6E700ED00E01EF0040F0CBFEFF3C4
:103060000880EFF30980816911F8021C0229FFD062
:1030700001B5724608F01CF901BD00BF40B200283E
:1030800007DB044A4109012300F01F00834042F896
:103090002130704700E100E040B200280CDB43091A
:1030A000064900F01F0020330122824041F823200E
:1030B000BFF34F8FBFF36F8F704700BF00E100E099
:1030C000054B420900F01F0053F82220012303FAA8
:1030D00000F01040704700BF00E100E040B200285F
:1030E000A8BF00F1604001F10101B8BF064B4FEAF3
:1030F0004111ACBF00F5614000F00F00C9B2B4BF90
:10310000195480F80013704714ED00E0044B054A91
:1031100023F07F039360BFF34F8FBFF36F8F704730
:103120000000000000ED00E008B5FFF7EFFF0B4ADC
:10313000D2F8883023F47003C2F88830EFF3148398
:1031400023F0040383F31488BFF36F8FFFF7C2FDEE
:10315000FFF7CCFD00F092F804F09EFE00ED00E0D9
:1031600042F8203C009B42F81C3C0A49019B42F873
:10317000183C029B42F8143C21F001014FF080738F
:1031800042F8043C42F8081C0023203A02654367D9
:10319000704700BF351E000000B50B4B98600B4B0D
:1031A0001546026F1A600E462C4686F309880020E9
:1031B000034B98472046002100220023014C204762
:1031C000D5B20000351E000018220020E8150020AE
:1031D000014B10221A61704700ED00E0054B5A695F
:1031E0009B689A421FBF044A536843F08053536060
:1031F000704700BF1822002000ED00E0084B9B68DC
:1032000083420BD1EFF3058343B1064B5A6842F07A
:1032100080525A605A6A22F400425A6209F0D3BDC1
:103220001822002000ED00E011498A684FF03000BC
:103230001044EFF3098C80E8F01F202080F31288FF
:10324000BFF36F8F0B4F4FF000664A698A603E6094
:10325000106F094C2060506F0023536780F3118872
:1032600002F1300090E8F01F8CF3098870470000ED
:103270001822002004ED00E0E81500200448002397
:103280002021C2180133302B82F80013F9D1704786
:1032900000E100E008B5EFF30583064A103B02EBBE
:1032A000C30152F8330049688847BDE80840FFF77A
:1032B00095BF00BF1CE30000014800687047000094
:1032C000E8150020024B034A0348012100F066B8CC
:1032D000000004200000002054E60000084AC2F864
:1032E00098000B6823F01F03034343F01003C2F858
:1032F0009C308B6843F00103C2F8A030704700BFD8
:1033000000ED00E02DE9F043DFF8608085B00E4667
:103310001F4604464FF00009B14523DA6068D8B172
:103320003FB1411E08421BD11F2819D923681942F9
:1033300016D12368019307F0F0FFA36803430393BA
:10334000D8F89050C5F30725D0B2013DA84207D860
:1033500001A9FFF7C3FF421C09F101090C34DBE7A7
:103360006FF01502104605B0BDE8F08300ED00E0F7
:10337000044B0522C3F89420BFF34F8FBFF36F8F28
:10338000704700BF00ED00E0BFF35F8F024B0022EB
:10339000C3F89420704700BF00ED00E010B5034C67
:1033A00001232278FFF7AEFF207010BD9267002046
:1033B0002DE9F0435A4B5B4DD3F890302C68C3F3A2
:1033C00007239C4285B000F2A780FFF7DDFF0020B5
:1033D0000C2684421AD1544EDFF84491347068466A
:1033E000FDF7A8FB514C524D80460027B84514D13B
:1033F00033784B490020D1F89020C2F30722934242
:10340000C0F28480FFF7B4FF002045E0696806FB46
:103410000011FFF763FF0130DBE7009800EB0711B5
:103420004FEA071CCB682340B3F5000F4DD00AD8F4
:10343000B3F5001F33D0B3F5800F3BD0B3F5801F39
:1034400013D00137D2E7B3F1007F47D0B3F1805FEB
:103450004DD0B3F1807FF4D150F80C3088684A68C1
:1034600007F05BFF40F0887009E050F80C30886886
:103470004A6807F052FF40F0885040F43020CDE910
:1034800001230390D9F890303078C3F30723013B30
:10349000984234D96FF0150005B0BDE8F08350F8BC
:1034A0000C3088684A6807F038FF40F0885040F4D4
:1034B0000020E4E750F80C3088684A6807F02DFFD8
:1034C00040F0007040F40030D9E750F80C308868C4
:1034D0004A6807F022FF40F08270D0E750F80C30C5
:1034E00088684A6807F019FF40F48020C7E750F861
:1034F0000C3088684A6807F010FF2843BFE701A92D
:10350000FFF7ECFE3378013333709AE7C1F8983057
:10351000C1F8A00001336EE74FF0FF30BCE700BFF9
:1035200000ED00E060E60000926700200000F0FF80
:103530000000021108B5024806F03CFEFEE700BF9D
:1035400052EB000008B5024B1B689847002008BDED
:10355000EC15002008B5054807F096F9002383F321
:103560001188BFF36F8F0423184602DF57EB00006A
:1035700000B5FFF7A1FE034B0C221A5000205DF8A6
:1035800004FB00BF0C000000024B0122C3F84025E1
:103590000020704700E0014048B1054B054A1B6818
:1035A000B3FBF2F35843044B43F001031847704751
:1035B0007002002040420F00F0E50000BFF34F8F83
:1035C0000549064BCA6802F4E0621343CB60BFF3BF
:1035D0004F8F00BFFDE700BF00ED00E00400FA05DB
:1035E00008B5054A054B136010463F23536003F0AE
:1035F0009FFA002008BD00BFF0150020FFFF0F005C
:1036000000F07F03082B42B204D010F0780F01D0F5
:1036100000207047002A00F00F0300F0080004DAD1
:1036200030B9054800EB4310704718B90348F9E773
:103630000348704703487047441600206417002071
:1036400044170020641800200149024809F096BB85
:1036500020160020B00400200146014809F022BBDA
:103660002003002002480022002304F07FBD00BF99
:103670002003002013B5114800F0C4FE0446C8B969
:103680000F4803F097FD0F4803F0D2FD0E490F4895
:1036900000944FF0FF334FF4806204F0FBFE0C49BE
:1036A0000A4809F08DFB0B490B4809F04BFB2046FB
:1036B00002B010BD6FF00404F9E700BFC938000084
:1036C00074EE000084E60000C06B0020B00400200F
:1036D00060EB0000E53900002016002010B50E490F
:1036E000BFF35B8F002351E8002F012A03D141E88B
:1036F00000300028F7D1BFF35B8F0CD151F8044C98
:103700001439204607F0B9F9783004D12046BDE8D5
:10371000104007F08EB910BD1816002038B50024EF
:1037200064F07F00C0B2FFF76BFF013407F022FEA8
:10373000082CF5D10E4D0024E0B2FFF761FF0369BC
:1037400003B90561013407F015FE082C05F14005A9
:10375000F2D1084807F00EFE074BD3F87C2212B9CD
:10376000064AC3F87C22BDE83840054807F002BE8F
:10377000881C002044170020F8150020881800201D
:103780006418002008B5FFF76DFF20B141680248BA
:1037900009F0B7F9F7E708BDE002002007B50023FC
:1037A0000E48002201A904F0F1FB90B1FFF7EAFFF7
:1037B0000A480022002301A904F0E8FB38B9019867
:1037C000042340600374FFF747FFFFF73DFF00202D
:1037D00001E00198406003B05DF804FBE0020020C6
:1037E00010B50446FFF7DAFF60B1002202740472DC
:1037F000FFF732FF044B93F824301BB1BDE81040B3
:10380000FFF722BF10BD00BFF8150020022803D823
:10381000024B185CFFF7E4BF704700BF71EE000079
:1038200070B5817806460846FFF7EAFE0B06F57884
:10383000044612D5002D43D1FFF7B0FF0346002800
:103840003ED00122A5770274032202739C60FFF729
:1038500003FFBDE87040FFF7F7BE4DB1012D2FD13A
:10386000FFF79CFF034658B3657705740573EDE7D2
:10387000FFF794FF20B3B278124B12F0800F02F0E2
:10388000080111D041B1D3F8A836E36001230374D5
:10389000022303738460DAE702F00F02142101FBB4
:1038A0000233D3F80836F0E711B1D3F8A837ECE7C4
:1038B00002F00F02142101FB0233D3F80837E4E7CA
:1038C00070BD00BF00700240F0B5064689B01422FA
:1038D000002103A80AF000FC3378013B052B21D816
:1038E000DFE803F07A0314146A1603238DF814300A
:1038F0000024FFF753FF0346A0B1047400F108024F
:10390000DDE9050182E8030018461DE00423EDE728
:10391000B1780846FFF774FE837A044623B1013B71
:10392000022B43D909B0F0BD0B06F57813D5002D55
:10393000F8D1FFF733FF03460028F3D00122A57723
:103940000274032202739C60FFF786FE09B0BDE893
:10395000F040FFF779BE55B1012DE3D1FFF71EFF0F
:1039600003460028DED0657705740573EBE7FFF7A3
:1039700015FF07460028D5D00123037402230373E3
:10398000846004F10C01B07807F062FD134AE1682D
:10399000B2F88C328B4206D95B1AA2F88C3201F055
:1039A0007DF83846D0E7A2F88C52FAE7304609B0E5
:1039B000BDE8F040FFF734BF01A801F04DF89DF8D5
:1039C0000530052B04D19DF8043013F0600FA9D009
:1039D000034B059301248CE702248AE7F8150020A5
:1039E000641700202DE9FF41AD4C8046FFF73AFEF9
:1039F000074610B904B0BDE8F08194F825303A7C50
:103A00003BB9002A00F085807968A64809F079F86A
:103A1000ECE7042AF8D8DFE812F07C000500020188
:103A2000180133013B7BBD68032BEDD8DFE803F0C1
:103A3000023C595E6E699C4B002232607260D3F882
:103A400080143170D3F884147170D3F88814D3F8CB
:103A50008C0441EA00217180D3F89014D3F89404C7
:103A600041EA0021B180D3F89814D3F89C3441EA9C
:103A70000323F3800823EB60306871688B4B03C32A
:103A800011462B68687A984796F90030002B07DBBF
:103A9000F3889AB222B1A4F88C3200F0FFFFB3E7AA
:103AA0000023A4F88C32AFE76B7F002BACD02B7FC8
:103AB000002BA9D000266E774FF0FF327C482E777E
:103AC0004FF0FF3307F069FC6B6901936B68CDE938
:103AD000023601A9687A00F0E7FC754807F05FFC40
:103AE00092E72B680121687A98478DE7AB7A6BB92A
:103AF000EB7F5BB96E484FF0FF324FF0FF3307F0BA
:103B00004CFC00F0D1FF6A4807F049FC2B68022109
:103B1000E9E73A7A042A3FF677AFDFE802F05B0381
:103B20002569750000F02EFC054600287FF46CAF77
:103B300000F068FBBFF35B8F5E49012351E8002F63
:103B4000002A03D141E800300028F7D1BFF35B8F92
:103B50007FF45AAF41F8085C41F8105CE06963619A
:103B6000143906F01BFF4FE7002565F07F00C0B257
:103B7000FFF746FD037A13B1407A01F0F7F80135FB
:103B8000082DF2D194F854311BB194F8550101F08D
:103B9000EDF80025E8B2FFF733FD037A13B1407A60
:103BA00001F0E4F80135082DF4D194F874321BB11A
:103BB00094F8750201F0DAF8002000F0C7FB012349
:103BC00084F825302368002B3FF41EAF002102202B
:103BD000984719E7002584F8255001F02DF8FFF7E4
:103BE0007DFD2368002B3FF40FAF29460420EFE74B
:103BF000002B3FF409AF00F0CFFB2368002B3FF40C
:103C000003AF00210520E3E72268002A3FF4FCAE61
:103C1000002B3FF4F9AE002106209047F4E608F1AE
:103C200010054FF0FF334FF0FF32284607F0B5FB89
:103C3000FFF774FD284607F0B2FB58F8283C002B2C
:103C40003FF4E2AE00210120C2E794F874327BB168
:103C5000012584F8895284F88852FFF79FFD38B116
:103C6000154A057405738260FFF7F6FCFFF7ECFC5C
:103C700058F8283C002B3FF4C7AE00210A20A7E7E4
:103C800008F019FB00F0D8FF00F0B2FAFFF77AFD58
:103C9000FFF744FD08F008FB084800F0B3FBB3E66B
:103CA000F8150020E002002000700240FC15002002
:103CB000301600201816002064180020C9380000B3
:103CC00038B5144C94F824500DBB04F1380008F0BA
:103CD00062FF284601F076FC2A460121E061272098
:103CE000FFF7FCF908F0E0FAFFF718FD012384F86C
:103CF0002430094B1B680BB1FFF7A6FC4FF0804343
:103D0000D3F83834DB0702D50120FFF769FD002026
:103D100038BD00BFF81500202003002010B50D4865
:103D20004FF0FF324FF0FF3307F037FBFFF72AFD6C
:103D300000F028FB08B100F07FFFFFF7CFFC08F090
:103D4000BAFA0548002480F82440383007F027FBF1
:103D5000204610BD30160020F8150020074B93F8C0
:103D600024203AB193F82530002B0CBF6FF01200DD
:103D7000002070476FF01200704700BFF815002058
:103D800010B5104B93F824300146BBB1047820469F
:103D9000FFF736FC10B96FF0150010BD44720B79B7
:103DA00083724B88436008784988030702D44B1E0E
:103DB0000B42F0D107F047FB0020EEE76FF0120056
:103DC000EBE700BFF815002010B5124B93F8242044
:103DD0000146CAB193F82530B3B1FFF711FC044690
:103DE000A8B1837A012B12D007D9023B012B07D946
:103DF0006369A3610020E06010BD00F05BFEF7E79F
:103E0000084600F0FDFDF3E76FF01200F4E76FF0F5
:103E10001500F1E7F815002038B50E4B93F8242073
:103E2000054682B193F825306BB1FFF7E9FB68B125
:103E300015F008040AD1284600F004FE284600F0D8
:103E4000CDFF204638BD6FF01200FBE76FF0150084
:103E5000F8E700BFF815002038B50C4B93F8242084
:103E600005460C4662B193F825304BB1FFF7C8FB0D
:103E700048B141B1284600F0CBFD2070002038BD8C
:103E80006FF01200FBE76FF01500F8E7F81500205F
:103E900070B5134E96F824300446C3B1FFF7B0FB5B
:103EA0000546B8B1230705D4204600F0CBFD2046D7
:103EB00000F094FF2B7A83B901232B7296F82530FA
:103EC0000BB9002070BD204600F050FFF9E76FF0FD
:103ED0001200F7E76FF01500F4E76FF07700F1E7F5
:103EE000F81500202DE9F043DFF8DC801F4698F834
:103EF000243085B0044689461646002B5DD098F8DC
:103F00002530002B59D003065AD5FFF779FB05461B
:103F1000002855D0037A002B52D04FF0FF334FF0DA
:103F2000FF3208F1380007F038FAAB7F4BB108F1E7
:103F3000380007F034FA6FF00A04204605B0BDE8F7
:103F4000F08316B9EB7F03B1EE77AB7ABBB95EB104
:103F5000B8F80A30B34207D96A68B6FBF2F302FB3D
:103F600013630BB90123EB7700F0AAFDA04206D042
:103F700000F09AFD154807F012FA0024DDE701234E
:103F80002046AB774FF0000801A9CDE90196CDF8A6
:103F90000C8000F089FA044658B185F81E802FB9CC
:103FA0006FF00404094807F0FAF9C6E7C7F8008083
:103FB000F6E7002FF6D03E60F4E76FF01204BCE79E
:103FC0006FF01504B9E700BFF81500203016002087
:103FD0002DE9F0411D46204B174693F824200E464C
:103FE000002A33D093F8253083B3030631D401B9C6
:103FF0007FBBFFF705FB044658B3037A4BB34FF082
:10400000FF3316484FF0FF3207F0C7F9E3689F42CD
:10401000B84628BF984646B93FB905B12B600F484E
:1040200007F0BDF90020BDE8F081A16942463046A5
:104030000AF02BF8A3694344A361E368A3EB0803E8
:10404000E360002DEBD0C5F80080E8E76FF01200C8
:10405000E9E76FF01500E6E7F815002030160020BC
:1040600070B51E4D95F82420034682B395F825209F
:104070006AB31B062ED4FFF7C3FA044650B3037A83
:1040800043B34FF0FF334FF0FF3205F1380007F034
:1040900084F9E368B3B9012663692677A361637F76
:1040A00083B1FFF77BFB30B905F1380007F077F9F2
:1040B0006FF00B0070BD067484600673FFF7CCFAD6
:1040C000FFF7C2FA064807F06AF90020F2E76FF03E
:1040D0001200EFE76FF01500ECE700BFF8150020C5
:1040E0003016002008B5084B93F824302BB1FFF7A9
:1040F00087FA28B10160002008BD6FF01200FBE7CD
:104100006FF01500F8E700BFF8150020014B1860AC
:10411000704700BFF815002008B5074B93F824300E
:1041200023B1FFF76DFA20B1406808BD6FF01200AF
:10413000FBE76FF01500F8E7F8150020064B10F0CC
:10414000800F03F1D80218BF134600F00F001822A9
:1041500002FB0030704700BFC81E0020EFF3118043
:10416000202383F31288BFF36F8F0A4BD3F8001C10
:10417000032261B949F27531C3F8001CC3F8142D4C
:10418000C3F8001C80F31188BFF36F8F7047C3F82A
:10419000142DF7E700E00640EFF31180202383F3AE
:1041A0001288BFF36F8F0A4BD3F8001C61B949F234
:1041B0007532C3F8002CC3F8141DC3F8002C80F32B
:1041C0001188BFF36F8F70470022C3F8142DF6E7F4
:1041D00000E006404FF08053D3F83031082B02BF87
:1041E000024B0022C3F81C2C704700BF0070024035
:1041F000024A00231360024A137070478020002097
:104200009767002008B54A4B4FF40062C3F80024BA
:1042100007F003F908B1FFF7A1FF4FF08053D3F87F
:104220003031082B18D1EFF31180202383F312884B
:10423000BFF36F8F3F4BD3F8001CC02200296ED113
:1042400049F27531C3F8001CC3F8142CC3F8001CE4
:1042500080F31188BFF36F8F354B0122C3F800251F
:10426000D3F800241205FBD54FF40062C3F80024F4
:104270004FF08053D3F83031082B17D1EFF3118072
:10428000202383F31288BFF36F8F2A4BD3F8001CCF
:10429000002947D149F27532C3F8002CC3F8141C29
:1042A000C3F8002C80F31188BFF36F8F07F0B5F8C7
:1042B00030B1FFF771FF07F0B0F808B1FFF74EFF1C
:1042C0004FF08053D3F83031082B194B0AD140F20C
:1042D000E372C3F800284022C3F80428BFF36F8FAD
:1042E000BFF34F8F8022C3F81C250122C3F830256D
:1042F000114B40F2FF121A60104B00211960104B55
:104300001970FFF767FF0F4B19700F4B02221A70DD
:1043100007F083F850B1BDE80840FFF73DBFC3F890
:10432000142C95E70022C3F8142CBBE708BD00BF8E
:104330000070024000E006407C2000207820002031
:10434000936700209567002097670020094B0022A3
:1043500010B51A70084A094B094C002808BF1346CB
:10436000C4F800332720FEF789FE0123C4F8043582
:1043700010BD00BF96670020FDFFDF01FDFFFF01BC
:1043800000700240034B1878012894BF00200120E0
:10439000704700BF9767002010B54FF0FF324FF015
:1043A000FF33154803F048FFEFF31181202383F317
:1043B0001288BFF36F8F114B1B7803F0FF0483B19A
:1043C0000F4BD3F8002412F400720AD10120C3F875
:1043D0002C05D3F82C05D3F80004800502D5C3F8CA
:1043E0002C25002481F31188BFF36F8F024803F05E
:1043F000EFFE204610BD00BF10030020966700208E
:1044000000700240F8B51C4B1C7894BB1B4A10602E
:1044100001221A7040F2FF17264664F07F0514F05F
:10442000080FEDB214BF39464021284607F00BF8BB
:104430002846FFF783FE0134092C86750673066152
:10444000EBD1002440F2FF17254614F0080FE6B226
:1044500014BF39464021304606F0F5FF3046FFF7DD
:104460006DFE0134092C857505730561EDD10020C1
:10447000F8BD6FF07700FBE79767002080200020F1
:10448000084B10F0800F14BFD3F81035D3F8143553
:1044900000F00F02012090401840003818BF0120A2
:1044A000704700BF007002402DE9F843024606F055
:1044B000C2FFEFF31188202383F31288BFF36F8FBD
:1044C000130703D1174B1B78934224D1164B174F78
:1044D0001C683E68E4434FF00109A4B209FA00F5F4
:1044E00034432C401AD11046FFF728FE80F80C9078
:1044F000034607C91C6183E807009C750C4B2E43DB
:1045000080223E602046C3F8042188F31188BFF35F
:104510006F8FBDE8F8836FF00D00F6E76FF00F00C6
:10452000F3E700BF956700207C2000207820002062
:1045300000E100E010F0080F074B06D0D3F8C004EC
:1045400010F4803F18BF0020704700F00F0000F506
:10455000947053F820007047007002402DE9F74F27
:10456000594BDFF86881D3F85421EAB10022C3F82F
:104570005421D3F80413890216D58DF80420D3F8FA
:104580002025ADF80620D3F8C034002BD8F8003031
:1045900014BF4FF001224FF480721343C8F800306B
:1045A0004B4B01A81B689847474BD3F8604134B187
:1045B0000022C3F86021D3F86C44C3F86C44D3F8EC
:1045C00028214AB10022C3F82821424B187806F06E
:1045D00032FF012383401C43DFF8FCA09AF800500F
:1045E0009AF9006015F0080005F00F0238D1002E8E
:1045F000B4BF3A4B3A4B91000B441968DFF8E49092
:1046000051B300211960304B88BB8E424FF014012A
:1046100001FB0233B4BFD3F80836D3F80837324A67
:10462000117803F001034B401370FFF7D3FD2F48BF
:1046300003F0CEFD2846FFF781FD837D032B1DD1BE
:10464000284606F0F8FE012303FA00F0D9F80030FE
:1046500023EA0003C9F800301D4F0125062672E049
:10466000234B244933EA260328BF0B46C5E7002E17
:10467000B4BFD3F8A836D3F8A837D0E7037BE3B9A3
:10468000284606F0D8FE012303FA00F0D9F80030DE
:10469000002E23EA0003C9F8003001DA882DDBD1AF
:1046A00006238DF8043000238DF80730084B8DF871
:1046B00006501B6801A89847CEE7002DCCD1024BCD
:1046C0000122DA64C8E700BF007002407C200020AD
:1046D0008020002095670020946700200871024028
:1046E00030710240782000209367002010030020E2
:1046F000507102402C71024094FAA4F3B3FA83F390
:104700000F2BD8F800201946C8BFA3F1100105FAF5
:1047100003F342EA0302C8F80020D9F80020CCBF16
:10472000C9B241F0800124EA030413400A0640F1B3
:10473000938043B98DF804608DF806108DF807302A
:104740003B6801A89847002CD6D1A74BD3F800218D
:104750005AB1C3F80041A54B1C70A54B1C70012336
:104760000193A44B01A81B6898479F4BD3F858218D
:10477000002A2ED00022C3F85821D3F80044C3F8F1
:104780000044E60508D5994B01221A7002230193D3
:10479000984B01A81B689847A50508D5934B0022A4
:1047A0001A7003230193934B01A81B689847640573
:1047B0000FD58E4B1A7862B100221A708A4B0122F3
:1047C000C3F808259A65042301938A4B01A81B6846
:1047D0009847854BD3F85C3123B3874B9B681BB953
:1047E0009AF8003058061DD07F4B0022C3F85C2198
:1047F000D3F880347E4A23F07F031370D9F8003059
:1048000023F00113C9F80030D8F8003023F48033C6
:1048100043F00103C8F8003005230193754B01A84C
:104820001B689847D9F80020D8F800301A4200F0E9
:10483000C88071480022002303F0FEFC002840F0ED
:10484000C080694BD3F82C35002B44D06A4803B0A4
:10485000BDE8F04F03F0BCBC002B7FF474AF8DF8C3
:1048600004608DF806108DF8075069E70B4661E08B
:10487000003A69E02046FFF75DFED5E90032B5F861
:1048800014C090429FBF121AC7182F606A6094BF6D
:104890000746002760450CBF4FF0010C4FF0000C9D
:1048A000002A08BF4FF0000C002B53D0874251D292
:1048B0000123B34021EA0303C9F8003006238DF831
:1048C00004304C4B8DF8064002221B68AA758DF807
:1048D000072001A89847D9F80010D8F800600E40CA
:1048E000B4D016F0012314BF93FAA3F696FAA6F6F5
:1048F000B6FA86F6F4B20F2EC6BF103CE4B244F00E
:1049000080042046FFF71AFC4FFA84FBBBF1000F2E
:104910000546AFDA4368878A01689F4228BF1F4671
:1049200001F06043B3F1005FA0D034483A4609F08B
:10493000ACFB324B29686A6839442960A968D21BEC
:10494000C9076A6094D53A1E18BF01222AB900220D
:104950002A7302E0BCF1000FF9D04FF08052012021
:10496000D2F83021082A02BF1F4A8221C2F81C1C3B
:10497000D8F800208AF8004000FA06F622EA06027B
:10498000C8F800202A6914F0080F3A442A61164A30
:104990001AD1BBF1000F04F00F044FF0140101FB1A
:1049A0000421A9BF0A3402EB8402C1F80037C1F820
:1049B0000477AFBF42F82400C1F80036C1F804768E
:1049C000506003B0BDE8F08FBBF1000FB5BFC2F877
:1049D000A036C2F8A037C2F8A476C2F8A477B4BF54
:1049E00050629064EDE700BF0070024096670020BF
:1049F000956700208020002010030020881E0020E2
:104A0000024B40F48070C3F81805704700700240F4
:104A1000030713D400F00F0310F0800F084A0BBFF8
:104A200003F5887303F5847302EB830252F82300C5
:104A300008BF5068003818BF012070470020704739
:104A400000700240034BC3F80C0540F48070C3F8BB
:104A50000C057047007002400023036043600E4B5A
:104A6000D3F880240270D3F884244270D3F88824C9
:104A7000D3F88C1442EA01224280D3F89024D3F870
:104A8000941442EA01228280D3F89824D3F89C340B
:104A900042EA0323C380704700700240014B0122A9
:104AA000DA64704700700240014B01221A657047BA
:104AB00000700240014B01225A65704700700240AD
:104AC000014B1878704700BF9567002010B502466B
:104AD000EFF31184202383F31288BFF36F8F06F066
:104AE000AAFC0B49012303FA00F00B6823EA000338
:104AF0000B6012F0080101BF02F00F02054B02F536
:104B0000947243F8221084F31188BFF36F8F10BDA5
:104B10007C20002000700240F7B50146EFF31185BC
:104B2000202383F31288BFF36F8FFFF707FB06463E
:104B3000084606F080FC012211F0800F02FA00F214
:104B40002D4818D1036832EA03040AD00846FFF75B
:104B5000BDFF0323B37585F31188BFF36F8F03B0D7
:104B6000F0BD2649347323EA020303600B6823EA8D
:104B700002030B60EDE70B0715D48029204B2FD0E3
:104B800001F00F0404F2DA346400C3F80048D3F8EB
:104B90000448D3F80478E4B244F002043C43C3F878
:104BA0000448D3F80438154F04683B6864EA030CE2
:104BB0001CEA020FCFD013433B600023337303235F
:104BC000B3758DF807300F4B8DF8061024EA0204F8
:104BD000062204601B688DF8042001A89847BAE7F4
:104BE00040F2B474C3F80048D3F80448D3F804780A
:104BF000E4B244F00404D1E7782000207C200020B7
:104C0000007002408020002010B504464FF0FF32B3
:104C10004FF0FF33064803F00FFB2046FFF77CFF01
:104C2000034803F0D5FA034B8022C3F8042110BDDA
:104C30001003002000E100E0F8B54FF0FF324FF024
:104C4000FF332B4803F0F8FA2A4B8022C3F8842163
:104C50002720FEF735FA98B1274E284B34681B6899
:104C60006FF30F041C43012764BB254D40F2FF1373
:104C700033602720C5F80445FEF70EFAC5F8004357
:104C8000204A13788BB11E4B0021C3F80811012173
:104C9000C3F80026C3F804165960D3F80811002998
:104CA000FBD00021C3F808111170154B0022C3F886
:104CB0000025FFF78FFA0E4803F08AFA124B012203
:104CC0001A70F8BD94FAA4F5B5FA85F50F2D2846AB
:104CD000C6BFA5F11000C0B240F08000030701D4A8
:104CE000FFF71AFF07FA05F524EA0504BCE700BF41
:104CF0001003002000E100E07C200020782000204C
:104D000000700240936700209767002010B50446AA
:104D10004FF0FF324FF0FF33114803F08DFA204679
:104D2000FFF7FAFE04F00F02012393400D4A14F03E
:104D3000800F14BFD2F81015D2F814156FEA0303D0
:104D400015BF0B400B40C2F81035C2F814350448AB
:104D500003F03EFA044B8022C3F8042110BD00BFCB
:104D6000100300200070024000E100E070B504462E
:104D7000FFF786FB68B904F00F02012514F0800FDD
:104D8000144B05FA02F205D0D3F810150A43C3F804
:104D9000102570BDD3F814150A43C3F81425631EFB
:104DA000062BF6D8EFF31186202383F31288BFF386
:104DB0006F8F2046FFF78AFE204606F03CFB064A2E
:104DC0001368854023EA0503136086F31188BFF357
:104DD0006F8FDEE70070024078200020030610B5D8
:104DE000044605D4FFF714FE10B12046FFF76EFE0F
:104DF000014BC3F8184510BD00700240142870B56F
:104E000003460C4612D80B4A12F81010D4E90005DC
:104E100002EB4302A0FB01065278002301FB05616F
:104E2000FBF76EF9C4E90001002070BD6FF01500BA
:104E3000FBE700BF75EE000030B585B0002301939D
:104E4000CDF807304B798DF80B300B7913F0200536
:104E500019D08A797F2A08BFFF228DF80C20C3F36E
:104E6000040203F01F03072B8DF80D2015D80A78D4
:104E70000C2A12D8DFE802F00C09151117111911CC
:104E8000111B1D111F00FF22E7E701228DF80620EC
:104E90004A78032A11D0042A12D06FF0150005B009
:104EA00030BD0222F2E70322F0E70422EEE70522FA
:104EB000ECE70622EAE70722E8E701228DF807205F
:104EC0004A8844F20A00824228D843F6FE708242A1
:104ED00003D8002AE1D102222FE0A2F57F523F3A07
:104EE0000B2ADAD801A050F822F000BF754F00005D
:104EF0009B4E00009B4E00009B4E00003F4F000069
:104F00009B4E0000394F00009B4E00009B4E00005E
:104F10009B4E00009B4E0000D74E000044F2140050
:104F2000824225D044F22800824223D044F20F006E
:104F30008242B2D1032200E001228DF808201A48F3
:104F4000012404FA03F390F85020DBB2F5B18D7917
:104F50007F2D11D1134380F850300B7990F85120F8
:104F600003F01F0304FA03F3134380F8513009E000
:104F70000422E2E70522E0E722EA03028DF8094075
:104F800080F8502001A807F0C4F988E7134380F89F
:104F900050300B7990F8512003F01F0304FA03F30B
:104FA00022EA0303E1E700BFB000002010B50B4C7C
:104FB00094F83A3023B1BDE81040094802F00ABD28
:104FC00002F05AFC40B16FF00403636204F1140074
:104FD000BDE8104006F052BA10BD00BFB00000207E
:104FE000E54F0000F8B50378002B40F09480514C59
:104FF000E36A94F850701F42254607D1A36A002B3C
:105000003FD14D48BDE8F84006F038BA94F8981002
:10501000A26D94F85160A1B90121DBB20B420BD013
:105020000F4208D016EA010CB2F9000024D000EBC0
:10503000D070401010800232490089B2B942EDD9D7
:10504000DCE73340018915D002EB41019142D5D014
:10505000B2F9003003EBD3735B1022F8023BF5E7A3
:1050600032F91360002EB8BF22F8130001338B42CF
:10507000F6DBC3E71846FAE70028B8BFA2F800C07D
:10508000D9E7236C43B1B4F84C202C492C489847FD
:1050900001280BD0022831D0B4F84C30B4F84820A5
:1050A0009A422BD90133A4F84C30002094F8983060
:1050B00083B994F8521018B9A36D03EB4103A365AB
:1050C000A06D02F099FB28B16FF004031A486362E7
:1050D00006F0D4F9E36B1BB9BDE8F840FFF766BFF3
:1050E000BFF35B8F55E8003F5A1E45E800210029B9
:1050F000F8D1BFF35B8F012BEEDCF8BDE36B002B27
:105100003FF47FAF94F89830002B7FF47AAF0D48CE
:1051100004F07AF875E7022B09D102F0ADFB002804
:10512000EBD004486FF00403436214306AE7052BA8
:10513000E3D166E7B0000020C4000020D8000020C2
:10514000ACE2000010010020094BBFF35B8F53E875
:10515000002F511C43E800100028F8D1BFF35B8FEB
:105160000AB9FFF723BF6FF00F025A62704700BF02
:10517000B000002010B50D490D48002207F08CFF4B
:10518000002002F065FA044660B9024601210720BA
:10519000FDF7A4FF0748C36813B9043006F06EF9A1
:1051A000204610BD6FF00404FAE700BF495100002B
:1051B00010010020B00000202DE9FF410F464FF004
:1051C000FF336E484FF0FF3203F036F87E68731EEF
:1051D000FE2B21D80024254626FA04F3DA0706D54B
:1051E00002F07EFAE040C30716D50135EDB2013476
:1051F000082CF1D185B13B7C083B062B0CD8DFE8AD
:1052000003F0140B160B040B18000221012D7A7CFD
:1052100011D0002A00F095806FF01504574806F071
:105220002DF9204604B0BDE8F0810021EEE7012110
:10523000ECE70321EAE7082AEED8DFE802F00505EB
:1052400005050505050505003B68002B79D05C6860
:10525000002C76D1186801387F2872D88DF8082084
:105260008DF809401B68464A1B01013BADF80A3026
:10527000012382F898308DF80C3002AA414B304659
:1052800002F06AFA04460028C8D13A686B0012B1ED
:10529000928902FB0333FA689A426CD3384E86F83F
:1052A000525096F89830B868B065B046002B51D08F
:1052B0003B689D890135A9B202F09EFA0446002898
:1052C000ACD1BC46BCE80F002F4D0FC5DCF8003058
:1052D0002B6074623B68002B4AD00FCB2F1D87E8F0
:1052E0000F00F36BB762A6F84C40002B40D0BFF321
:1052F0005B8F58E8003F48E80042002AF9D1BFF32D
:105300005B8F96F8981039BBF46B2048204A4FF415
:1053100000470023E4FB0701FAF742FF0022CDE932
:105320000001002305F1280003F046FF19484FF063
:10533000FF324FF0FF3302F07FFF00B17062746AFA
:105340006CE70F4B002083F898000E4B304602F0BC
:10535000CDF997E72946AFE702F08EFA0028E5D0AD
:105360006FF00403A5F12400736206F087F8DDE70F
:10537000FFF71CFEDAE76FF00B044FE7B4000020E4
:10538000B0000020E54F0000D80000203F420F0091
:1053900040420F00C4000020084B70B5C31A0D46F0
:1053A00007499B10044659430648402206F071F80D
:1053B0002B4601462046BDE8704018479820002043
:1053C000B76DDBB604E2000073B50C4C0C4A402309
:1053D000041B00930D460B460A49A4106143064680
:1053E000094806F082F8014628B130462B4602B043
:1053F000BDE87040184702B070BD00BF9820002083
:1054000057B50000B76DDBB604E200000022F8B526
:10541000012105461046FDF761FE114801F0B0FB81
:105420000446D0B9286900F0D1F901F0C9FB2F6911
:105430000C49384605F09FFA031E09DB01263E643D
:105440002D69084905F11C0005F095FA031E02DAE2
:105450001C462046F8BDEE64FBE76FF00404F8E755
:105460001955000088E600001FB500220123CDE990
:1054700002236C46074A6B46CDE9004406F064F807
:1054800028B94FF480420023684602F0D5FE04B0EC
:1054900010BD00BF69B5000010B5EFF311842023E3
:1054A00083F31288BFF36F8F074A136823F002015A
:1054B000DB07116002D4012006F0D1FB84F31188D0
:1054C000BFF36F8F10BD00BFE820002030B4104B39
:1054D0000C2202FB003301460020D3E90E529863F0
:1054E000EFF31180202484F31288BFF36F8F1C6CBC
:1054F00004F0C00444F002041C6480F31188BFF37C
:105500006F8F1DB12B46034830BC184730BC704725
:105510009820002004E20000012810B504460AD0BB
:1055200003280CD078B9084B1B6C5B070BD1BDE886
:105530001040FFF7CBBF00F057F92046F7E7BDE872
:10554000104000F05FB910BD9820002010B4EFF3B8
:105550001180202282F31288BFF36F8F17490B68E6
:1055600043F0020413F001030C601AD04FF08043A3
:10557000D3F80C14D3F80C3413F0010311D0EFF36B
:10558000118182F31288BFF36F8F0D4A136C03F001
:10559000C00343F00203136481F31188BFF36F8FDC
:1055A000012380F31188BFF36F8F1BB110BC002063
:1055B000FFF78CBF10BC012006F049BBE82000209B
:1055C00098200020024AC3B21C2000FB0320704731
:1055D00098200020F8B52A49BFF35B8F06460122C8
:1055E00051E8003F41E800200028F9D1BFF35B8F6C
:1055F00033B9244924484B60CB608A6005F0CEF96A
:10560000731E012B35D807F0D5FB044660B1012489
:10561000EFF31185202383F31288BFF36F8F1B4BA9
:105620000122C3F8802109E0194B1B78002BEED032
:105630004FF080430222C3F8082305464FF080470D
:10564000D7F81824D7F81834D20303D59B070BD00A
:10565000012E09D01CB1284605F050FED8E70021E4
:10566000212007F072FCEBE724B185F31188BFF32A
:105670006F8FF8BD4FF080430222C3F80423F8E790
:105680009420002084200020B420002000E100E0CD
:10569000BE6700200D4BBFF35B8F012253E8001F54
:1056A000002903D143E800200028F7D1BFF35B8F26
:1056B0000BD1074A0023D360064B5360032393604A
:1056C000054B1146186805F069B97047082100209C
:1056D000F0200020A1570000EC20002007B5002298
:1056E0000023CDE9002308484FF40032002303F0E3
:1056F00063FD064B186805F09CF9054B00221A6003
:1057000003B05DF804FB00BFA8020020EC200020DD
:105710000821002073B51D4D1D4CAE684C21F36867
:105720002846984770B1002323701A46217809B1A2
:10573000012A1FDD174A138006F099FA012323700E
:1057400002B070BD0C2133696A462846984700288C
:10575000E9D1114A019B93FBF2F3009A03EB820318
:105760000C4AB2F900201BB29A1A002AB8BF524262
:1057700012B2DBE7094A1368013901332170136063
:1057800002B0BDE87040FFF7A9BF00BFE4E200002F
:1057900098670020B645002090D00300002100202B
:1057A00008B5074807F075F928B906F060FA054B07
:1057B00001221A7008BDBDE80840034802F064BE2B
:1057C000E4E20000986700203C020020034B044AFA
:1057D000186000231360034A13607047EC20002018
:1057E0000421002000210020024B00221A70FFF744
:1057F00051BF00BF98670020014803F005BD00BFFE
:10580000A8020020024A136801331360FFF766BF45
:1058100004210020EFF31182202383F31288BFF3C9
:105820006F8F0A4BD3F8001161B10021D3F808053E
:10583000C3F80011D3F80031C0B282F31188BFF36E
:105840006F8F70476FF00A00F7E700BF00D000408D
:10585000F0B503468478C678EFF3118E202080F3EC
:105860001288BFF36F8F1D7893F801C0641B34401A
:10587000A24288BFA2B2AF18374028461F708EF3ED
:105880001188BFF36F8F8F188F4218D165450CD1E7
:10589000EFF31181202080F31288BFF36F8F187807
:1058A000587081F31188BFF36F8F1B79A41AA3423C
:1058B00028BF074B90B224BF01221A60F0BD03EB52
:1058C000000E01309EF805E001F801EB3040DBE707
:1058D00000D00040DB432DE9F04713F001050F46EF
:1058E000144604D02448FFF7B3FFBDE8F087B2B3F5
:1058F000EFF31186202383F31288BFF36F8F0D20FF
:10590000FDF7DEFB80460D20FDF7C6FB86F3118810
:10591000BFF36F8FDFF864A0194ECAF80051DAF8B0
:1059200000314FF400590123CAF800302546C6F86B
:105930008091DAF80031A3B1FFF76CFF031EA4BF1A
:1059400005F1FF35ADB2C6F88091A8BF7B55002D9B
:10595000EFD1B8F1000F02D00D20FDF78FFB2046EC
:10596000C3E7EFF31180202383F31288BFF36F8F17
:1059700005F0C4FCDDE700BF2C21002000D0004072
:1059800000E100E070B50D4614460CB9204670BD2C
:105990004FF0FF334FF0FF320C4802F04DFC22462F
:1059A00029460B48FFF754FF0646084802F010FC52
:1059B0003EB94FF0FF324FF0FF33064802F03CFC97
:1059C000E6E7A41BA4B23544DFE700BF0C210020AA
:1059D000412100201C21002038B501221146174822
:1059E00007F06BF9154D0122002105F1100007F0B9
:1059F00064F940F207432B874FF070632B620C234E
:105A000085F8243000240E4B85F83540EC86D3F819
:105A1000042522F00102C3F804250121C3F8004146
:105A2000D3F80021C3F80413224619600D20FDF7B6
:105A300055FB0D20FDF722FB204638BD0C21002030
:105A400000D0004010B5FFF7E5FE002820DB174B23
:105A500093F8222093F8214093F82310141B31EA85
:105A60000404C0B20DD193F8372093F8364093F870
:105A70003810141B31EA04040BD10D4B01225A607B
:105A80000EE09C180132114084F8250083F82210A2
:105A900010BD9C180132114084F83A0083F8371089
:105AA0000448BDE8104002F093BB00BF0C21002069
:105AB00000D000401C210020024B0B60012313602A
:105AC000704700BF5021002000487047ACE600003E
:105AD00010B5012211460648064C07F0EEF806F014
:105AE000D3FB206006F0CCFB6060002010BD00BF3F
:105AF00058210020502100204FF08042D2F810158C
:105B0000D2F8103501F01E0123F01F030B4343F0C0
:105B10000103C2F81035024B00221A70704700BF13
:105B2000996700204FF08053D3F83031082B20D1F3
:105B30004FF08042D2F81015CB071AD5D2F81035A5
:105B400001F01E0123F01F030B43C2F81035D2F8F9
:105B500008315BB1D2F8103523F01F030B4343F03B
:105B60000103C2F810356FF08B007047024B012221
:105B70001A700020704700BF996700202DE9F0419E
:105B80000D46164606F07CFB31460746284605F0D2
:105B900063FD78B3B5FBF7F307FB135353BBB6FBB9
:105BA000F7F407FB14642CBBB7421DD84FF0FF324B
:105BB0004FF0FF331148DFF8488002F03DFB06F05C
:105BC0005FFB0746FFF7AEFF044680B9284601F0A9
:105BD000C7FA98F800300BB1FFF78EFFF61B3D4473
:105BE000F0D1064802F0F4FA2046BDE8F0816FF0EB
:105BF0008B04F6E76FF01504F6E700BF582100208C
:105C0000996700202DE9F8430E463046194617469D
:105C10001C4605F021FD88B346EA040515F003058E
:105C20002CD1BCB11748DFF860904FF0FF324FF035
:105C3000FF3302F001FB24F00304AC4206EB05083D
:105C40000BD1124AD2F80034DB07FBD500240D48F3
:105C500002F0BEFA2046BDE8F883FFF763FF50B9B3
:105C60007959404601F098FA99F800300BB1FFF7E6
:105C700043FF0435E1E76FF08B04E8E76FF01504AC
:105C8000E8E700BF582100209967002000E00140AC
:105C90002DE9F043476840F20636D0063B7C87B0DA
:105CA00002EA060654BFC2F3401C4FF0030C01F099
:105CB0001F05B6F5837F144645EA43158DF803C0EA
:105CC00044D00DD8062E16D005D8A6B1022E3FD04E
:105CD0006FF0150037E0B6F5807FF9D101260AE0B4
:105CE00040F20222964235D0B6F5407F34D0B6F568
:105CF000007FEDD10226220330D57A6801238B4044
:105D0000C2F80835B868A0BB05F01F036D092DD097
:105D1000012D77D13E4A02EB8302C4F30043D2F84F
:105D2000001783F00103C4F3404444EA430421F420
:105D3000E16144EA8C0421F0070144EA06230B43A5
:105D4000C2F80037002007B0BDE8F0830726D2E78D
:105D50000426D0E70526CEE70326CCE7630341BF40
:105D600001237A688B40C2F80C35CBE74FF0A04294
:105D7000D1E70DF10202294606F0F2F914F4403F92
:105D800080460CD1B868294606F01FFAB8F1000F1A
:105D9000D8D19DF80210B86801F0DEF8D2E74FF0D4
:105DA000000901ABCDE90199CDE90439CDF80C909A
:105DB000B86803AA294606F0A8F84845C2DB14F4DF
:105DC000003314D0C4F300449DF803308DF80E3036
:105DD00084F001048DF80C608DF80D40B8684B46D6
:105DE00003AA294606F044F90028CFDAAAE7CDE94C
:105DF00004330DF103030393B86803AA294606F0A0
:105E000084F8F1E703F5E07350F82330FFDE00BFBC
:105E100000030050420970B5034602D0012A17D092
:105E200070BD0D4E326951680029F9D003F01F038F
:105E300001250C689D400029F2D08A682A4002D0D2
:105E40004B68304698472CB1236821461C46F2E740
:105E5000024EE7E72346F8E73CE2000020E20000BC
:105E600038B54568A86890B106F0A9F9014670B93F
:105E7000A86806F088F9044658B902460649A86899
:105E800006F06BF9224605210620FDF727F90020D0
:105E900038BD6FF00400FBE7155E0000F0B5446804
:105EA0001646A068227C01F01F0587B045EA42151E
:105EB00000286DD0B6F5001F04D1294606F0D8F9A8
:105EC000002056E06268607CC2F8240501AA002028
:105ED000B6F5800F0190506037D1B3F1007F14BF49
:105EE000052304238DF804300023CDE90423039314
:105EF000E36823FA01F111F001010DF103073AD132
:105F0000B6F1A07F37D105F01F036A0903F5E073EE
:105F100026D0012A3FD1214A52F82330DB072AD468
:105F2000A0683A46294606F01BF916301BD00297A6
:105F3000A06803AA294605F0E8FF002819DBA0683D
:105F40000122294606F043F9BAE7B3F1C06F05D044
:105F5000B3F1007F14BF01230223C3E70323C1E78A
:105F60004FF0A042D8E7A068394600F0FBFF0028B8
:105F7000DDDA07B0F0BDA0683A46294606F0F0F831
:105F80000028D5D19DF80310A06800F0E5FFCFE709
:105F90006FF08500EDE751F82330FFDE000300507D
:105FA000036803F01F025B09026004D0012B034861
:105FB00018BF002070474FF0A0407047000300500A
:105FC0002DE9F04F00EB8109554985B0154607468C
:105FD00040F2FF1AB94503D1002005B0BDE8F08FAB
:105FE0003B68C3F3C72818F00808C3F3C322C3F300
:105FF000080440F08F804B481B0E865C544508BF58
:106000004FF0FF34192B00F28880DFE803F00D1EFB
:106010002534282F3486868686373D868686868672
:1060200086868686407A7D80C5F80C45621C66D0DF
:1060300003A80394FFF7B4FF039A012303FA02F2C3
:10604000C0F808259B46584637E0C5F81445631C40
:1060500055D04FF0000BF6E7C5F80845E6E7C5F860
:1060600008454FF0000B601C1CD148E0C5F80C45FA
:106070004FF0010BF7E7C5F81045E8E7C5F808450C
:10608000002EE4D10626E2E7C5F80C45F8E7C5F88E
:1060900060457B88621C03F0010330D0002BC7D120
:1060A0004FF0010B03A80394FFF77AFF039A84468D
:1060B000012000FA02F2CCF80C253A68019202F4B1
:1060C000004CBCF1000F08BF804603A818BF4FF07A
:1060D000010B0394FFF764FF039C019A00EB84001B
:1060E000C2F34122D0F80047360246EA820646EA69
:1060F00008060C40264346EA4B06C0F80067043702
:1061000068E7C5F86445C4E7C5F86845C1E7C5F860
:106110006C45BEE76FF015005FE76FF085005CE748
:10612000F0F8FCFF9FEE0000014B01221A6070475F
:1061300000C000400C2903690BD15B6A064907487F
:106140004B4393FBF0F100FB1133116053600020CF
:1061500070476FF08500704790D0030040420F00F9
:10616000044B00690022C3F80021D3F8003102F08B
:106170002FB800BF00C000407FB50569AB6A63B3AC
:1061800021F040010C292BD105F110064FF0FF3210
:106190004FF0FF33304601F027FF134B0193A86AFD
:1061A0000323002469460394029304F0F7FB4FF0A5
:1061B000FF324FF0FF33284602F03EF8A86A04F0A1
:1061C00038FC0A4BD3F808256A6201225A6030462F
:1061D00001F07CFF204604B070BD6FF00A00FAE7C2
:1061E0006FF08500F7E700BF2961000000C00040A4
:1061F00010B504690020FFF7E5F9A0624FF0FF3207
:106200000021204606F059FD04F1100006F0C3FC01
:10621000002201210C20FCF761FF0C20FCF72EFF6F
:10622000024B0122C3F80423002010BD00C000402F
:10623000F7B52A2945680369144652D1AA7A1B8CFE
:1062400012F020016A7918BF1BB2002A49D0EA79FE
:106250002E7C042A09BF2A68EA899268128909B14A
:10626000013EF6B24FF47A7783FB0232A3FB07318B
:1062700007FB0212A8796946CDE90032FEF7BEFDA0
:10628000074658BB0198009BC6F12001B6F12002D9
:1062900000FA01F123FA06F343EA01035CBF40FA76
:1062A00002F213436E694FEAE37C184661467EB101
:1062B000A6FB0301AA690E4D002306FB0C11F9F79A
:1062C0001FFF0C4BC61845EB0102B34293410BD3A1
:1062D000084A0023F9F714FFC4E90002384603B066
:1062E000F0BD6FF08507F9E76FF02107F6E700BF13
:1062F00020A1070040420F00F7B50023456804695C
:1063000007460022684606F081FEDDE90023C4E965
:106310000623286806F0BDFB20B96FF01206304650
:1063200003B0F0BDE869002846D1284605F038FAE8
:1063300006460028F3D16B79002B65D02A7901231A
:10634000934063602B7C23746B7C637404F12003A3
:10635000A3600223E36095F8283083F00103A3745F
:106360007B68D86900282CD17C68E0690028D6D0E9
:1063700094F820303D690121994003691B68194256
:10638000836814BF1B69DB6898472149606A214A0A
:106390000C464FF400470021E0FB07410023204654
:1063A000F9F7FEFE02460B46684606F02FFEDDE9D1
:1063B0000023C5E90623B2E706F06BFB0028B4D141
:1063C000ABE793F820105B8CD0F810C0D0F808E051
:1063D000DCF80040DA0754BF43F4B01383F4D01361
:1063E000012523F480128D40DB074CBF2C43AC43C6
:1063F000CCF80040DEF8003098470028B4DA10F1FD
:10640000860FB1D006468AE76FF0850687E700BFA2
:106410003F420F0040420F002DE9F041044647681B
:106420000D4606F0C7FC88B14FF02008EFF3118647
:10643000314688F31288BFF36F8F606805F086FAE3
:1064400050BB86F31188BFF36F8FEFE71F4B1B78AC
:10645000002BE9D04FF020086426606805F076FA3A
:1064600070B9012005F0A2FB013EF6D100212120E8
:1064700006F06BFDF0E786F31188BFF36F8FF5E749
:10648000EFF31186314688F31288BFF36F8F60688F
:1064900005F05CFA0028EED0BB691D706368BA692C
:1064A0001B680020C3F844250122C3F84825C3F81F
:1064B0002001D3F82041C3F85801D3F858019A605D
:1064C00081F31188BFF36F8FBDE8F081BE670020B4
:1064D00070B5012383400F4ABFF35B8FDC4352E862
:1064E000001F01EA040542E80056002EF7D1BFF371
:1064F0005B8F4FF4803282400748C0F80823BFF317
:106500005F8FBFF36F8F03EA0100003818BF0120CF
:1065100070BD00BFB02100200010014070B41249CE
:10652000D1E90034D01AC31844F1000422F07F46A8
:10653000C1E90034A6F50013B3F5400F09D20B4BA7
:106540001B681A0A1B069C19094B42F10005C3E996
:106550000045EFF31181202383F31288BFF36F8F7F
:1065600070BC02F033BD00BF88050020B4210020BC
:106570009005002011B3BFF35B8F0123104A8340C5
:1065800052E800CF4CEA030C42E800C10029F7D1E1
:10659000BFF35B8F0B4A4FF480338340C2F8043360
:1065A000094BBFF35B8F1B68BFF35B8FC340DB07F7
:1065B00042BF064B4FF40032C3F80021704700BFC2
:1065C000B021002000100140AC21002000E100E0DB
:1065D0000D4B1868010A0006BFF35F8F0B4BD3F811
:1065E0000435181841F10001B3F5801F0AD2084B99
:1065F000D3E90023904271EB030303D210F18070C2
:1066000041F10001704700BFB4210020001001409B
:10661000900500202DE9F04F85B016461F469DF8E5
:1066200040A00446FFF754FF0190FFF7D1FFB042AE
:1066300071EB07035ED23E4B301A67EB01019842C3
:1066400071F1000109D36FF0150520460199FFF79C
:1066500091FF284605B0BDE8F08F364B03EB0413DD
:10666000D3E902239F4208BF964254D032494FF4E7
:10667000803804F1500508FA04F8AD00C1F84883E9
:106680002046ADB205F076FA26F07F4B05F1804545
:1066900004F5A87305F58835DC464FF0030902932D
:1066A000029A2CF07F4341F82230C1F84483D1F89C
:1066B0000435224A6FF00200C01A604420F07F4087
:1066C000904228D9286868B1D1F804350393A3EB28
:1066D0000B0020F07F40B0F5000F1CD9204605F0DC
:1066E00049FA039BBAF1000FADD109EB030C09F194
:1066F0000109D5E7BAF1000FA5D10123104ABFF374
:106700005B8FA34052E8000F184342E800010029C4
:10671000F8D1BFF35B8F07490E98230101EB0412F8
:10672000C8500F9B5360C2E9026700258DE700BF88
:10673000010080007805002000100140FDFF7F006F
:10674000AC2100207FB51C4C1C4BC4F80833C4F8A6
:1067500048331B4B00254FF0FF304FF0FF31C4F89A
:106760000855C3E902014FF48033C4F80433154BD4
:1067700002264FF400320121C4F804631120C3F84B
:1067800080212A46FCF7AAFC1120FCF777FC0E4A70
:106790000123A360236013600C4B0D4A0093CDE9E5
:1067A000015500232846FFF735FF3046FEF712FF5C
:1067B000284604B070BD00BF0010014003000F0068
:1067C0007805002000E100E0B02100201D650000F8
:1067D000FFFF7F002DE9F7432E4CD4F804339907CF
:1067E0000BD5D4F8043143B12B4A0023C4F804314B
:1067F000D4F80431136801331360D4F80433DA0396
:1068000043D5BFF35B8F254B53E8002F22F00101E6
:1068100043E800100028F7D1BFF35B8FD30702D401
:10682000D4F840318BB30025C4F84051D4F840313E
:10683000FFF7CEFEEFF31182202383F31288BFF31C
:106840006F8F174BD3E90267B042B94120D34FF0A5
:10685000FF304FF0FF31C3E90201D3E900981D601A
:106860004FF48033C4F84833C4F84051D4F8403171
:1068700082F31188BFF36F8FB9F1000F05D0CDF807
:10688000008032463B460020C84703B0BDE8F08395
:10689000A946EDE700100140B4210020AC21002002
:1068A0007805002030B5431C124C85B005D08442D9
:1068B000A8BF0446012CB8BF0124FFF789FE0E4B88
:1068C0000C4DD3E90013401AB0F5000F10D2221876
:1068D000AA4228BF2A4652184FF0000007490091EB
:1068E000CDE9010043F10003FFF794FE05B030BD90
:1068F0002A46F0E7FFFF7F00880500201D650000A5
:1069000008B5FFF765FE024B1B68C01A08BD00BF43
:106910008805002010B5084C012363601120FCF7A6
:10692000BBFB064BC4F80833C4F84833044B4FF4A0
:106930000032C3F8802110BD0010014003000F0099
:1069400000E100E0BFF34F8F0549064BCA6802F42F
:10695000E0621343CB60BFF34F8F00BFFDE700BF82
:1069600000ED00E00400FA05024AD2F80034002BE2
:10697000FBD0704700E0014010B54FF08053D3F8D2
:106980003021082A4ED14FF080420021C2F80C116C
:10699000C2F81011C2F8381502F54042D3F80414B9
:1069A000C2F82015D3F80814C2F82415D3F80C1433
:1069B000C2F82815D3F81014C2F82C15D3F8141403
:1069C000C2F83015D3F81814C2F83415D3F81C14D3
:1069D000C2F84015D3F82014C2F84415D3F8241493
:1069E000C2F84815D3F82814C2F84C15D3F82C1463
:1069F000C2F85015D3F83014C2F85415D3F8341433
:106A0000C2F86015D3F83814C2F86415D3F83C14F2
:106A1000C2F86815D3F84014C2F86C15D3F84434A2
:106A2000C2F8703505F0B2F818B13C4B3C4AC3F8D7
:106A30008C2605F0ABF818B13A4BFB22C3F81825A9
:106A400005F0A4F858B14FF080424FF08051D2F8D1
:106A5000E43ED1F8581261F30303C2F8E43E05F0B6
:106A600095F820B1304B4FF40072C3F840264FF038
:106A70008053D3F83031082B17D14FF08043D3F82F
:106A80000024D20744BF6FF00102C3F800244FF086
:106A90008053D3F83431042B81BF4FF01023D3F847
:106AA00008224FF08043C3F858254FF01021D1F849
:106AB0000C32DB0714D51D480123C0F80435FFF75D
:106AC00053FFD1F80C3223F00103C1F80C32FFF769
:106AD0004BFF0023C0F80435FFF746FFFFF732FFF6
:106AE000D1F80032002B03DBD1F80432002B14DA8A
:106AF0000E4901234FF01020C1F804351224FFF78E
:106B000033FFC0F80042FFF72FFFC0F80442FFF741
:106B10002BFF0023C1F80435DEE710BD0050004014
:106B20004881030000F000400090024000E0014076
:106B3000014B1860704700BFB821002010B5054B0D
:106B40001868144605F034F80028A4BF207000200F
:106B500010BD00BFB8210020024A01238340C2F8C3
:106B60000435704700F00140014B00201B681847B6
:106B7000BC210020014B1B68184700BFBC2100202E
:106B800010B50C4C237993B9012323710A4B206073
:106B9000002818BF184600F04BF850B92368074882
:106BA000002BBDE8104008BF184600F091B86FF008
:106BB000770010BDBC210020696B0000756B0000E0
:106BC00008B5064B1B682BB10020FCF779FA08B911
:106BD000FCF754FA024B01221A7008BDBC210020B8
:106BE000BC67002038B54FF080440123C4F8083357
:106BF00063600023C4F80031D4F8003142F210750C
:106C0000D4F80C24D4F80C34D20307D5DB0705D50F
:106C1000012004F0CBFF013DF2D138BD05F030F882
:106C20000028FAD0014B00225A71F6E7C421002057
:106C300010B508490C794CB9012308600B7105F0B7
:106C40001FF808B9002010BD4C71FBE76FF077000A
:106C5000F9E700BFC42100204FF080430022C3F8B1
:106C60000021D3F80021094901221A60096811B1F5
:106C7000C3F804237047D3F80021002AFBD0002278
:106C8000C3F80021D3F80031704700BFC4210020B1
:106C900010B54FF08043D3F80423D20715D5D3F8AD
:106CA000002192B10022C3F800210121D3F8002174
:106CB000C3F8081304F0E4FF044B10B15A7922B969
:106CC0005971BDE810401B68184710BDC421002051
:106CD000074A13794BB901215371106011714FF0BC
:106CE00080421846C2F8183570476FF07700704739
:106CF000CC21002010B54FF080431B4CD3F8181462
:106D0000D3F8182411F4803F15D0900701D004F077
:106D1000D7FF4FF080430022C3F81825C3F80421A1
:106D2000D3F8042101229A60226872B9D3F80421B1
:106D3000002AFBD011E0D3F81424D107E9D5D3F809
:106D40001C249207E3D122681AB10222C3F804235B
:106D500010BDD3F80421002AFBD00022C3F804217F
:106D6000D3F80431F4E700BFCC21002038B54FF050
:106D70008041D1F80C24D1F80C34D0032AD5DA079D
:106D800028D5D1F81834DB0324D5154C637903F0EA
:106D9000FF0213BBC1F80C210125D1F80C3165713C
:106DA00004F07FFF10B10223C1F8343C4FF0804360
:106DB0001D61226822B10822C3F80423002038BDD7
:106DC000D3F80C21002AFBD00022C3F80C21D3F801
:106DD0000C31F3E76FF07600F1E76FF00F00EEE7AC
:106DE000CC2100202DE9F0414FF08043164FD3F81D
:106DF0000443012504F01A0400260CB9BDE8F08113
:106E0000B4FA84F1C1F11F018B0003F580739BB2CA
:106E100003F1804305FA01F2186892B224EA0204F1
:106E20000028EAD04FF080481E60082A1B68C8F886
:106E3000082305D104F035FF08B1C8F8346C7E7121
:106E40003B68C8B29847D8E7CC210020036803F01C
:106E50001F025B09026004D0012B034818BF002009
:106E600070474FF0A040704700030050034A4309A9
:106E700000F01F00D35C1844C0B27047A7EE0000BA
:106E8000024611F0010030B515D18B07C1F3400067
:106E900022D51249D1F8200550604FF08052C1F838
:106EA0002005D2F83021082A08BFD1F82025003863
:106EB00018BF012010E04FF0A0444FF08055D4F8E7
:106EC00020351360C4F82035D5F83051082D08BF9F
:106ED000D4F82045002BD8D030BD00BF00030050AF
:106EE000F7B504460846FFF7C1FF04EB40060D4620
:106EF000B38ADB072AD5204604F0E5FF2946204661
:106F000004F051FF50B1204604F063FF276807EBFF
:106F100080000023C0F81035C0F8103529462046FF
:106F200004F080FF0021B18201A80195FFF78EFFD8
:106F3000019B00EB8300074BD0F80027134043F080
:106F40000203C0F80037084603B0F0BD6FF015002B
:106F5000FAE700BFF0F8FCFF014804F047BE00BFAD
:106F60007402002010B504480C4604F021FE0028ED
:106F7000A4BF2070002010BD740200202DE9F04F46
:106F8000074689B057F8049BD9F80413C9B2834661
:106F9000082241F00041484604F06DFF051E2FDA3B
:106FA0000023032106A8CDE90633FFF769FF634BF1
:106FB00001930DF118084FF0000A019A604912F888
:106FC000013B0192DA0803F007038A5C22FA03F31B
:106FD000DB071CD40AF10103022B08F104084FF06F
:106FE000010AEAD14FF000410022484604F043FF75
:106FF000032106A8FFF744FF0028D8D125F000455B
:107000000124002D40F0848009B0BDE8F08F4D4B85
:1070100053440293D8F80060002EDBD0029B96FA0E
:10702000A6F61C78B6FA86F646EA44142046FFF720
:107030001DFF0BEB4000F208818A18F8020005944E
:10704000C1F382030393009306F00706012303FABA
:1070500006F620EA060008F8020005A8FFF7F6FE8B
:10706000059A039B02F5E07211F0100F50F82260B0
:10707000C6F3014633D0009A3846214604F0B3FEE9
:1070800005A80594FFF7E2FE059B03F5E073F6B251
:1070900050F82330C3F301439E4207D1002120461C
:1070A00004F072FE3146204604F06EFE05A80594F9
:1070B000FFF7CCFE059B012202FA03F3C0F820354E
:1070C0004FF08053D3F83031082B01BFD0F8203572
:1070D000D0F82035D0F82035D0F820359AE7022EA8
:1070E00014BF022103212046039304F04DFE039BAD
:1070F000032B03D0022E07D1012BD7D1009A2146B2
:10710000384604F070FED1E7032ECFD1022BF4E70E
:1071100095FAA5F3B3FA83F304FA03F225EA02051C
:1071200003F5A2720BEB430359F82220B3F87C104D
:10713000C2F30142384604F056FE62E7B7EE0000A3
:1071400048E70000B7EE0000044AD2F80034DB073D
:10715000FBD50160BFF35F8F704700BF00E00140C7
:107160004FF080531A69B0FBF2F302FB13036BB9C3
:10717000084B0222C3F80425C3F80805D3F80024FD
:10718000D207FBD50020C3F8040570476FF00C0050
:10719000704700BF00E0014010B5054C0123C4F862
:1071A0000435FFF7D1FF0023C4F8043510BD00BF3C
:1071B00000E0014010B5174C23783BBB0278C2F3C6
:1071C000400392070FD54FF08053D3F83021082A9F
:1071D00008D1D3F83431022B02BF4FF08043012293
:1071E000C3F8382601234FF08042C2F88035037877
:1071F00003F00103C2F878350020FBF761FF08B9FE
:10720000FBF73CFF01232370002010BD6FF07700D7
:10721000FBE700BFBD6700204FF080434FF4607272
:10722000C3F80823014B00221A607047D4210020C4
:1072300008B5FFF7F1FF03680BB1014A136008BD01
:10724000D421002010B54FF08043D3F804436207E7
:1072500007D54FF4847005F01BF810B11E4B1B6866
:107260009847A30608D54FF48A7005F011F818B1B5
:107270001A4B00201B689847600608D54FF48C70A5
:1072800005F006F818B1154B01201B689847210638
:1072900008D54FF48E7004F0FBFF18B1104B00209E
:1072A0001B689847E20508D54FF4907004F0F0FF92
:1072B00018B10B4B01201B689847A3050AD54FF462
:1072C000927004F0E5FF28B1054BBDE810401B6843
:1072D0000220184710BD00BFDC210020D82100206B
:1072E000D421002080F08003042B04D8054B0344F4
:1072F00013F8800C704707289ABF034B185C0020D6
:10730000704700BFB9EE0000BEEE0000064B93F8D8
:107310002E00012806D0022818BF042814BF01201F
:107320000020704700207047E021002010B5164B68
:10733000164A0020C3F8000592F82F40D3F8041332
:1073400082F82E40146821F033010CB141F0230182
:10735000C3F81C01D3F81C41C3F81801D3F8184135
:10736000C3F80801D3F8080192F8340092F83320EA
:1073700002F0010200F00100D20142EA80120A4349
:10738000C3F8002310BD00BF00700040E0210020C2
:1073900070B50D4A002392F8301001251E4618B929
:1073A0000BB182F8301070BD90FAA0F3B3FA83F3FA
:1073B00005FA03F40C3302EB430320EA0400DE80F9
:1073C00021EA04010123EAE7E021002073B500234C
:1073D000044601AA0E464FF48071019304F079FF30
:1073E0004FF48A71204604F074FF4FF48271054611
:1073F000204604F06EFF20B11EB115B1144BD3F836
:10740000343601AA4FF48471204604F062FF4FF431
:107410008671204604F05DFF4FF48871204604F029
:1074200058FF0C4B234083B14FF48E75294601AAB7
:10743000204604F04EFF291F083589B22046ADB220
:1074400004F047FFB5F5AE7FF0D1019802B070BDF2
:1074500000700040C0FF3F002DE9F04F9A464FF00A
:10746000805393B0D3F830411C9D082C3FD1D3F802
:107470003431012B3BD00DF1080C0AAF3E4C3E4697
:10748000E046002304EB031E0133DEF8189548F8AC
:10749000049B082BDEF81CE546F804EBF2D1D4F887
:1074A000F065D4F8403601934FF0010E0023D4F874
:1074B0004496D4F84886C4F8FC3FC4F8FCEF2E4C40
:1074C0005CF804BB04EB031E0133CEF818B557F883
:1074D00004BBCEF81CB5082BF2D1019BC4F8403692
:1074E000F6B2C4F84496C4F84886C4F8F065234B55
:1074F000002483F8334083F834409C601C611D6095
:1075000083F831009C831C4BC3F8F015C3F8F425B5
:107510007DB32322C3F80023184D174C0022012706
:10752000110107FA02F301F18046034006F5E04637
:1075300019BF95F81EE095F81FC09C469E46002B8B
:1075400004EB0103C6F810E5C6F814C5D3F8181506
:1075500014BF5646002621F08071013241EA0661CF
:10756000082AC3F8181505F10205D9D113B0BDE8F2
:10757000F08FC3F80053CFE700700040E0210020F7
:10758000F8B50446067A4779417AC079FFF7AAFE32
:1075900010B96FF01500F8BD214A01F10C0502EB9E
:1075A0004503012F987139D13046FFF79BFE002823
:1075B000EFD002EB4505E871E378A0781B030002E9
:1075C00000F4E06003F480530343207800F00300EC
:1075D00003432079000400F4E020034360780001B5
:1075E00000F030000343A079000600F080700343F0
:1075F0006079000500F480100343080100F1804029
:1076000000F5E040C0F81835012303FA01F192F8C3
:1076100030300B4382F830300020BCE70020C8E750
:10762000E0210020084B01229A600022C3F81421B7
:10763000D3F8141105498020C1F88001C3F8002552
:10764000C3F80025704700BF0070004000E100E073
:1076500070B5204D95F82E40002C38D1FF20012622
:1076600085F82E60FFF794FE1B4B1C48C3F80041C1
:10767000D3F80021C3F80441D3F80421C3F8104122
:10768000D3F81021C3F81441D3F814311C239A08FD
:1076900006FA02F111F0330F1CBF03F1804101F52E
:1076A000E24102F1FF3218BF0C6006FA02F218BF85
:1076B000096812F0330F1CBF1C501A5808335C2B9A
:1076C000E5D10720FBF7DAFC0020286070BD6FF0E1
:1076D0007700FBE7E021002000700040FC700040D4
:1076E000014B93F830007047E02100202DE9F7436B
:1076F00007469946FFF70AFE044608BBDFF85080AC
:1077000098F83030082601252F4203D02B421CD098
:107710000134E4B2013E4FEA4505F5D10D4BC3F803
:10772000F865131E18BF01233846CDF80090FFF707
:1077300093FE022388F8324088F82E30304601E06C
:107740006FF00F0003B0BDE8F0836FF01500F9E7AC
:10775000E0210020007000402DE9F34180461546ED
:107760001A46FFF7D3FD0646002837D1204F97F879
:1077700030C008203446012318EA030F04D013EA6E
:107780000C0F2ED00134E4B201384FEA4303F3D199
:107790006B8813B1012C27D832B328786B7818B1D5
:1077A00013B9012C20D80126009202464046FFF76B
:1077B00053FE6B880F4A0BB143F48053C2F8F8357F
:1077C00087F832402B7987F83530042387F8366004
:1077D00087F82E30002002B0BDE8F0816FF00F0076
:1077E000F9E76FF01500F6E76FF08500F3E700BFEB
:1077F000E02100200070004030B51D4A13690446A6
:107800006BBB00F06043B3F1005F2BD192F83250B4
:10781000B1FBF5F305FB131038BB0BB2002B24DDD5
:1078200092F82E30052B06D8032B0BD8022B0ED046
:107830006FF0760030BD062BFAD10E4BC3F82C4604
:10784000C3F8301693683BB1C2E90441F2E78D42B8
:107850000BD1C2E90245EDE7C2E90241EAE76FF068
:107860007700E7E76FF00C00E4E76FF00600E1E770
:10787000E0210020007000402DE9FF41524CA36838
:10788000002B00F09D8094F82E20022A06D0042AB6
:1078900033D06FF0760004B0BDE8F0814B4D012687
:1078A000C5F800652168E26849B1032184F82E100B
:1078B000C5F82C36C5F830262E600020EBE7C5F859
:1078C0002C36C5F830262E6004F01BFD04F10803A9
:1078D0006E60019301990220FFF778FD0028F9D02E
:1078E0003A4B0022C3F80821D3F80811C3F80C2141
:1078F000D3F80C11C3F80025DFE7344D4FF0010831
:10790000C5F80085276857B1052284F82E20E26863
:10791000C5F82C36C5F83026C5F80080CDE7A18B18
:1079200094F83220039203EB41030293C5F82C36FE
:10793000C5F83026C5F8008004F0E3FC94F8363032
:1079400063BB224D01236B6002A90220FFF73EFDBD
:107950000028F9D00023C5F80831D5F80821C5F86A
:107960000C31D5F80C21A18B94F832200A44E1683F
:1079700092B28A42A28321BF154AA383D2E90201AF
:10798000236124BFC2E900011846104B4FF00002EA
:1079900038BF6FF00F00C3F800257CE7D5F8F46519
:1079A000F6B208FA06F6013EBE42CAD9C5F804800E
:1079B00000210420FFF70AFD0028F9D00137F3E782
:1079C0006FF00B0067E700BFE0210020007000406F
:1079D000E8210020F8B50246FFF798FC002851D1B5
:1079E0002A4E2B4C96F82E3086F82F30072386F837
:1079F0002E3001237260C4F80035D4F80453C4F863
:107A00000003E3603AB125F0C00545F03305C4F842
:107A100000530020F8BD00211020FFF7D7FC0028FC
:107A2000F9D00023C4F80431D4F80431194BC4F858
:107A30002C3601270223C4F83036276004F061FC9D
:107A4000A76000212020FFF7C1FC0028F9D0104BCF
:107A50000022C3F80421D3F80411C3F80821D3F895
:107A60000811C3F8002596F82F1086F82E10C3F8D9
:107A70001C21D3F81C11C3F81821D3F81821C3F81E
:107A80000053C6E76FF00F00C4E700BFE0210020FD
:107A900000700040F82100207FB56249614E33201C
:107AA000FFF794FC10F0100F05460BD05E4B102230
:107AB000C3F80823B218C3F82C260222C3F83026D4
:107AC00001221A6015F0200F584C10D094F82E3077
:107AD000554A072B05D0D2F834369BB2E360002319
:107AE0002361D2F80433DB0601D5FFF71FFCA8079A
:107AF00017D5002294F82E308DF80420A268029247
:107B0000062BE268ADF80C2017D0072B33D0032BDF
:107B100007D1FFF787FD022384F82E30236801A8E0
:107B20009847E9074ED594F82E30033B042B49D8EB
:107B3000DFE803F0594828405D0094F8353023B160
:107B4000236913B1384B01221A60236801A89847B2
:107B5000374B93E8030086E8030000232361A36802
:107B6000002BDED1FFF75EFD042384F82E300523C1
:107B70008DF80430D2E7FFF7D9FB02238DF80430EB
:107B80006368CCE704238DF8043001A82368984784
:107B9000254BD3F8F825D20444BF01225A6022694C
:107BA000062384F82E302AB11F4B6169C3F82C26B6
:107BB000C3F8301623692BB903238DF8043001A8CC
:107BC0002368984794F82E30072B0AD0164B194893
:107BD000D3F8043300211840FFF7F8FB012685098C
:107BE0004DB904B070BD104B01225A60EAE70E4B4C
:107BF00001229A60E6E795FAA5F3B3FA83F306FA51
:107C000003F225EA02055A08DB4303F001038DF86D
:107C100009308DF8046023688DF8082001A8984782
:107C2000DEE700BFE821002000700040E0210020D6
:107C3000F0210020C0FF3F0070B50A460C4620230B
:107C40000021054602F0FEFF28B11548452102F04B
:107C5000DFFF012070BD2268124B9A4205D0124806
:107C6000452102F0D5FF0320F4E7236913F0100249
:107C700004D00E48452102F0CBFFF4E7E6682189E5
:107C8000AB68891906D20A466189891802D29942DD
:107C90000A46DFD30648452102F0BAFFE3E700BFFA
:107CA000FBEB00003DB8F3961CEC000037EC000045
:107CB0004FEC000070B516461D465A1C036813446D
:107CC000C2689A42044605D2006A082104F0FAFD0F
:107CD000002070BD65B93278204604F0F6FD00281A
:107CE000F6D03544B5420CD1A3680133A360F0E768
:107CF000AB1E062B9ABF064AD35C00231833DAB2B8
:107D0000EAE723685A1C226015F8012D1A70E9E78A
:107D1000C6EE000038B5EFF31185202383F31288F7
:107D2000BFF36F8F064B9C6804F0C6FE85F3118885
:107D3000BFF36F8F2046BDE83840FBF75FBA00BF46
:107D40001822002038B50A4B53F82040013053F870
:107D50002050A54200D838BD606830B1037EDB07F3
:107D600001D404F07EFE0834F3E723689847FAE76D
:107D70004CE7000070B5294B294C2A4D86B00122F2
:107D800003201A70FFF7DEFF0420FFF7DBFF264613
:107D9000AE4204F130040FD300F066FF204CAC4239
:107DA00026D300F075FFF8F77BFB1F4A938923F079
:107DB0000103938106B070BD54F80C3C059354F850
:107DC000103C049354F8143C039354F8183C029369
:107DD00054F81C3C019354F8203C009354E90A23C6
:107DE00054E90C0100F0C0FB54F8303C5E65CEE76E
:107DF000D4E90A23B3F1FF3F08BFB2F1FF3F05D03A
:107E000052EA0301206803D100F0FEFB3034C6E7DC
:107E10000649183000F0FAFFF8E700BFBE670020FF
:107E20009CE400009CE4000018060020E9CE00005D
:107E300070B5002386B00122CDE90423114E124D06
:107E400001930F22CDE902321049142303FB0055A0
:107E500006EBC0164FF4A072044602FB00110C4B57
:107E60000095304600F080FB337C2C7423F0040333
:107E70003374084BEE60013403EBC4236B6006B02F
:107E800070BD00BF9805002018220020C077002098
:107E900071CB0000C06F00207FB50020FFF752FFBC
:107EA000284B83F30888284C636943F400736361AB
:107EB0000025E02384F82230E57725766576A576DF
:107EC00084F82050636A43F4E023636284F823500B
:107ED000FBF77EF8FBF77CF94FF0FF33A362E36218
:107EE000FBF766FAFBF7EEF91848194C00F080FB37
:107EF0000120FFF727FF0220FFF724FF00F0ACFE70
:107F0000144B15495C61154B059301234FF4205226
:107F1000CDE90353CDE90155114B0095204600F002
:107F200023FB237C064623F004032046237404F03D
:107F3000A3FF2846FFF77CFF094A31462046FBF79E
:107F40002BF900BFC077002000ED00E0980600206C
:107F500018060020182200200079002086EC00007E
:107F6000757D000038B5074C074DAC4201D30020A9
:107F700038BD204604F0A3FD08B91C34F5E76FF0C6
:107F80001500F5E7E0020020FC02002073B50C4666
:107F9000EFF31181202585F31288BFF36F8FC56839
:107FA0005DB125602B68C360836901338361002064
:107FB00081F31188BFF36F8F11E052EA030603D1FA
:107FC00025606FF00B00F3E7CDE90023024608308F
:107FD00000F030FD18B9034B9B685B69236002B069
:107FE00070BD00BF182200202DE9F341044617465A
:107FF0001E46EFF31188202383F31288BFF36F8F9F
:10800000304BC2689B6872B18068984217D057EABB
:10801000060216D188F31188BFF36F8F6FF00F003F
:1080200002B0BDE8F08193F90E1021610132C4E97C
:10803000023288F31188BFF36F8F0020F0E72169C7
:10804000F3E793F90E1090F90E30994230DA994225
:10805000A8BF194604F097FD0546CDE900761A48F9
:108060002246414600F0E6FC0028E6D0EFF31186F8
:10807000202383F31288BFF36F8FA068D0B12368E9
:1080800021699C420AD04BB193F90E309942A8BFA6
:1080900019466FF07F039942B8BF194604F073FD8B
:1080A00040B10948314604F04DFF6FF00A00B7E7D0
:1080B0000025D2E7002DF4D186F31188BFF36F8F2E
:1080C000F3E700BF18220020BF670020F8B58368DF
:1080D0000546002B3FD0234A926893423ED1C368A5
:1080E000012B03D9013BC3600020F8BDEFF31187DA
:1080F000202383F31288BFF36F8F0169806804F037
:1081000042FD2C68A54207D10023C5E9023387F35D
:108110001188BFF36F8FE7E7002CF5D0D4E9003268
:1081200013605A60237C002623F002032374C4E901
:108130000066A66004F1180000F000FFAC6094F93E
:108140000E302B612046A66704F096FE064839469D
:1081500004F0F8FEC8E76FF01500C6E74FF0FF30F7
:10816000C3E700BF18220020BF67002037B51146C3
:10817000EFF31185202282F31288BFF36F8F04681A
:108180009CB12368426823F003039442036008BF54
:1081900043600121204604F079FD044685F31188EF
:1081A000BFF36F8F204603B030BD51EA0302F5D014
:1081B00000F10802CDE900131046294600F03AFC10
:1081C0000028EFD1014B9B685C69EBE71822002087
:1081D00070B5EFF31186202383F31288BFF36F8FFE
:1081E0000468A0421AD0CCB1D4E9003213605A60BE
:1081F000237C002523F002032374C4E90055A56005
:1082000004F1180000F09AFE2046A56704F034FE41
:1082100031460848BDE8704004F094BED0E902320F
:108220009A4218BF0133836086F31188BFF36F8FC2
:1082300070BD00BFBF67002013B5EFF3118120248C
:1082400084F31288BFF36F8F846844B1013C84606B
:1082500081F31188BFF36F8F002002B010BD52EA86
:10826000030406D181F31188BFF36F8F6FF00F0005
:10827000F3E7CDE900230246014800F0DBFBECE721
:10828000BF6700202DE9FF41544E04462027EFF33D
:10829000118887F31288BFF36F8FD4F88450F5B933
:1082A000022104F19C0004F014FD002870D004F1B8
:1082B000940500220121284604F060FE0028F8D130
:1082C000002302934FF0FF324FF0FF33CDE900233C
:1082D000414604F18C02424800F0F0FCD7E7D4F8A4
:1082E00088202B68C4F88430954208BFC4F88830D1
:1082F000D4F89C3043F00203C4F89C30EB6823F0C0
:10830000040343F00103EB606B6888F31188BFF34B
:108310006F8F28469847EFF3118887F31288BFF3D1
:108320006F8FEB68D80623F001023ED4EA60EB6859
:108330009A0717D5306823F00203EB6090B1036809
:10834000002178B1426895423DD10368002934D1BB
:1083500072683360904200D17360002340F8083B9C
:10836000FFF736FFD4F89C3023F00203C4F89C30AA
:10837000DB0530D4D4F88430003B18BF012388F3E8
:108380001188BFF36F8F002B81D004F03BFD7EE797
:10839000D4F89C30D90693D5C4F89C0088F3118892
:1083A000BFF36F8F04B0BDE8F08123F01103EB60E1
:1083B00005F11000FFF70CFFB9E70B6073689842F6
:1083C00008BF7160C9E701461BB11A681846134619
:1083D000B7E71A46FAE70023D1E700BF38220020AA
:1083E000BF670020F8B5C3689A0704460E46C3F37A
:1083F000400542D45F0742D40B680BB983680B6019
:10840000E368D80744BFA368336037684CBF0225D0
:10841000012557B31B4B9A68D7F880309A421ED17A
:1084200004F0C8FC80F00100C0B2D7F89C30D90736
:10843000C3F380021CD5F2B1F8B100232360D7F852
:10844000883073B9C7E92144384604F04DFCE3682D
:1084500043F00403E3603368A3602846F8BD0020BE
:10846000E3E71C60C7F88840EEE76FF0150506E00B
:108470006FF0120503E01B07DFD56FF00F05002337
:108480003360EAE7182200200146014804F076BC78
:1084900038070020F0B589B004460020C4E9210067
:1084A0000E9D04F18C00C4E9230004F19400C4E99A
:1084B000250055B32879002840F2011008BF01209B
:1084C000C4F89C0000204FF0FF364FF0FF37CDE995
:1084D0000330CDE90100CDE906670D4B009420463D
:1084E00000F0B6F855B1296811B1204604F068FCD7
:1084F0006B791BB1A38943F00103A381204600F0EF
:1085000083F8C4F8804009B0F0BD0120D8E700BF6F
:108510008582000037B501900846EFF311842021D1
:1085200081F31288BFF36F8FC16811F01E0F16D14F
:1085300053EA020508D101A9FFF754FF84F311881B
:10854000BFF36F8F03B030BD41F00801C1600199E6
:1085500081620449103000F059FC0120EEE7002050
:10856000ECE700BFF7CC00002DE9F04F85B098464E
:1085700000F158030732C0E91633129B838122F0C1
:10858000070504230026037401EB0509119B83737F
:108590004FF0000A4FF0000B0F46C0E9066649464F
:1085A000C0E90AAB8660C6730446FAF7BFFB073022
:1085B000109B20F00700A066C4E9187502930F9B7A
:1085C0000193A9EB00090E9B00934A4643463946A6
:1085D0002046FAF7C5FD054B66659B6803B1DB6E67
:1085E000E366484605B0BDE8F08F00BF18220020C2
:1085F0000123037483810023C0E91833C366014B50
:10860000986070471822002038B50446EFF31185B2
:10861000202383F31288BFF36F8F037C5B070FD592
:10862000183000F08BFC237C23F0040320462374D5
:1086300004F031FC29460548BDE8384004F082BC0E
:1086400085F31188BFF36F8F38BD00BFBF6700206F
:10865000F0B587B000250595109D04950F9D0395F5
:108660000E9D0295DDE912760D9D01950C9D0095FC
:108670000446FFF779FFB6F1FF3F08BFB7F1FF3FB0
:1086800005D056EA070305D12046FFF7BDFF204677
:1086900007B0F0BD3A46334604F11800014900F036
:1086A000B5FBF4E7E9CE0000094A93686FF00A01D0
:1086B0009967084958674B6843F080534B60002323
:1086C00083F31188BFF36F8F9368986F704700BF73
:1086D0001822002000ED00E038B590F91020037C4E
:1086E000002A014604DA03F07F03037404F08CFBD4
:1086F0000D4D2A46AB6852F8184F944200D004B989
:10870000EC688B4207D01A7CD20604D1DA897F2A22
:1087100001D9A2692AB1A34202D0204600F010FB81
:1087200023466B6138BD00BF1822002070B590F958
:108730001020037C002A2FDBD9062DD11A4C63F0C0
:108740007F032246037452F8183FE169934207D130
:10875000C0E900210860E0610FE09942F8D01B6891
:10876000002BF5D093F90E6090F90E50AE42F4DD77
:108770005968C0E9003108605860A569954200D089
:1087800005B9E568A3681A7CD20606D1DA897F2A82
:1087900003D9AA690AB9636170BDAB4202D0284609
:1087A00000F0CEFA6561F7E718220020034648B9C9
:1087B000EFF3058232B9064A51699268914201D0BD
:1087C000FFF772BF83F31188BFF36F8F704700BF4D
:1087D0001822002038B5184CA168E0690B68814266
:1087E00014BF1A46002249680B605960A368E1690A
:1087F0002AB9124AC3E900210B60E3610AE092F949
:108800000E5093F90E00854212DD5168C3E9002134
:108810000B605360A569094B9D4200D005B9E5681E
:10882000A3689D4202D0284600F08AFA656138BDEF
:108830008A42DED01268DBE71822002030220020B6
:108840002DE9F047002A027C0CBF4FF010094FF0D1
:10885000080919EA020F04460E460F4628D149EAD4
:108860000203D20946D10374B9F1080F48D04FF082
:108870000008DFF8F0A0534653F8185F9D4200D07F
:108880000DB9DAF80C50DAF80830AB4202D02846BD
:1088900000F056FAB9F1100FCAF8145008D020466B
:1088A00002F015FDB8F1000F02D02F48FFF7A0FE2F
:1088B0002C4B9B68A3424FD1EFF30583002B4BD188
:1088C000A289D20711D586F31188BFF36F8F83F386
:1088D0001188BFF36F8F0423184602DFEFF311876F
:1088E000202383F31288BFF36F8F3846BDE8F0472B
:1088F000FFF7DABE03F07F03037404F085FAB3E7F1
:10890000A36813B1204604F087FA04F1180000F0C0
:1089100015FBA56D04F15808A84511D04FF0000AC9
:1089200075B1284604F078FA05F1180000F006FB4E
:10893000C5F878A02846FFF7F9FEA56DA845EFD148
:10894000084B9B689C4292D1EFF30588B8F1000870
:1089500018BF4FF001088CE786F31188BFF36F8FC3
:10896000BDE8F087182200209806002070B50F4D52
:108970002B46064653F8184F9C4200D004B9EC68C9
:10898000AB681A7CD20604D1DA897F2A01D9A269A0
:108990002AB1A34202D0204600F0D2F923466B61EF
:1089A0003046BDE87040FFF701BF00BF182200202D
:1089B00070B5EFF31186202383F31288BFF36F8F16
:1089C0001A4CA168E0690B68814214BF1A46002264
:1089D00049680B605960A368E1692AB9144AC3E980
:1089E00000210B60E3610AE092F90E5093F90E004A
:1089F000854216DD5168C3E900210B605360A5690B
:108A00000B4B9D4200D005B9E568A3689D4202D09A
:108A1000284600F095F965613046BDE87040FFF7E3
:108A200043BE8A42DAD01268D7E700BF182200207E
:108A300030220020F8B5124B0C461146114A9868B6
:108A40001060DDE90676EFF31182202282F31288AE
:108A5000BFF36F8F9D68284604F0E8F9B6F1FF3F39
:108A600008BFB7F1FF3F06D007493A46334605F144
:108A7000180000F0CBF92046BDE8F840FFF714BE1F
:108A80001822002040220020E9CE0000F8B504465C
:108A9000EFF31187202383F31288BFF36F8F037CDA
:108AA00003F01F02002A0CBF0126002649B235D16F
:108AB00003F07F03037404F0A7F9294D037C81734D
:108AC00063F07F032A46037452F8183FE869934223
:108AD00007D1C4E900200460EC610DE09842F8D0B1
:108AE0001B68002BF5D093F90EC08C45F6DD596854
:108AF000C4E900310C605C60AC69944200D004B9F8
:108B0000EC68AB689C4202D0204600F019F96C6119
:108B100087F31188BFF36F8F3046F8BD9B071CD5D4
:108B2000856804F071F981732B689D4209D16B68E7
:108B3000C4E900531C606C60EAE76A689A42F6D0A8
:108B40001B68002BF3D093F90E208A42F5DD5A689A
:108B5000C4E9003214605C60DAE78173D8E700BFD3
:108B600018220020034648B9EFF3058232B9064ABD
:108B700051699268914201D0FFF796BD83F3118845
:108B8000BFF36F8F704700BF18220020F8B550EA7E
:108B9000010306460C4603D104F034F90020F8BD69
:108BA000EFF31187202383F31288BFF36F8F174DE4
:108BB000174BA868186004F070F9A8681549324688
:108BC0002346183000F022F9AB681A7C5F6742F048
:108BD00004021A746FF00A029A670F4A536843F04E
:108BE000805353600446002383F31188BFF36F8FD3
:108BF000AA68D2E90A12B2F1004F08BF9942CDD15A
:108C000004F0FEF9201A20EAE070C8E718220020DC
:108C100040220020E9CE000000ED00E00C490D4AA2
:108C200008B58C464FF4004E0021C0FB0EC1002356
:108C30006046F7F7B5FAC117FFF7A8FF054947F6F1
:108C4000FF730022E0FB0132DB0B43EA424008BD28
:108C50003F420F0040420F00024B03F11802C3E9EC
:108C60000622704718220020EFF31181202383F39E
:108C70001288BFF36F8F054B9A68D37B013BD37388
:108C800081F31188BFF36F8F704700BF1822002057
:108C9000EFF31180202383F31288BFF36F8F034B10
:108CA0009A68D37B0133D373FFF760BE182200208C
:108CB000014B9868704700BF18220020D3B5DDE94A
:108CC0000667089CCDE90067FFF7B4FE1CB1034BB3
:108CD0009B685B69236002B0D0BD00BF18220020F2
:108CE000027C12F01F02034610D10A4988420DD0BF
:108CF0000949086868B1D9897F2909D893F90E20F4
:108D0000064B1B689A42B8BF00207047002070478E
:108D10001046704798050020780200204422002069
:108D2000044BC01A044BC0105843044B01221A5480
:108D3000704700BF18070020ABAAAAAABF6700208F
:108D4000F8B50C4B0C4D1E7C0C4FFFF7C9FF1823D8
:108D500003FB06550446284600F0F0F834B1BB5D2D
:108D60000749E21AD317284600F050F80023BB55F4
:108D7000F8BD00BF1822002018070020BF670020A0
:108D8000218D000070B5EFF31186202383F3128844
:108D9000BFF36F8F0F4D104BAC681868A04202D123
:108DA000FFF7CEFF11E000221A602B7C0B4AD35C48
:108DB0005BB12046FFF794FF38B1237CDB0604D17A
:108DC000FFF708FD6869A042EAD086F31188BFF377
:108DD0006F8F70BD1822002040220020BF67002046
:108DE000024B1868984208BF00207047800200209C
:108DF00008B5044B186820B1FDF782FD024B1B68D3
:108E0000184408BD7C02002048220020B3F1FF3F37
:108E100008BFB2F1FF3F2DE9F84F044699461546C9
:108E20001F4600F081808160EFF31188202383F3D7
:108E30001288BFF36F8FB9F1000FDFF8F4A025DBC4
:108E4000FFF7D6FF3B4B1B68003B18BF01234519BA
:108E500049EBE0795B19DAE9005749F10002C4E90E
:108E600004325D19064642EB07074FF00109FFF790
:108E7000B7FFDFF8C4E0DEF804A00346EBB9C4E9AD
:108E800000EACAF80040CEF8044028E0DAE900120F
:108E90006FF001035B1A4FF0FF3161EB02025B1BC5
:108EA00062EB0902012B72F10001BCBF0123002219
:108EB000C0E904324FF00009D9E7D3E9041CD4E932
:108EC00004208A4270EB0C0B25DA891A5A686CEB85
:108ED0000000C3E90410C4E9003214605C60FFF7CD
:108EE0007FFF84420FD1134B1B6801330BD1B9F1C3
:108EF000000F02D1FFF77CFF0646304604F069F808
:108F00000021FDF7CFFC88F31188BFF36F8F28464F
:108F10003946BDE8F88F521A60EB0C005345C4E99E
:108F20000420ACD01B68A9E700252F46EFE700BF5F
:108F3000300700207C02002080020020F8B50246A5
:108F4000EFF31185202383F31288BFF36F8F01683D
:108F500051B3FFF745FF1C4B5B689A4208D0D1E93B
:108F60000434D2E90476DB1944EB0604C1E9043485
:108F7000D2E90031002400264FF0004790420B60F8
:108F80005960C2E90044C2E9046705D0002085F3B6
:108F90001188BFF36F8FF8BDFFF72AFF04F019F8AF
:108FA0002146FDF77FFCF1E7D0E90413B3F1004F50
:108FB00008BF012904D100204FF00041C2E904019B
:108FC0006FF01500E3E700BF800200202DE9F84FA5
:108FD000DFF8BC902F4CC9F8000000232360FFF796
:108FE000FFFEDFF8B4800D4601264FF00047D9F8A8
:108FF0000020D8E900CE4FEAE27A50B1D0E904313E
:109000009A427AEB010B1EDA9B1A61EB0A01C0E966
:10901000043112EB0C024EEB0A030026C8E90023D0
:1090200030464FF0FF332360C9F8006003F0D1FFF2
:109030003146FDF737FC85F31188BFF36F8FBDE82C
:10904000F84FFFF79FBE13EB0C0CA2EB0303C9F81C
:109050000030D0E90032D0F808A0136041EB0E01D7
:109060005A600023C8E900C1C0E90033C0E90467C1
:1090700085F31188BFF36F8FD047EFF3118520235D
:1090800083F31288BFF36F8FFFF7AAFEAFE700BF2D
:10909000482200207C0200203007002010B5EFF3AA
:1090A0001184202383F31288BFF36F8FFFF7A0FE94
:1090B000054A0346D2E90001181841EBE37184F335
:1090C0001188BFF36F8F10BD300700202DE9F041EC
:1090D0000446EFF31187202383F31288BFF36F8FC9
:1090E000D0E904234FF00046B34208BF012A05D05F
:1090F00087F31188BFF36F8FBDE8F081D0E90A587C
:109100006A1C48F10003022A73F1000324D303F020
:109110007BFF281848EB0101012871F1000141DBB8
:1091200003F072FF6FF00203281848EB010183423D
:109130006FF000438B413ADB03F066FF6FF00102F2
:109140002D1848EB01084FF0FF33521B63EB080367
:1091500018492046FFF75AFE236B01332363236A25
:1091600063B187F31188BFF36F8F20469847EFF301
:109170001187202383F31288BFF36F8F54F8185F91
:10918000A542B5D0002DB3D0284603F088FE0023B9
:10919000AB6787F31188BFF36F8F2846BDE8F041B6
:1091A00003F06ABE6FF001024FF0FF33D0E70022F8
:1091B0003346CDE7CD900000F8B5044616461D466F
:1091C000EFF31187202383F31288BFF36F8FB5F17C
:1091D000FF3F08BFB2F1FF3F04D187F31188BFF30F
:1091E0006F8FF8BDFFF7AAFEDDE906010023C4E991
:1091F0000A01236332462B4620460249FFF706FE4A
:10920000EBE700BFCD90000070B50546EFF3118489
:10921000202686F31288BFF36F8FFFF78FFE20B1F1
:1092200084F31188BFF36F8F70BD6B6A63B184F3F1
:109230001188BFF36F8F6B6A28469847EFF311844C
:1092400086F31288BFF36F8F05F1180003F064FEF8
:109250000028E5D003F010FE21460248BDE870402A
:1092600003F070BEC0670020F8B507460C461646EE
:1092700003F0A0FD08B10020F8BD0D4B9B68DD6E2A
:10928000002DF8D0221DF6D2EFF31184202383F3B2
:109290001288BFF36F8F47F004012846B04784F36C
:1092A0001188BFF36F8F0028E5D040F8045BE3E737
:1092B000182200200146024A0020FFF7D5BF00BF58
:1092C000FDA7000038B5064C064DAC4201D3002086
:1092D00038BDD4E90112204603F002FF1434F4E74C
:1092E000FC020020FC02002007B5074B0093074951
:1092F00007484FF0FF334FF48062FFF7CBF80020B0
:1093000003B05DF804FB00BF64E7000000A100208B
:1093100038070020054B1B680131434001320840EB
:1093200022EA03020243501E00B27047602200206E
:109330002DE9F04F99B0CDE90210002118460192B5
:10934000059304F082F8002800F0E8818F4B149315
:109350004FF0010915AB05990198ADF83090ADF8C3
:109360003890CDF84090CDF84890139303F0F6FF75
:1093700001301ED1039B33B9029B9BB900231846D1
:1093800019B0BDE8F08F0398002103F06BFF0028AF
:10939000F2D000240094A046A246274626466FF04D
:1093A0008C03D5E0DDE9011003F025FF0028F0D1A2
:1093B000E4E7002501990B950BA8ADF8325003F0B6
:1093C0001AFF0B9EBDF832700446002840F09F81C2
:1093D0000D90ADF83A0005990DA803F00CFFDDF8EB
:1093E00034A0BDF83A800546002840F09581019BE5
:1093F0000F90D988ADF8389002310FA8ADF83090B1
:1094000003F089FE044618B10F9B00932C46C6E773
:1094100001460FA803F026FF0F9B00930028BED142
:10942000019B1190D98811A8023103F074FE119CA0
:1094300083460028B3D10DA803F040FF00F01F00C1
:109440001F2870D0C0F11F0319460BA8049303F026
:109450005DFF0B9EBDF832700028A0D104990DA8C5
:1094600003F054FFDDF834A0BDF83A80002896D10F
:10947000C1463D46A7EB080B4FEA4B1319460DA812
:10948000CDF834A0ADF83A80079303F03FFFDDF844
:1094900034A0BDF83A80002881D1009B03EB8B0BF0
:1094A0000DA90BA80B96ADF83270CDF834A0ADF82D
:1094B0003A8003F082FF00283ADA09F1FF33079976
:1094C00006930DA803F041FF09F1FF330AEB830374
:1094D000079309F18043023B0AEB830305F1FF3B4D
:1094E00005F180450993013D009BA5EB090503EBC0
:1094F0008505069B9B454BD8039B73B10FA9184666
:1095000003F079FE00287FF44AAF019B059A9B88FF
:10951000928813FB02F3039A9380029B002B40F086
:10952000D980002314E0C1463D46CDF810B0A1E734
:10953000DBF800300BA90133CBF800300DAA084648
:1095400004F073F80B9EBDF8327003460028A7D0D4
:109550000BA801930B96ADF8327003F0CEFD0DA869
:10956000CDF834A0ADF83A8003F0C7FD009B0F930F
:109570000FA803F0C2FD11A8119403F0BEFD0C2149
:1095800015A800F061FD019BF9E600BF0100030092
:10959000079B56F82B101A684FEA8B09A9F10400B3
:1095A0003318914208934BD200233058F6F7F8FD58
:1095B000002914BF4FF0FF330346BBF1010F18BF62
:1095C000B1442B6014BF59F8083C00231593089B45
:1095D0001B68169306EB8B031B6817932B680133EC
:1095E0002B602B68013B2B60002111A8119403F024
:1095F00039FE119C00287FF4D2AE069B1BB3099B59
:109600001B682360079B1B68636011A92A680846D2
:1096100004F00FF8119C00287FF4C1AE13A911A823
:1096200003F0CBFE0028DCDC2A68CDF834A00DA9BD
:1096300011A8ADF83A8003F0FCFF30B1119CAEE602
:109640004FF0FF33B9E7069BDBE7009A6FF00703A3
:109650004FEAC50902FB0399494611A803F056FEDB
:10966000119C00287FF49BAE0BA911AA08460B960B
:10967000ADF8327003F0D9FF0B9EBDF8327003468F
:1096800000287FF465AF01460BA803F0DEFE00283A
:109690001CDA0DA911A803F0AEFD0028CED1494671
:1096A00011A803F033FE119C00287FF478AE0BA9BB
:1096B00011AA084603F0B6FF0B9EBDF832700346B0
:1096C00000287FF445AF2B68013B2B600BF1FF3B7B
:1096D000043D0EE704990B960BA8ADF8327003F029
:1096E00034FE019B02989B88ADF830300BA903F043
:1096F00082FD014600287FF452AE029803F0A5FED9
:1097000000287FF40EAF029A0123938009E72C46CC
:109710000095A846AA4642E6009440E66FF00B0387
:109720002DE600BF044B1B68584043085B42404293
:109730001843C017704700BF6022002010B50B4CC3
:10974000226823684240594081EA0200C00FFFF7B7
:10975000E9FF2368521A434022EA030208401043FB
:10976000BDE81040C00FFFF7DDBF00BF6022002042
:109770008842F0B504D0094F04380025AA4200D130
:10978000F0BD3E6850F8044F5E4024EA060451F8EC
:1097900025601E40344304600135EFE7602200205D
:1097A0002DE9F74F0025DFF854B0804689469246F0
:1097B0002C469D4203D1204603B0BDE8F08F59F8F6
:1097C0002560019321463046FFF7B8FF361B5AF853
:1097D0002510DBF80020009107463046FFF7AEFF6A
:1097E0000099DBF80020019B00F0010407F001075D
:1097F000761A48F825603C440135DAE760220020FB
:109800008B422DE9F84328BF0B46DE08089CA1EBEC
:10981000030803F00709844615460346B6460021AF
:109820000EF1FF3EBEF1FF3F03F1200305F12005DD
:1098300014D102EB46104FEA89050CEB461600EBFB
:109840008907ACEB0202B84279D14A4C2E44B8F1F8
:10985000000F40F083800846BDE8F88355F8207C6F
:10986000A7FB0470CF1953F8201C40F10000CF195A
:1098700043F8207C55F81C1C40F10000A1FB0417A4
:10988000401853F81C1C47F10007091843F81C1C2A
:1098900055F8181C47F10007A1FB04107F1853F876
:1098A000181C40F10000C91943F8181C55F8141C85
:1098B00040F10000A1FB0417401853F8141C47F1B5
:1098C0000007091843F8141C55F8101C47F100074D
:1098D000A1FB04107F1853F8101C40F10000C919B7
:1098E00043F8101C55F80C1C40F10000A1FB0417B4
:1098F000401853F80C1C47F10007091843F80C1CDA
:1099000055F8081C47F10007A1FB04107F1853F815
:10991000081C40F10000C91943F8081C55F8041C44
:1099200040F10000A1FB0417401847F1000153F873
:10993000047C3F1841F1000143F8047C70E7844641
:109940005CF8043BA3FB043ECB1881584EF1000E9B
:10995000CB1883504EF10001604674E7306808442C
:1099600046F8040BFFF7EAFE08F1FF38236800F021
:1099700001016CE7602200202DE9F04F8DB01D46FB
:10998000189B179F1A9E0592B3F12A3F83468A4679
:1099900040F08D803946169803F0A7FF012838BFA4
:1099A0000120470900F01F047B01502B34BF012325
:1099B0000323012B0A930CBF022308230B930A9B5A
:1099C000059805FA03F306EB8303069303EB85037F
:1099D000079304F087F84FEA850808904246002173
:1099E000304604F079FB01233360079B0393089B07
:1099F000199ACDE90153059B009331462B46304619
:109A000006EB080904F082F851464246484604F045
:109A10003CFB0223494609930B9B099A934248D188
:109A200042463146584604F030FB4FF00009CA4622
:109A3000079B0393089BCDE90153059B00935A466E
:109A40002B465946584604F061F8002C47D1013F97
:109A50001F24169B53F82730E34003F0010343EA29
:109A600049090A9B0AF1010A534503D0002CDFD1B2
:109A7000002FDDD1189BB3F12A3F32D10698424620
:109A800009FB086104F001FB079B0393089B069AFE
:109A9000CDE90153059B009359462B46584604F0E7
:109AA00035F8002CC1D1BFB90DB0BDE8F08F00244E
:109AB0007AE7079B0393089B01EB080ACDE9015362
:109AC000059B00934A462B46504604F01FF8099B1D
:109AD0000133099351469FE7A146A246A8E7013CFE
:109AE000B7E731464FF0000A0A4B18681B68584028
:109AF00080EA090080EA0A00FFF714FE2A46C34301
:109B00000698FFF735FE099B0AF1010A53454144C7
:109B1000EAD1B9E76022002070B50021044604F0C4
:109B2000C3F8054610B10E4D284670BD261D3046BF
:109B300003F0C4FB7F28F6D90C342946204603F0F5
:109B4000ADFB0028EFD0204603F0B8FB0128EAD98E
:109B50003146204603F031FC0028E5DBE3E700BF97
:109B600000BEFFFF2DE9F04FCFB00446039100F196
:109B7000480346AD00F16806186859682A4603C2D2
:109B80000833B3421546F7D104AAD2E94483D2E997
:109B90004797D2E942160193D2F824B13D4BD2F84F
:109BA000185102934FF0000CBCF10F0F5AD8039BD1
:109BB00053F82C301BBA4FEAF52E87EA0900DDF87E
:109BC00008A093608EEAB51E28408EEA756E784034
:109BD00070445AF804EBCDF808A0704403444FEAEF
:109BE000713E46EA010006EA010A8EEAB10E00EA79
:109BF000080040EA0A008EEAB15EDDF804A0CDF864
:109C000004800CF1010C5B448644BCF1400F9A4483
:109C100002F104027344BB461DD104A8C0E9489771
:109C2000C0E946A5C0E94468C0E94231C0E9003E48
:109C300045A904F14403643453F8042F51F8045F38
:109C40009C422A441A60F7D14FF4947100F0FCF959
:109C50004FB0BDE8F08FB0464F460E46A9461946B4
:109C60005546A1E7136852F834AC52F8380C4FEA65
:109C7000F34E8EEA734E8EEA932E52F8143C034450
:109C80004FEABA4080EAFA10734480EADA000344EB
:109C900091E700BF70E7000003460846C1B9C3E979
:109CA00010110D4A0D49DFF838C0C3E912120D4AF0
:109CB0000D49C3E914C20D4AC3E916120C4A1A66CB
:109CC00002F17452A2F52302A2F692425A6670473C
:109CD0006FF08600704700BF85AE67BB67E6096A14
:109CE00072F36E3C3AF54FA57F520E518C68059B7E
:109CF000ABD9831F0928024818BF0020704700BF56
:109D0000CDEE000001680E4A9142034615D1C169AB
:109D1000A2F11022A2F1EF1291420ED18268012A23
:109D20000BD8C26812B101698A4206D0586928B1BD
:109D30009B691B1A5842584170470120704700BF69
:109D400055AA00FF70B50E4B9E68B6B13046FFF7BE
:109D5000D9FF044618B9F3687BB935690DB92046B7
:109D600070BD2846FFF7CEFF28B9EB68B34204D197
:109D70002E462D69F2E70446F1E70124EFE700BF24
:109D80004C2200202DE9F8433F4E3468D4B1B4682A
:109D9000C4B1002875D0002973D001FB00F5B5FBD4
:109DA000F0F088426DD1281D6BD8A9070DD025F0A1
:109DB00003070437F46803E06368BB4207D2A46971
:109DC000002CF9D12046BDE8F8832F46F2E7A368BE
:109DD0001BB12E4B01201B6898476268D21B232AB7
:109DE00004F120081FD80123A360D4E90523C2B1E0
:109DF0009361A3690BB162695A610023C4E9053319
:109E00003369DA0706D5FFF79DFF18B11F4B1B68B2
:109E1000012098472A4600214046444604F05CF958
:109E2000D0E7F360E5E707F120016318203A5A60B4
:109E30000022C3E90224164822691A6160501549BC
:109E4000D96102B1D36062695A61A1699961B2B105
:109E500093619A6902B153614FF00109C4E9017934
:109E600023610023C4E905333369DB07D2D5FFF74B
:109E700069FF0028CED0054B48461B68C9E7F36050
:109E8000E7E700249EE700BF4C2200208802002064
:109E900055AA00FF669911EE70B50546002800F03E
:109EA0008480424E3368002B7FD0B268002A7CD079
:109EB000834203D872681344984203D33C4B012079
:109EC0001B689847A5F120042046FFF71BFF18B137
:109ED000374B01201B68984755F8183C012B03D0DD
:109EE000334B01201B68984755F8143C002245F875
:109EF000182CC3B19968002942D155F81C2C02F1E5
:109F000020015A680A445A6055E905321A6155F829
:109F1000145C2B6903B1DD6020462022002104F08F
:109F2000DBF823462C462069002836D08268002AB8
:109F300033D163684268203313446360036923614B
:109F4000D4E90523F2B923BB436963618269A26145
:109F50000BB39C61A36903B15C61236903B1DC604D
:109F60002022002104F0B8F833699B071DD5FFF7C4
:109F7000E9FED0B10E4BBDE870401B6801201847C8
:109F80001346D0E79361A369002BDDD062695A6163
:109F9000DAE7F360F7E7F460DCE7002BE4D1F3687D
:109FA000A36103B15C61F460DEE770BD4C22002068
:109FB0008802002038B514220C46054600211348BB
:109FC00004F08AF81249134800F034F8232C1CD905
:109FD00015F003031FBF043CE418C3F10403ED189C
:109FE00022460021284604F077F8084B0A499D6074
:109FF000C3E90054203C6C609A6811609A68DA608A
:10A00000A1F11021A1F1EF11D16138BD4C22002046
:10A01000999E0000859D000055AA00FF014B1B681A
:10A02000184700BF90020020014B1B68184700BF73
:10A030008C020020024B1860024B00201960704710
:10A04000900200208C02002010B50A46044619B187
:10A05000024B00211B68984710BD00BF70E800004C
:10A06000F0B5114C059F24684440002B14BF9C465A
:10A070008C46E443002303F1040E774502D2BB4231
:10A0800009D3F0BDD5585CF8036005402640354340
:10A09000CD507346EFE7D55C1CF8036005402640C1
:10A0A0003543CD540133EAE760220020054B5A784E
:10A0B000022A04D11878C31F584258417047002023
:10A0C000704700BF6422002010B5114C2378580758
:10A0D00044BF03F0FB032370990705D500F052F845
:10A0E000237823F00203237063781BB1094A00230D
:10A0F000636053600023074863700821FFF7A4FFE3
:10A100002378DA0744BF23F00103237010BD00BF9A
:10A11000642200206822002038B5FFF7C7FFD8B9B5
:10A12000124C2378DA075CBF43F0010323709D07CC
:10A1300007D400F01FF8237843F00203237005468C
:10A1400088B9627832B9D90704D5094962604A6092
:10A1500002226270580702D50025284638BD43F018
:10A1600004032370F8E7FFF7AFFFF6E7642200204F
:10A1700068220020024B012283F840230020704710
:10A1800070420020F8B5094C002501270326E7613D
:10A1900026762046013503F05AFF102D04F50D7484
:10A1A000F5D1034B002283F84023F8BD7022002034
:10A1B00070420020F8B50E4B1D68AB789B07064631
:10A1C00012D56F6816F8014B29462CB90A20B847FA
:10A1D000002805DB204609E02046B8470028F1DAD0
:10A1E000AB7843F00403AB704FF0FF30F8BD00BF15
:10A1F00080E600000CB430B58BB004460D4620223A
:10A20000002102A803F068FF02238DF80A30002D18
:10A210000C4B0393069412DB01D06B1E1C440FAA57
:10A220000E99079402A8019200F00EF815B1069B52
:10A2300000221A700BB0BDE8304002B07047002415
:10A24000EDE700BF4BE100002DE9F04F8378D0F837
:10A25000048015469A0785B0074640F19F80002686
:10A260000878002800F09C80252808D001F1010A18
:10A2700001363946C047002880F286808AE091F88E
:10A2800001B0BBF1250F01F1020AF1D00024012138
:10A290001F2C25D8ABF12002102A06D8844B01FAD6
:10A2A00002F018420ED1032A5AD0ABF13002092A2B
:10A2B00008D9BBF12A0F33D1630605F1040501D497
:10A2C00044F020041AF801BBBBF1000FE0D139467D
:10A2D0002520C04700285DDB023639465846C9E7CD
:10A2E0007F2CE2D9BBF16C0F29D021D8BBF1680FCC
:10A2F0002CD0BBF16A0F30D0BBF14C0F2DD0ABF19D
:10A300006302122A00F2A580DFE802F02C4EA3A31C
:10A31000A3A34EA3A3A3A3A3AD9DA3A331A377009F
:10A32000BBF12E0FDED160063AD444F04004C9E7F9
:10A33000BBF1740FC6D0BBF17A0FC3D0DFE72206A2
:10A3400048BF44F4007444F08004BBE7E30548BF11
:10A3500044F4007444F48074B4E744F42074B1E726
:10A360001024AFE715F8040B0136394682E72C6854
:10A37000504B002C08BF1C46A1464B4619F8010B58
:10A3800020B9341B1E190435514669E73946C047C8
:10A390000028F2DABB7843F00403BB704FF0FF36BD
:10A3A000304605B0BDE8F08F20061DD5A10545BF9C
:10A3B000073525F0070555F8040B55F8080B00285C
:10A3C0000DF10409B8BF404249464FF00A02B8BF38
:10A3D00044F4806403F09FFE6405A0EB090956D4A1
:10A3E0004C460DF1040B5EE0E20555F8040BE6D592
:10A3F000A3054CBF40B200B2E1E724F01004A4B2C0
:10A400000A22200633D5A10545BF073525F00705EB
:10A4100055F8040B55F8080B10B924F01004A4B239
:10A420000DF10409494603F076FEE306A0EB0909A5
:10A43000D6D539463020C0470028ABDBBBF1000F32
:10A440001ED10136CCE744F0100410224FF0780BF7
:10A45000D7E74BF02002782A7FF439AFCBF17802AE
:10A4600042F01002CDE708224FF0000BC9E7E305E8
:10A4700055F8040BD0D5A1054CBFC0B280B2CBE7D4
:10A48000023639465846C0470028A9DA82E7013625
:10A4900039462D20F7E7013C39461BF80400C04738
:10A4A0000028FFF677AF002CF5D14E446CE700BFD3
:10A4B0008128010094EC000038B5044C044DAC42F6
:10A4C00000D138BD54F8043D9847F8E7000000007B
:10A4D000000000007047F0B41346DA02876806698E
:10A4E00007D513F4402F1EBF43F3000202F44022AD
:10A4F0005340346801258D4023F48012DB074CBFA4
:10A500002C43AC4334603B68F0BC1847012303FA8A
:10A5100001F103691B68194203D022B183681B69EA
:10A5200003E0002AFAD08368DB681847002914BFCB
:10A530006FF01500012070470020704730B50029EA
:10A5400085B00446154611DB83688B420ED96368DB
:10A55000C068194401AA01F046F828B96268019B55
:10A560009B1A2B60029B6B6005B030BD6FF0210021
:10A57000FAE7704700EBC100408840087047F8B523
:10A580000346FFF7F7FFB0FA80F0C0F11F0003EBBE
:10A59000800CCA00DCF81060171D0C4606328DB224
:10A5A00056B9012101FA00F0D9680143D960CCF80D
:10A5B0001040DD539D52F8BDF1000431585AD85374
:10A5C00003EBC0009E52C5805D52F4E710B500EB6E
:10A5D000C104E3888B4202F104010AD1012303FA8A
:10A5E00002F2C36823EA0203C360002340F821306B
:10A5F00010BDA28840F8213000EBC20100EBC3007F
:10A60000CB808280F4E708B50346FFF7B3FFB0FACA
:10A6100080F2C2F11F021846BDE80840FFF7D6BF1E
:10A620002DE9F843B1FA81F3C3F11F0200EB82096F
:10A630000646D9F810700D4687B9C3F120034FF0D4
:10A64000FF349C40F3681C4014D094FAA4F2B2FA90
:10A6500082F2131D56F82340214608E03C464FF095
:10A66000030821463046FFF785FF854205D830466E
:10A67000FFF7ACFF2046BDE8F88306EBC404B8F151
:10A680000108E488C9F81040D7D0BC42E9D1D4E72A
:10A6900038B50446FFF76EFF0D46034611462046C7
:10A6A000FFF768FF03449BB204EBC5055A006A80BC
:10A6B0002046FFF75FFF014424F8313038BD70B504
:10A6C0000446FFF757FF0B4604EBC305511A9B1ACC
:10A6D00089B203444E009BB204EBC2006E805D0061
:10A6E000458024F8321020461146FFF743FF01440D
:10A6F00024F8313070BDF8B5002951D004680D1F21
:10A700002D1BEE0825F007056219538813F001038D
:10A7100006D183F31188BFF36F8F0423184602DF3D
:10A7200031462046FFF726FF304434F83030C01A57
:10A73000B04207D0002383F31188BFF36F8F042347
:10A74000184602DF538823F0010353803146204628
:10A75000FFF710FF371804EBC7035B88DA0708D44C
:10A7600039462046FFF74FFF3A4631462046FFF76D
:10A770008FFF655B751B04EBC5035B88DB0709D4A2
:10A7800029462046FFF73FFF324629462046FFF77D
:10A790007FFF2E4631462046BDE8F840FFF7EFBE6A
:10A7A000F8BD70B509B9002070BD056801F0070358
:10A7B0000B33CC0804EBD304AB689C4228BF1C4687
:10A7C00021462846FFF72CFF06460028EBD001461D
:10A7D0002846FFF7CFFEA04207D932192846FFF7D7
:10A7E0006EFF11462846FFF7CAFE05EBC60210466B
:10A7F000538843F0010353800430D5E71146FFF737
:10A80000D0BF043A2DE9F843CC1D114424F00704CD
:10A8100021F00706A6EB04084FEAD807B7FA87F23B
:10A82000C2F12405AD004FF000090735C2F1200246
:10A83000ED0804604946A760C4F80C90920004F14A
:10A84000100003F049FCAAB2530043F001036380F7
:10A850007B1B9BB204EBC5015800A4F80090488014
:10A8600024F83520A6F8029024F8083004EBC7033A
:10A8700029465A8842F001025A802046BDE8F84332
:10A88000FFF77DBE002070470FB407B504A951F84B
:10A89000040B0191F5F712FF03B05DF804EB04B06F
:10A8A0007047036800220BB9184670478B4210D1DD
:10A8B0000B6842B942680360914200D143600023B3
:10A8C0000B600120704713604368994208BF4260E3
:10A8D000F5E71A461B68E6E7038B13F0070306D17A
:10A8E0000368002B18BF032008BF00207047022B0D
:10A8F00005D1408BB0FA80F0400980007047012BF1
:10A9000004D10368002B18BF0520EDE70020704735
:10A9100010B50C4600B111B96FF0150010BD081D3F
:10A9200000F0C6F80028F9D1A368032BF6D9F3E7A5
:10A930002DE9F0410D4607461946281D90461E4652
:10A9400000F0C7F8044638B1334642462946384637
:10A95000A446BDE8F0416047BDE8F08110B4EFF3D4
:10A960001182202484F31288BFF36F8F416110BCE1
:10A970000121F5F7EBBF38B50C46054658B151B18A
:10A980000B6843B14B6833B11C22002103F0A4FBD8
:10A990002C61002038BD6FF01500FBE7F8B50446C8
:10A9A0000E46FFF7B5FF051E3BDBEFF311822023B8
:10A9B00083F31288BFF36F8F638B278B4FF6FF7182
:10A9C0008B4207F007072ED0062F2FD8DFE807F0BD
:10A9D000182E082E180418006FF08505002303E0D8
:10A9E000013363830225012382F31188BFF36F8F44
:10A9F000BBB100233A4631462046FFF799FF10E0ED
:10AA000000233360636823B9C4E9006627B13D467B
:10AA1000E4E71E606660F9E702212046F5F796FF3D
:10AA20003D462846F8BD6FF00A05D7E76FF00405EC
:10AA3000D4E710B5EFF31182202383F31288BFF31C
:10AA40006F8F048B04F00704022C0AD0012C0CBF7A
:10AA50006FF004006FF0850082F31188BFF36F8FF1
:10AA600008E0438B013B9BB2438323B92146F5F7B2
:10AA70006DFF204610BD2046EEE738B5A8B1A1B164
:10AA8000EFF31185202282F31288BFF36F8F048BBE
:10AA9000FFF707FF30B104F0070085F31188BFF31B
:10AAA0006F8F38BD6FF07700F7E76FF01500F8E7AC
:10AAB000034658B1426802F00302012A03D0032A78
:10AAC00004D1026812B10020986070476FF0150041
:10AAD00070474268816002F00302032A4FF00002CF
:10AAE00003460CBF006810465A60704770B50C886A
:10AAF00006468888241A3069A4B2844285B224BFED
:10AB0000641BA4B22D1BA8B2984228BF1846336814
:10AB1000234413600B8803440B8070BD70B4838999
:10AB200085880669ED1AADB2731B934228BF1346A0
:10AB300070BC0A46011DFFF7D9BF70B40E4601462E
:10AB4000C58831F80A3FEC1AA3B2934228BF1346D6
:10AB5000324670BCFFF7CABF10B54B880C88E41AA8
:10AB6000A4B294420ED31A4492B28B884A800A80CF
:10AB70000069D21A92B2824201D2002010BD034471
:10AB80008B80FAE76FF01500F8E72DE9F3410646F0
:10AB90000F4615464FF000082A4601A93046FFF738
:10ABA000BDFF044640B102463946019803F06DFAF4
:10ABB0002D1BA0442744EFD14246311D3046FFF7FC
:10ABC000CBFF404602B0BDE8F0812DE9F3410746D6
:10ABD0000E4615464FF000082A4601A93846FFF7F1
:10ABE000ACFF044648B12EB102460199304603F04D
:10ABF0004CFA26442D1BA044EED1424607F10A012F
:10AC00003846FFF7A9FF404602B0BDE8F081704723
:10AC10000FB407B504A951F8040B0191F5F74EFDE7
:10AC200003B05DF804EB04B07047002908DB8068CE
:10AC3000884205D9401A904234BF00200120704755
:10AC40000020704770B516461A4605460C46FFF7B9
:10AC5000ECFF48B16968E8682144826814683246AC
:10AC6000A446BDE8704060476FF0150070BD70B538
:10AC700016461A4605460C46FFF7D7FF48B16968E5
:10AC8000E8682144826854683246A446BDE87040B2
:10AC900060476FF0150070BD10B50B460446FFF716
:10ACA000C4FF40B16168E068194483689B682BB1B8
:10ACB000BDE8104018476FF0150010BD6FF0570049
:10ACC000FBE708B5C0688368DB689847006808BD83
:10ACD00008B5C0688368DB689847407908BD30B51F
:10ACE0004C680368A34201D2012030BD8A68224427
:10ACF000934201D30020F8E7D1E90452954203D3EF
:10AD00006FF00B038B61F5E7CA681B1B42F8353007
:10AD10004368086902EBC00253600B6901330B61A1
:10AD2000E2E737B50C46C0B201A91546F5F708FFB2
:10AD3000002807DB019828B12A462146F5F726FFAF
:10AD400003B030BD6FF01500FAE710F0700F08D1B6
:10AD500000F07F0310F0800F18BF103301209840DF
:10AD60007047002070472DE9F84306460F4690468D
:10AD7000994604254B46424639463046F9F7B2F823
:10AD800010F10B0F044603D102F03CF8013DF1D164
:10AD90002046BDE8F883006840B150F8043C5B6889
:10ADA0008B42A0F1040001D04068F5E770470068CD
:10ADB00050B150F8043C5B685B689B788B42A0F113
:10ADC000040001D04068F3E7704730B5006888B1EF
:10ADD00050F8043C5B681A6A1D7F04380023043A6B
:10ADE000DCB2A54201D84068F1E7013312F83340E4
:10ADF0008C42F5D130BD08B5F6F796FC28B1406815
:10AE000010F1100F14BF0020012008BD4B1CDBB255
:10AE10008170817680F82530C37600F8061C704773
:10AE200050E90231D0F89C0018470369002283F8EA
:10AE30004A207047036993F84A0050B193F84800DC
:10AE400038B1D3F890209388918910695B1A9BB22E
:10AE5000C01A70470369002283F84B2070470369CA
:10AE600093F8490008B193F84B00704708B50246C3
:10AE7000FFF7F5FF28B91046FFF7DCFF003818BFD1
:10AE8000012008BD0369C3E90012704770B5046969
:10AE90000546D4F88C00FFF798FE94F8A0300646DB
:10AEA000B3B1D4F88C209388918912695B1A9BB254
:10AEB000D31A3F2B0CD994F89E3033B16B681B6AC0
:10AEC0002246187B0021F6F721FF002384F8A030EA
:10AED000304670BD08B50122FFF7D8FF013818BF12
:10AEE0004FF0FF3008BD0269D2F890108B88888936
:10AEF00009691B1A9BB2994204BF002382F84830AB
:10AF0000D2F88C30D9885B89994204BF002382F83B
:10AF1000493070472DE9F0479AB0DDE9245768467B
:10AF20000C46229E9246994602F0A3FF00216846F5
:10AF3000FEF7B2FE35B1002F04DD3A4629466846D9
:10AF400002F0A0FF63892289D4F80C80134498444E
:10AF50000025A84508D82399684602F0D3FF684623
:10AF600002F08BFF00240FE0A8EB0507B74228BFD3
:10AF700037463B464A4629465046FFF763FE04469D
:10AF800030B1684602F079FF20461AB0BDE8F0877C
:10AF90003A464946684602F075FF3D44D9E72DE937
:10AFA000F7430E4617469946044628B94FF0FF3836
:10AFB000404603B0BDE8F0830029F7D0002AF5D061
:10AFC000CB680D891D4404230DEB03022946384646
:10AFD000FFF738FE80460028E8D1BDF804107389D9
:10AFE00046F60812914225D1BDF806109942DDD1EE
:10AFF00004230DEB030229443846FFF723FE002803
:10B00000D4D1BDF8042046F607139A42CED1C4E944
:10B0100000679DF82830A4F80890A3727389BDF8E2
:10B0200006202B44E360738913442B440435636189
:10B030002561BDE7002BE4D0B8E72DE9F3410E46CA
:10B0400017461D46044620B94FF0FF3002B0BDE858
:10B05000F0810368002BF7D04368002BF4D04FF643
:10B06000FF78D4E90413994215D223685B8923B190
:10B07000E3688B4204BF04312161042360680DEB57
:10B080000302FFF7DFFD0028DED1A37A2BB1D4E95C
:10B0900003329A4201D30120D8E72389BDF8061074
:10B0A000434501F1040203D0BDF804C09C450BD117
:10B0B00015B1BDF804302B80236904333360398027
:10B0C000236913442361C1E7236913442361C8E75B
:10B0D00048B103683BB143682BB1C068884294BF54
:10B0E0000020012070474FF0FF30704703F003B895
:10B0F00010B50446FFF7E5FD00F01DF8A36898427F
:10B1000001D900F01AF9181A10BD0846FFF7F0BF70
:10B1100013B57423012904460193084608D1626AD5
:10B1200001A9FFF7FEFD08B9019BA36202B010BDA3
:10B130000120FBE77047302070472DE9F7431F4699
:10B1400083688B4206460D46914633D95B1A93427B
:10B1500030D307B36A46FFF7F1F9041E2CDB013D3B
:10B16000DDF800804D446A4629463046FFF7E6F98F
:10B17000041E21DBDDE9009530462A464946FFF7EB
:10B180008BFD041E18DBF5F773FA77B1C84513D2AF
:10B1900009F1FF35E7E701396A464944FFF7CEF97F
:10B1A000041E09DBDDF80080DDE74D44A84503D32C
:10B1B0000135D8E74FF0FF34204603B0BDE8F083F7
:10B1C0003422002102F088BF00F120010120F5F7B0
:10B1D000B7BC704770B506460D460024AC4200DB94
:10B1E00070BD305DF7F7E8F80130F9D00134F5E7CC
:10B1F0002DE9F04F85B005460E4690461F4601F0FA
:10B2000093FA20B96FF04C0005B0BDE8F08F002331
:10B210004FF014093B6009FB086934464FF0010AFE
:10B2200002A9284601F074FA60B1DDE902324FF05C
:10B23000000B0093C3450CD10021284601F0B4FA5D
:10B240000028EDD1284601F098FA0028DAD0002035
:10B25000DAE7A14598BF344661688A4214D1216873
:10B260000098019202F047FF019A68B9237C7BB9EC
:10B27000D4E902312846984768B184F810A03B68A9
:10B28000013314343B60CBE714340BF1010BD1E7ED
:10B290006FF06F00B8E76FF02200B5E702F01CBF57
:10B2A00002F0F3BE012801D1EFF30583FCF732BDB4
:10B2B00001460068FFF7F6BF08B5F7F733FDBDE8B4
:10B2C0000840F7F78BBF00210120FFF7EBBF6FF0BD
:10B2D0008500704761B662B680F31188BFF36F8F47
:10B2E000704772B6002383F31188BFF36F8FBFF3EB
:10B2F0004F8F30BF62B6BFF36F8F704772B60023B7
:10B3000083F31188BFF36F8FBFF34F8F20BF80F39C
:10B310001188BFF36F8F62B67047202809D9B0F14A
:10B32000004F08D80138B0FA80F0C0F11F0040008B
:10B330007047082070473E20704708B5F8F70AF9B3
:10B3400008B5F8F7FFF8002008BD70470A448A42A4
:10B3500000D1704711F8013B40BA80B25840C0F3A9
:10B3600003134340180380B24340580100F4FF50D8
:10B370005840ECE710B50369C0E905330023C3600A
:10B38000837F044613B1407AF9F73EFC012323770B
:10B3900000236377E377A37710BDFCF725BEFCF7A6
:10B3A00095BE0378027903F00F011AB951B14FF03D
:10B3B000FF3070470829FAD8012A03D1C3F3C0002F
:10B3C0000138704743F3C000704738B50146F8F7BD
:10B3D00017F9054660B1037A6BB108460024F9F706
:10B3E00095FC2846AC77FFF7C5FF2C72204638BD88
:10B3F0006FF01500FBE76FF07700F8E770B50446D3
:10B400000E461546F8F7E4FD30B906B925B12046D9
:10B41000BDE87040F8F724BE70BD4FF08053D3F8FC
:10B420003021082A05D1D3F83401003818BF012093
:10B43000704700207047C343C3F3C01300F00F00F0
:10B4400000EB0310704708B5F8F778FE818208BD5D
:10B4500008B5F8F773FEEFF31183202282F3128808
:10B46000BFF36F8F02690A60027B2AB9807D83F384
:10B470001188BFF36F8F08BD0420F8E7FCF7A8BE62
:10B480000369C9B20C2202FB0133186C00F00700FB
:10B49000704770B50346C9B20069EFF311862024E6
:10B4A00084F31288BFF36F8F0C2505FB0104246C15
:10B4B00014F0C00401D0A24211D105FB0100012209
:10B4C0000264002086F31188BFF36F8F30B95B6888
:10B4D0000C2202FB01335B689847002070BD4FF0DF
:10B4E000FF30EFE78022FFF7D4BFF8B5069F04696D
:10B4F0000546C9B2EFF3118C202080F31288BFF308
:10B500006F8F0C2606FB0146306C00F0070EBEF173
:10B51000010F10D1376400268CF31188BFF36F8FB1
:10B520003EB90C2041430C44C4E90E236B685B58C0
:10B5300098473046F8BD00F0C00087420CBF6FF05E
:10B5400077064FF0FF36E7E713B580240094FFF746
:10B55000CCFF02B010BD10B40069CBB21C2404FBB8
:10B560000300002110BC10471046FCF731BE08B59F
:10B57000FAF742F9BDE8084000F0BBBBFBF7BABBE5
:10B58000FAF788B8F7B51C46164600238268236090
:10B59000A36053690D4601AA69469847019B5A1E4C
:10B5A00001921BB96FF0150003B0F0BD0098A268BE
:10B5B00047682168676085B9B31AD0F800C0634551
:10B5C00028BF63461A4403FB07112160A26002688A
:10B5D0009A4206D808300090E0E76B1AB3FBF7F305
:10B5E000EBE70020E0E713460022FFF7CBBF2DE991
:10B5F000F047836886B05B698846914601A902AA34
:10B6000098470024A2462546029BAB4202D806B0CA
:10B61000BDE8F087019F07EBC50700267B68049310
:10B620003A68B2420AEB060302D801359A46EBE7C4
:10B6300003940593494603A8C0470028E7D0049B1C
:10B6400001361C44ECE710B50C4600F013FE002355
:10B65000C4E90003184610BD38B505460C4600F095
:10B6600009FE002D07DBA84205D9401B84428CBF90
:10B670000020012038BD0020FCE770B50D462846AB
:10B68000194616461C46FFF7E7FF38B124B122469B
:10B690002946304602F0F9FC002070BD6FF015001D
:10B6A000FBE743685B68D3F810350B6000207047F8
:10B6B00043685B6802EA010021EA0201C3F8080559
:10B6C000C3F80C150020704743685B680020C3F87E
:10B6D0000815704743685B680020C3F80C15704775
:10B6E00043685B68D3F8042521EA02001140C3F8DF
:10B6F0000805C3F80C150020704730B50369586879
:10B7000000B30024884219D108688CB99C6858603D
:10B71000A14200D19860002008602AB15A680A60EE
:10B720009A68596002B9996000200FE02846E9E75D
:10B7300020609868814208BF9C60ECE70568044679
:10B74000002DF3D1002AE9D16FF0150030BDFBF7D1
:10B7500015BC13B54FF080520829136E526E28BFE6
:10B76000082112BA00921BBA0C460A466946019398
:10B7700002F08BFC204602B010BD30B54368136068
:10B78000057A446804EBC504A34202D36FF00100BC
:10B7900030BD5C798C4203F10803F0D10020F7E75B
:10B7A0004379014623B151F8060B83681B6818479B
:10B7B0006FF08500704737B52A294568046901D0C4
:10B7C0004C2914D16846D4E9062301F044FCDDE994
:10B7D000000101F0BAFB2846FFF7E2FF48B92868EC
:10B7E00083685B68214603B0BDE8304018476FF0BE
:10B7F000850003B030BD43681B68D3F88004C3F8EC
:10B800008004704742681368D3F8100150B1D269C0
:10B81000002012780A70C3F81001D3F81021012219
:10B820001A6070474FF0FF307047002A0FDD426802
:10B830001368D3F8100158B10020C3F81001D26981
:10B84000D3F8100112780A700120186070470020A8
:10B85000704710B543681C680369EFF3118020221C
:10B8600082F31288BFF36F8F1A68D17B39B9917355
:10B870001B680122DA734FF48003C4F8043380F3A9
:10B880001188BFF36F8F10BD03691A68D17B21B196
:10B89000012191731B680022DA73704702691168F5
:10B8A0000346C87B40B15B681B68D3F8580118B1E8
:10B8B00000230B6113689889704743681B68D3F8AD
:10B8C0001001003818BF0120704743681B68D3F887
:10B8D0000423D2065CBF1022C3F8042370474368D8
:10B8E0001B68D3F80423D20644BF1022C3F80823F0
:10B8F000704743681B684FF40072C3F80423704715
:10B9000043681B684FF40072C3F80823704738B5CA
:10B9100043681D68D5F804335B02044605D4D5F8A6
:10B92000040310F0100006D138BDFFF7B7FF002860
:10B93000F5D00120F8E72046BDE83840FFF7BDBF4D
:10B940000369186801601B685A6070470268034603
:10B95000D2F8580140B95B68DB0706D4D2F8200161
:10B96000003818BF012070470120704710B44368A9
:10B9700002691B68D3F80413C90517D5D3F8201141
:10B98000A1B1EFF31181202484F31288BFF36F8FEC
:10B99000D3F8204134B10024C3F82041D3F820412A
:10B9A0000124DC6081F31188BFF36F8F1168D3F835
:10B9B000584171B17CB100240C611168C97B19B97F
:10B9C0004FF48001C3F8081311688C7B1CB100236D
:10B9D0008B7310BC7047D3F8241121B10021C3F838
:10B9E0002411D3F8243112681368002BF1D0516868
:10B9F00010BC184713B501AA0446FFF7BEFE002885
:10BA000005DB019B226819791868FAF7D9FA02B0A8
:10BA100010BDF8B50022054601210220F7F75EFBB4
:10BA20000220F7F72BFB6C680121E068FFF7E2FFCB
:10BA30006B681A682369C2F82435617D237D0B4346
:10BA4000A17D0B43C2F86C356E68D6E9004313F054
:10BA500001030ED02F6904F10C0107F10C0204F56B
:10BA6000907000F0E0F800283ADB387BFBF774F8C0
:10BA700001230822C4F80025B269C4F84425012135
:10BA80000022C4F84825A1606BB9D4F82031002BFE
:10BA9000FBD0C4F82021D4F820310123E3604FF417
:10BAA0008073C4F80433D4F85831002BFBD0002144
:10BAB000C4F800156D682C68E868FFF79BFF082341
:10BAC000C4F800352A7A52B9EB69C4F83435012339
:10BAD000C4F83835C4F81021D4F8102123600020B0
:10BAE000F8BD2DE9F041066933689C89BFF35B8F8F
:10BAF00094420546A8BF14461033012753E8002F8F
:10BB0000002A03D143E800700028F7D1BFF35B8F10
:10BB10000CBF3B4600232BD133682246986802F0C5
:10BB2000B4FAEFF31188202383F31288BFF36F8FE9
:10BB300069680846FFF70AFF326840B91061044699
:10BB400088F31188BFF36F8F2046BDE8F0810B6842
:10BB50009268C3F844250022C3F84845C3F8202161
:10BB6000D3F82011C3F85821D3F858219F60E7E794
:10BB70001C46E9E700F150039B009BB203F18043B0
:10BB800003F5883300221A601B6870474FF080531A
:10BB9000D3F83021082A03BFD3F83401B0FA80F07B
:10BBA00040090020704703460020184700F055BFA9
:10BBB00010B502461168B1B1BFF35B8FB1FA81F3E2
:10BBC000C3F11F000123834021EA030352E8004F21
:10BBD0008C4204D142E8003CBCF1000FF6D1BFF327
:10BBE0005B8FE7D110BD6FF00B00FBE710B503686A
:10BBF000CB40DB0714D401238B400268BFF35B8F7B
:10BC000043EA020150E8004F944204D140E8001C8E
:10BC1000BCF1000FF6D1BFF35B8FEED1002010BD59
:10BC20006FF01500FBE770B50C460021054608468D
:10BC30001646FAF783FF48B93378DB0003F18043F7
:10BC400003F5F833C3F81055C3F8144570BD10B1AF
:10BC5000012802D07047FBF74DB8FAF7FDBF18B1C5
:10BC6000012803D100F01BB800F043B87047FBF780
:10BC70007DB808B5FBF70CF8BDE80840FBF7B2B893
:10BC80004FF08053D3F83021082A06D1D3F834017D
:10BC900002288CBF00200120704700207047FAF76F
:10BCA000A1BF4FF08053D3F83021082A06D1D3F832
:10BCB000340102288CBF002001207047002070470B
:10BCC00038B54FF080440223C4F808330123E36001
:10BCD0000023C4F80431D4F8043142F21075D4F8CA
:10BCE0001834DB0304D50120FFF760FF013DF6D1D6
:10BCF00038BDFFF7E5BFF7B5019001A8DDE90847BA
:10BD000016461D46FBF7A2F8019BB6F1000C18BFC2
:10BD10004FF0010C00EB83000B1E18BF0123002D18
:10BD200043EA4C030CBF4FF0000C4FF00C0C002CFE
:10BD300043EA0C030CBF4FF0000C4FF4E06C002FF3
:10BD400043EA0C03D0F800270CBF4FF0000C4FF46F
:10BD5000403C43EA0C0322EA030301B109780EB127
:10BD60003678760019430DB12D78AD0031430CB112
:10BD70002478240229430FB13F783F040C433C430D
:10BD8000C0F8004703B0F0BD1FB50DF10F030193DC
:10BD900000238DF80F1000931A461946FFF7ABFFEA
:10BDA00005B05DF804FB10B504460846FBF75EF8E5
:10BDB00004EB4004207DC0F3401010BD10B50446D4
:10BDC0000846FBF753F804EB4004207DC0F3400025
:10BDD00010BD10B504460846FBF748F804EB4004D4
:10BDE000A08A400B10BD70B5044608461646FBF706
:10BDF0003DF808300D4634F81030DA0509D5C3F3A4
:10BE0000432304EBC302314654F8333052682846CA
:10BE10009847A3682BB1E26831462846BDE87040D8
:10BE2000184770BD10B504460846FBF71FF804EB31
:10BE30004000838ADA051DD5C3F3432123F4F85368
:10BE4000838204F1120204F1720032F8023F13F40B
:10BE5000807F03D0C3F3432399420BD08242F4D1B5
:10BE600004EBC10300225A6004F17800BDE81040E1
:10BE7000FFF7BCBE10BDF0B5034600F5807400208E
:10BE800005460127844695420AD1D3F87C2132B178
:10BE90000022C3F87C21D3F87C3140F00040F0BD93
:10BEA00025F0404607FA06F6314209D0D4F800E002
:10BEB000BEF1000F04D0C4F800C0D4F800E0304355
:10BEC00001350434DFE738B504460D46FFF76BFF54
:10BED000A8B12046FFF772FF88B92046FFF779FF27
:10BEE000226801238340C2F80833236803EB8000F3
:10BEF000D0F8103523F00303C0F8103538BD2846BC
:10BF00000021BDE83840FFF73FBF2DE9F043174659
:10BF100085B004460846FAF7A9FFD7F800800E4618
:10BF20000546B8F1000F1ED02046FFF747FF18B1B5
:10BF30002046FFF738FF20BB0023CDE900338DF802
:10BF40000E308DF80F300DF10F0243460DF10E014A
:10BF50003046FFF7D0FE04EB4502938A23F002033C
:10BF600043F0010393827B689BB33146204693F8EC
:10BF70000080D3F80490FFF721FF28B1B9F1000F3A
:10BF80001FD06FF0150027E004EB4500838A23F4EF
:10BF9000604323F020038382B9F1000F11D0B8F180
:10BFA000030FEED87B6821685B6893F800C04FEA06
:10BFB0008C031944B8F1000F11D1C1F81085C1F8F4
:10BFC000108504EB4502938A23F01C0343EA88039F
:10BFD0009382BB6843BB002005B0BDE8F083D1F875
:10BFE000102522F00302C1F8102522681344D3F86B
:10BFF000102522F44F3222F44072C3F81025320289
:10C00000D3F8101502F47C5242EA08420A43C3F8FE
:10C01000102504EB4C03A3F87C60838A43EA4C337D
:10C0200043F020038382CCE7D3E9007831462046F1
:10C03000FFF7F8FE002FCED063689F4206D004F1D0
:10C040007800FFF7B5FD002804DAC5E7A368984536
:10C05000F5D1002004EBC003C3E9017804EB4505EA
:10C06000C0B2AB8A43EA402343F48073AB82B2E7A9
:10C070002DE9F043054685B0084616461F46FAF7F7
:10C08000F5FE0C46804626B32846FFF797FE18B902
:10C090002846FFF788FE18BB05EB4809B9F81430AD
:10C0A00003F01C0313B17378012B19D001238DF811
:10C0B0000F300023CDE90063721CB31C0DF10F019A
:10C0C0002046FFF718FEB9F8143043F00303A9F82F
:10C0D0001430002F3FD021462846FFF76FFE20B9CD
:10C0E0006FF0150005B0BDE8F0833E782B6803EBD8
:10C0F00086030022C3F81025C3F8102505EB48027B
:10C100004FEA860C938A23F4604323F02003938242
:10C11000787800B32968BF7861440004D1F81035FD
:10C1200023F4991323F4F853C1F81035230200F4D3
:10C13000403003F47C5303433805D1F8105500F424
:10C14000801003432B43C1F81035938A43EA4633EA
:10C1500043F0200393820020C4E7C0E90312704734
:10C1600070B504461546FFF71EFE48B10846FAF7BB
:10C170007DFE04EB40040020A38A5B0B2B7070BD96
:10C180006FF01500FBE738B590F88C4005469CB978
:10C1900060222146143001F09FFF2868C0F87C41DE
:10C1A000D0F87C3140F30730F6F768FF012385F8BB
:10C1B0008C30AB67204638BD6FF07700FBE790F816
:10C1C0008C00003818BF01207047FAF789BE2DE9AE
:10C1D000F34104461746FFF7E6FD0D462668F0B129
:10C1E0002046FFF7EBFD8046C8B92046FFF7F1FD7A
:10C1F000820002F5807346F80380F35823681344E5
:10C20000D3F8102542F00102C3F8102527B12268A7
:10C2100001238340C2F8043302B0BDE8F081D6F8B0
:10C220000433002BA4BF4FF00043C6F80433284664
:10C23000FAF71CFE04EB4004A38AC3F38203042B29
:10C2400012D0052B12D001A80195FAF7FFFD019B32
:10C25000D0F81015D94001F001010231284602B092
:10C26000BDE8F041FFF790BD0321F7E70221F5E7B4
:10C27000FFF729BE4FF080531A6958695043704741
:10C280004FF08053186970474FF0805358697047DA
:10C2900000F180431A68002A1FBF00221A601B6841
:10C2A000012008BF002070474FF080434FF46072B8
:10C2B000C3F8042370474FF080434FF46072C3F813
:10C2C0000823704708B5FAF7BDFFBDE80840FFF73F
:10C2D000D0BC10B5A1F58074A4080123A340184078
:10C2E0000AD001F1804101F5E041086820B1002049
:10C2F000086009680AB9012010BD1168194311606E
:10C30000F9E708B500210120FBF760F80028F9D013
:10C3100008BD08B50246FAF7F9FF20B9BDE80840A4
:10C320001046FBF72DB96FF00F0008BD08B5FDF7FB
:10C33000F3FE002818BF6FF0040008BD30B5026A94
:10C340000346D2E9014084424FF0000002D30123AA
:10C35000D36030BD1874506801305060186A42686C
:10C36000541E0268242505FB042218465C1950F867
:10C37000045B42F8045BA042F9D199600120E8E730
:10C38000F0B5064604460F4694460FCE8BB001AD7D
:10C390000FC50FCE0FC5216A33684A682B6022B9DA
:10C3A0000223CB6000200BB0F0BDFB072068A5681E
:10C3B00013D50B682426013A06FB02337E0703D40B
:10C3C0001A7C0AB10F23ECE7224603F1240153F84B
:10C3D000046B42F8046B8B42F9D1B90741BF226A62
:10C3E000536803F1FF335360AC4505D2236A002B39
:10C3F000D8D00422DA60D5E77A0748BF20603B072F
:10C4000001D40120CFE706AB93E80700143484E899
:10C410000700F6E710B502601A44029B8360012909
:10C420004FF00003C26003740375836101D8036297
:10C4300010BD24224A43243A841804628350026ABD
:10C440008C1E9460026A5360026AD360026A13749D
:10C45000026A022953741EBF036A24301860E7E79A
:10C46000182871F100030ED3B0F5807F71F100033D
:10C470000BD3B0F5803F71F1000308D3002914BF3E
:10C4800009200520704701207047022070470320D3
:10C49000704737B508294FF000044FF00005CDE98B
:10C4A00000450A460AD80146684601F0EEFDDDE97E
:10C4B000000103B0BDE83040FFF7D2BF002003B059
:10C4C00030BD00B1C16070474368036083680133C9
:10C4D0008360006AFFF7F5BF08B50268C3689A4237
:10C4E00005D3006A0821FFF7ECFF002008BD0120FA
:10C4F000FCE738B504460D46FFF7EEFF40B1236870
:10C500001B78B5EB531F04D0206A0A21FFF7D9FF2F
:10C51000002038BD10B50446FFF7DEFF38B12368B0
:10C520001A78FF2A05D0206A0A21FFF7CAFF0020E7
:10C5300010BD01332360FBE710B5027D044632B124
:10C54000FFF7E8FF48B1002323754FF0FF32204684
:10C550000721BDE81040FFF713BF10BD2DE9F84FCC
:10C5600004460E4691461D46FFF7B6FF804628B1A9
:10C57000A36843B90321206AFFF7A3FF4FF0000827
:10C580004046BDE8F88F2268177807F01F0BBBF113
:10C590001F0F12D1FDB1206A18B1037C0BB1152118
:10C5A000EAE701232B7000252368636001352B44E3
:10C5B0002360A368013BA360E2E7BBF1170F0CD92E
:10C5C000ABF11803D9B2032905D801259D40A9452F
:10C5D00004D20521CFE70721CDE70025E36805F167
:10C5E000010A5244934201D20821C4E74A4600217D
:10C5F000304601F071FD15B986F800B0D3E7226826
:10C60000711E531913F8010901F8010F9342F9D172
:10C61000236A002BC8D01B7C002BC5D00737FFB284
:10C62000022FC1D949463046FFF733FF8245BBD0C0
:10C630001521A0E738B50C4611460546FFF759FF0E
:10C6400008B9002038BD04220023A1182846FFF7AE
:10C6500085FF0028F5D02B682360F3E737B500236A
:10C6600004468DF80330FFF744FFA8B104220DF112
:10C6700003030DEB02012046FFF770FF60B19DF848
:10C68000035065B901992046FFF758FE50B9636819
:10C690002360A3680133A360002003B030BD6FF0B6
:10C6A0000F01F0E72575F8E738B504460D46FFF7AA
:10C6B000C1FF48B12268E3689B1A6A689A4204D9AC
:10C6C00008212046FFF700FF002038BD70B50D4659
:10C6D000002104461646FFF70CFF38B132462946C2
:10C6E00020460023BDE87040FFF738BF70BD04222C
:10C6F000FFF7ECBFFFF7FBBF38B5022204460D463B
:10C70000FFF7D2FF18B123686A681344236038BD6D
:10C7100038B5032204460D46FFF7C6FF18B123685B
:10C720006A681344236038BD10B505210446FFF73D
:10C7300095FF50B1237D4BB9A3686FF0004293423F
:10C7400005D305212046FFF7BFFE002010BD5B008A
:10C75000A360FBE7037D23B98068B0FA80F040094D
:10C7600070470368C268934205D21878A0F1FF03AE
:10C7700058425841704700207047FFF7DDBE38B57A
:10C780000D4606210446FFF7B4FE08B9002038BD67
:10C790000023042229462046FFF7E0FE0028F5D0BA
:10C7A000A3680133A360F2E7F0B58FB00446FFF74A
:10C7B00093FE00285DD023681D7800220023CDE978
:10C7C00002236D09234605AA04F120071868596859
:10C7D000164603C60833BB423246F7D118683060AC
:10C7E000062D1CD02A1F0023012A4FF008028DF8C5
:10C7F00004300DEB020198BF01AB05A8FFF7AEFEB8
:10C800000646002835D0042D3BD019D8023D012D15
:10C8100021D9059B2360A368013BA3602AE001A9FD
:10C8200005A8FFF7ACFF20B3059B089A934204D3F9
:10C830000821206AFFF745FE1BE01D786D09CFE750
:10C84000052DE6D1DDE90232B3F1004F72F10001AE
:10C8500013D32946EDE7E3682168029A5B1A9A42EE
:10C8600003D8059B13440593D3E708212046FFF71F
:10C870002BFE002630460FB0F0BDDB185241CDE94B
:10C8800002329DF8045025B16FF00F020023CDE96C
:10C890000223029B07938DF8285005A8FFF75AFF43
:10C8A000014638B1002DB4D005A8FFF733FE0028AB
:10C8B000AFD1DEE705A8FFF777FF0028EDD1D8E775
:10C8C000FFF7A8BD00B1C160704710B50368C46828
:10C8D000A34205D3006A0821FFF7F4FF002010BD32
:10C8E00002F01F0242EA411119700368013303602C
:10C8F0000120F4E770B505460E4610461946144669
:10C90000FFF7C7FD2246431E31462846BDE870406A
:10C91000FBF7D0B9F8B51746C36802689A420446D7
:10C920000D4606D3206A0821FFF7CCFF00263046CB
:10C93000F8BD9B1A4A689A42F4D80E4656F8043B52
:10C9400053B104213046FFF7A4FD6A6823681344FD
:10C95000E26803449A42E5D332460423394620462E
:10C96000FFF7C8FF06460028E0D020682968884203
:10C9700002D06A6801F097FB23686A681344236059
:10C98000D5E7082A73B513460C4606D9006A052177
:10C99000FFF798FF002002B070BD8E1816F9012C29
:10C9A000002A0FDA0A466C466946B24204D10121D8
:10C9B0002246FFF79FFFEEE712F8015BED4301F817
:10C9C000015BF2E70021F3E713460A460021FFF777
:10C9D00091BF07B5042201910DEB0201FFF7D1FFD2
:10C9E00003B05DF804FB07B5042201910DEB0201D1
:10C9F000FFF7EAFF03B05DF804FB0222FFF78ABFEE
:10CA00000322FFF787BF07B5CDE900126946FFF79C
:10CA1000F4FF03B05DF804FB07B5CDE900126946E9
:10CA2000FFF7EEFF03B05DF804FB1F220421FFF7C0
:10CA30004CBF1F220521FFF748BF1F220721FFF728
:10CA400044BFFFF7FABF1FB50024CDE90144069C9F
:10CA50000094FFF7DFFC04B010BD08B1F6F79CBDF1
:10CA6000704710B5436904463BB90020E26853782B
:10CA700043F001035370404210BD98470028F4D0A2
:10CA80000028B8BF4042E368FF28A8BFFF20187005
:10CA9000ECE740B1C368587810F001001EBF187869
:10CAA000B0FA80F040097047EFF31183202383F33D
:10CAB0001288BFF36F8FFEE708B5FFF7F5FF10B5DB
:10CAC00042696AB1836842EA0301890708D10169B2
:10CAD000A2FB011424B95B182CBF0121002102D351
:10CAE0006FF0150005E0C1609B1A02698A4201D807
:10CAF000002010BDC2681A604269C36001319B1AF0
:10CB0000F3E72DE9F04105460F46EFF311882023A6
:10CB100083F31288BFF36F8FC668F6B90468A0422A
:10CB20001BD0D4B1D4E9003213605A60237CA660D4
:10CB300023F002032374C4E9006604F11800FCF733
:10CB4000FDF92046A667676100F096F9414605F1B8
:10CB50000800BDE8F04100F0F5B93E60AB69EF6058
:10CB6000013BAB6188F31188BFF36F8FBDE8F081A3
:10CB700010B52024EFF3118384F31288BFF36F8F75
:10CB8000FEF7AFFBF6E790F90E308B4201D0FBF7D2
:10CB90007DBF0020704703460020C3E90200C3E9BF
:10CBA00000337047D0E9003213605A60027C0023E2
:10CBB00022F00202C0E900330274836070472DE95D
:10CBC000F843904604469DF820200D46EFF3118768
:10CBD000202181F31288BFF36F8F02B14568A668E8
:10CBE00004F10809B14515D0A6B13046FFF7DAFFC8
:10CBF000002406F11800FCF7A1F93046B467C6F826
:10CC0000148000F039F94846394600F09BF9204677
:10CC1000BDE8F883A3B10820FCF74CFB002832D014
:10CC20000122C0F804800260016801F003015DB9CF
:10CC300022680A430260626820606AB960600BE0A3
:10CC4000C8F800304046EFE72A68032A10D8016090
:10CC5000616839B9C4E90000002087F31188BFF387
:10CC60006F8FD5E70A6802F0030202430A60E5E726
:10CC700022F003020A4302602A6802F0030240EA3B
:10CC800002032B60E8E76FF00B00E6E710B50446FF
:10CC900030B10268930703D0446809B100F00DFA7F
:10CCA000204610BD07B50123009300230A4619460C
:10CCB000FFF785FF03B05DF804FB3AB18A4205D364
:10CCC000C0E90212C0E90000002070476FF01500B3
:10CCD0007047026801238B4022EA0303036022FAB3
:10CCE00001F000F00100704720B1002211468C30A5
:10CCF00000F044B9704773B50446EFF31185202363
:10CD000083F31288BFF36F8F00230193D0E90423CC
:10CD1000B3F1004F08BF012A05D085F31188BFF396
:10CD20006F8F02B070BDA0F1100603210438FFF729
:10CD3000D0FF0028F1D0A369019301A93046FBF789
:10CD400051FBEAE738B504460D461022002101F0F8
:10CD5000C3F9656038BD13B501900846EFF311843F
:10CD6000202383F31288BFF36F8F01A9FBF73AFBEF
:10CD700084F31188BFF36F8F02B010BD10B5FFF7B9
:10CD8000EAFF041E08DDEFF31180202383F31288ED
:10CD9000BFF36F8FFBF7E6FE204610BD38B530229B
:10CDA00004460D46002101F097F94FF48073656049
:10CDB000E36038BDEFF30580003818BF01207047ED
:10CDC0006FF05700704738B58589EFF31181202245
:10CDD00082F31288BFF36F8F037C13F0080404D032
:10CDE00081F31188BFF36F8F38BD0122FBF728FD57
:10CDF000EB07F9D584F31188BFF36F8F042318462E
:10CE000002DFF1E7FBF7D4BDD0E9003213605A60CE
:10CE10000023C0E90033704708B5FFF7F5FF037C36
:10CE200023F0020303740023836008BD38B5044671
:10CE30000D46FBF751FC237C43F002032374D5B16C
:10CE4000A5602B689D4209D16B68C4E900531C6042
:10CE50006C6010E06A689A42F6D01B68002BF3D031
:10CE600093F90E1094F90E209142F3DD5A68C4E94B
:10CE7000003214605C6038BD10B5EFF311842023DC
:10CE800083F31288BFF36F8FFBF750FC84F3118894
:10CE9000BFF36F8F10BDFBF749BCFBF71DBC08B596
:10CEA000EFF31181202282F31288BFF36F8F836822
:10CEB0000BB1FFF7B1FF81F31188BFF36F8F08BD8E
:10CEC00008B5037C13F0280F01460CD183680BB121
:10CED000FFF7A2FF0B7C23F004030B740846BDE8A8
:10CEE0000840FBF723BC08BD10B5EFF311842023E5
:10CEF00083F31288BFF36F8FD0E90423B3F1004F9F
:10CF000008BF012A04D084F31188BFF36F8F10BDCE
:10CF10001838FFF7D5FFF6E708B50346EFF31181A0
:10CF2000202282F31288BFF36F8F0068834207D0FC
:10CF300008B1FFF771FF81F31188BFF36F8F08BD50
:10CF40000020F8E70846FBF731BC38B50C4605462B
:10CF5000FBF71CFEB4F1FF3F08BFB5F1FF3F1FBF59
:10CF600047F6FF7300224FF47A71E0FB01321ABFDB
:10CF7000D80B40EA42404FF0FF3038BD38B5EFF3F0
:10CF80001185202383F31288BFF36F8F0468A042BA
:10CF90001BD0E4B16261D4E90032A16713605A602A
:10CFA000227C002322F00202C4E900332274A36031
:10CFB00004F11800FBF7C2FF2046FFF76CFF0120C9
:10CFC00085F31188BFF36F8F38BD0020F8E7204646
:10CFD000F6E708B50246FBF703FF70B1D0E904316C
:10CFE0009B1A61EBE272B3F1004F72F1000104DAB7
:10CFF000002AACBF1846002008BD6FF00040FBE7D8
:10D0000008B5FCF74BF808BDFCF748B8B3F1FF3F93
:10D0100008BFB2F1FF3F70B506461D46144614D056
:10D020001A4316D0002B08DBFCF738F8041941EB43
:10D030000501C6E90041304670BD6FF001031C1BBD
:10D040004FF0FF3363EB0501F3E74FF0FF34214668
:10D05000EFE70024FBE7B3F1FF3F08BFB2F1FF3F6A
:10D06000F8B5074616461C4610D054EA020311D004
:10D07000FCF714F8B0420A46A14103460AD2F31A5B
:10D0800064EB0204C7E900343846F8BD4FF0FF33C3
:10D090001C46F7E70023FBE730B50023C0E9081280
:10D0A000002400F118020025C0E90622C0E900337F
:10D0B000C0E904450363436330BD10B5014670B158
:10D0C00051F8040DEFF31184202383F31288BFF38A
:10D0D0006F8FFDF710FB84F31188BFF36F8F10BDC6
:10D0E00010B400F10C04C0E9034410BCFDF789BB87
:10D0F00000220123C0E90023704710B5044648B15F
:10D10000006818B1E188890000F046FF0022012381
:10D11000C4E9002310BD42F21073994270B5044671
:10D120000D4602D96FF08C0070BDC3888B4201D3CD
:10D130000020F9E704212846FCF770FF0646002886
:10D14000F0D0216841B1E288920000F09EFFE188B2
:10D150002068890000F020FFE5802660E8E738B508
:10D1600004460D4619B9FFF7C8FF002038BDC28834
:10D170008A4207D100689200002100F0ADFF012330
:10D18000A380F2E7FFF7B9FF29462046BDE8384003
:10D19000FFF7C1BF42F21073994270B50A460546C7
:10D1A00002D96FF08C0070BDC3888B4207D8BDE8F0
:10D1B0007040FFF7B0BF296851F8231011B9013B47
:10D1C000002BF8D15C1C944238BF14460421204641
:10D1D000FCF724FF06460028E3D0296839B1A200F5
:10D1E00000F053FFE9882868890000F0D5FEEC8044
:10D1F0002E600020D7E7884270B505460E4609D05C
:10D20000C98849B9C2882AB1012383809200006885
:10D2100000F062FF002070BD4C1E74B9EA88B6F9B8
:10D220000430AB800134A2420ED221462846FFF7DB
:10D2300072FF88B16FF08C00EDE7336853F824304B
:10D24000002BEBD1013CE8E72868121B920000217B
:10D2500000EB840000F040FF31682868A20000F075
:10D2600014FFD7E770B50C4601210546FFF753FFC1
:10D27000064688B9EA8801469200286800F02CFF2B
:10D2800084EAE472A2EBE472E40FC4EBC4342B68CA
:10D29000640001341A60AC80304670BDC388B1EBC5
:10D2A000431F3FBF03684A0901F01F0153F82200E2
:10D2B0003ABFC84000F0010000207047C1880068F4
:10D2C00000F013BB08B5FFF7F9FF0730C00808BD31
:10D2D00070B50E4612F0030118BF012101EB920157
:10D2E00005461446FFF73BFF38B9E988286823460E
:10D2F0003246BDE8704000F01ABB6FF08C0070BD84
:10D3000013460A46C188006800F036BB38B50446AB
:10D310000D46FFF7D3FFE3882844B0EB431F06D840
:10D320002068E1882A4600F091FB002038BD10F00B
:10D330001F0118BF012101EB50112046FFF7EBFE42
:10D340000028EDD06FF08C00F0E708B50A46C188E0
:10D3500011B1006800F042FB002008BD10B5C38881
:10D3600023B9CA885AB9ABB1012017E0026802EBB1
:10D37000830252F8042C002AF3D1013BF0E70C6839
:10D3800004EB820454F8044C0CB9013AEAE79A42DF
:10D39000EAD30FD8013B5A1C01D1002010BD02680E
:10D3A00052F823400A6852F823209442DCD803F153
:10D3B000FF33F0D24FF0FF30F0E730B5C38823B928
:10D3C000CA885AB9002B3DD136E0026802EB8302CD
:10D3D00052F8042C002AF3D1013BF0E70C6804EB6F
:10D3E000820555F8045C4DBB013AEAE7B1F90450F7
:10D3F00003D2B1F90400404226E0B0F90420002A2B
:10D4000003DD002D0CDA01201EE0002D08DD3AB10D
:10D410004FF0FF3018E003F1FF330BD2504213E01E
:10D42000013B016851F8235054F823108D42F2D982
:10D43000104609E0591CF4D1002005E0002BD8D09B
:10D440009342D3D9B0F9040030BD1FB581EAE1732E
:10D45000A3EBE173C90FC1EBC13149000193013165
:10D460000123ADF80C10ADF80E3002A901AB029308
:10D47000FFF7A3FF05B05DF804FB90422DE9F041F2
:10D4800006460F46144602D0884206D1274601239D
:10D49000B380FC884CB9002005E0FFF7ACFE002803
:10D4A000F4D06FF08C00BDE8F0813B6803EB84039F
:10D4B0004FEA840853F8043C0BB9013CEAE72146E3
:10D4C0003046FFF728FE0028EBD135683A6823463E
:10D4D0002946284600F0F0FA05EB08030746002F1E
:10D4E000D9D0F288A24204F1010508D82946304675
:10D4F000FFF711FE0028D4D1336803EB84031A68C8
:10D50000D2192CBF01270027003F43F8042B18BF76
:10D5100001272C46E3E72DE9F041D48805460E4665
:10D5200090466CBBF1882846FFF7F5FD07460028BA
:10D5300042D1F288A2420BD9AE4209D028683168A4
:10D54000121B920001EB840100EB840000F09DFDB2
:10D55000EA88F088824207D92B68121A92000021CB
:10D5600003EB800000F0B8FDD8F80020316828688F
:10D570002346FCF715F9024698B90123AB800DE06C
:10D58000D8F8003003EB840353F8043C0BB9013C9A
:10D59000C7E7F188A142C6D26FF009073846BDE857
:10D5A000F0812968EB8801EB84011B1B084600F021
:10D5B0003FFB0028E1D0EFE76FF08C07EEE72DE9A5
:10D5C000F843B1F90440B2F804C01CFB04FC674600
:10D5D0007B4305460E4691461DD511463046FFF762
:10D5E000BDFEB0F1FF3F80460CD04A46314628468A
:10D5F000FFF791FF68B9B8F1000F08BF0124AC80B4
:10D60000002006E032462846FFF785FF08B964424D
:10D61000AC80BDE8F883FFF730FF0028EFD06FF053
:10D620008C00F6E70123FFF7CABF4FF0FF33FFF787
:10D63000C6BF2DE9F341CE8804460F46154636B1E4
:10D640003B6803EB860353F8043C3BB145B900212A
:10D65000204602B0BDE8F041FFF704BE013EEEE710
:10D66000711C2046FFF757FD28B16FF08C0840462B
:10D6700002B0BDE8F08139462046FFF7BCFD804688
:10D680000028F2D1013D00953A68E18820683346D0
:10D69000FCF7B6F8EBE770B504460D4610460021DE
:10D6A0001646FFF7D2FE002824DB2A4633462146E1
:10D6B0000020FBF73DFE054638B1284670BD3246D6
:10D6C00021462046FFF7AEFF90B900212046FFF724
:10D6D000BCFE0028F3DB31462046FFF76EFE002833
:10D6E000EBDB324621462046FFF79FFF0028F2D0B1
:10D6F0000546E2E76FF00905DFE72DE9F04F8BB053
:10D70000DDE9145706468B462846002191460793CB
:10D71000FFF79BFE002805DC6FF0860420460BB067
:10D72000BDE8F08F2B681B68D907F5D50021484666
:10D73000FFF78BFE0028EFDB4846FFF7BFFDB0F593
:10D74000005FE9D82846FFF7B9FDB0F5005FE3D8E0
:10D75000B9F8061031B9012130460BB0BDE8F04FE1
:10D76000FFF780BDE88800F037FA04210690FCF747
:10D7700055FC8046002800F0988000220123CDE966
:10D78000082317B13B68002B68D10DF1200A294608
:10D79000504600F007FA0446002866D11FB19AE807
:10D7A000030087E8030059463046FFF724FD0028B0
:10D7B00059D10123B38029463046FFF7FEFD0028EA
:10D7C00067DAE9883046FFF7A6FC044600284AD10C
:10D7D000286800F087F9089BCDF80880CDE90003A0
:10D7E0003168EB882A688246084600F041FAEB88E7
:10D7F0000593DDE9073E3168D9F80000B9F806C0A5
:10D800002A68B3F12A3FCDE9000CCDE902E8059B77
:10D81000084647D100F0FBF9CDE900A83168EB8854
:10D820002A68084600F030FABBF904A0BAF1FF3FBD
:10D830001BD1D9F800301B68DB0716D5F18830689A
:10D8400000F00AFA01225146FBF764FD3246B0802F
:10D8500029463046FFF7E6FE044606E0E9883846EA
:10D86000FFF759FC78B16FF08C04069B4046990095
:10D8700000F092FB1FB13B68002B7FF44FAF08A86C
:10D88000FFF73BFC4AE797E803000AAB03E9030014
:10D8900089E72A4631463046FFF7FDFE0446002858
:10D8A0008FD0E2E700F0A3F9B6E76FF08C0435E71C
:10D8B00013B5049CCDE900344FF02A33FFF71DFF68
:10D8C00002B010BD37B50223154601AA044600F088
:10D8D0009CFB40B9019A21682846FFF7F9FC2368B0
:10D8E000019A1344236003B030BD0139002901DAE5
:10D8F0000020704750F82130002BF6D0B3FA83F0A7
:10D900000131C0EB4110704739B101F1804101395B
:10D9100000EB81018142034600D270471B680A6810
:10D920001BBA12BA40F8042B41F80439F2E72DE98A
:10D93000F0411C4613F0030318BF012303EB9403CB
:10D940008B4206460D46904613D879B18F003A4671
:10D95000002100F0C1FB2CB1381B22464146304467
:10D9600000F093FB29463046FFF7CEFF0020BDE8CC
:10D97000F0816FF08900FAE7B3EB810F70B50446D0
:10D980004FEA8105104619D95A1B8618002100F06C
:10D99000A3FB30462B46C21800218B4210D1002039
:10D9A00070BD22F0030102F003066158F600F14059
:10D9B000C9B281B90132AA42F3D3ECE71A46FAE7B9
:10D9C00021F0030001F003052058ED00E84002F8C3
:10D9D000010D0131E1E76FF08900E1E753098B4266
:10D9E000F0B402F01F0401D805D13CB38A00F0BCAA
:10D9F000002100F071BB1F2A22D834B100EB810155
:10DA00000022C4F1200681420FD1F0BC704752F8C9
:10DA1000047B45F8047FB242F9D1CB1A00228B4235
:10DA2000EBD240F823200133F9E751F8045D25FAE1
:10DA300004F313430B6005FA06F2E4E71F2AE4D966
:10DA400000EB8302051F00EB8106E4E71F2AF0B517
:10DA50004FEA521402F01F0512D96FF0030606FBBD
:10DA600004060B469C4203F1FF3212D3631A8C4228
:10DA700088BF00230B4400EB8303002283420ED1B6
:10DA800035B100EB84000022C5F120078C4209D398
:10DA9000F0BD56F8223040F822301346E2E743F852
:10DAA000042DEBE7066806FA05F3134340F8043B40
:10DAB000013426FA07F2E9E7F0B50024844620464F
:10DAC0009C4200D1F0BD51F8245052F824702E1819
:10DAD0002CBF01250025BF194CF8247045F100002A
:10DAE0000134EDE70068831C5B0003F00803034486
:10DAF00003FB00F2C2F10202534303FB00F2C2F146
:10DB00000202534358430238584370472DE9F04FFF
:10DB100087B091460493109B0293DDE91183139D16
:10DB200005934FEAC80283468A46043200212846FC
:10DB300000F0D2FA08F102032E4600240393444574
:10DB400016D105EB84052346029A55F82470294620
:10DB50005846FBF725FE7840FBF7E4FDA6000023BE
:10DB60002A465946109607B0BDE8F04FFCF778BA40
:10DB70005AF82430D9F8002037680399009302FB43
:10DB80000377059A049B574330464A46FBF738FE15
:10DB90003046DDE9022100974346FBF731FE0436AB
:10DBA0000134CCE738B50D4601210446FFF75AFB96
:10DBB00088B9E98820468901FFF7A8FB58B92A46A9
:10DBC00021462046FFF767FD28B9E9882046BDE8D1
:10DBD0003840FFF7DFBA38BD4901502934BF012270
:10DBE000032201239340033358430130704710B59B
:10DBF00086B00B9C04940A9C039400240294099C14
:10DC00000194089C0094FBF7B7FE06B010BD10B558
:10DC100086B00B9C04940A9C03944FF02A3402941F
:10DC2000099C0194089C0094FBF7A6FE06B010BD69
:10DC300070B50646002410469C4200D170BD51F8D4
:10DC40002420151A34BF01220022101E46F8245049
:10DC500018BF01200134EFE7034600EB81010020EB
:10DC60008B4201D1FBF75EBD53F8042B1043F7E75D
:10DC70001FB5089C0394069C0092CDE90134079AD5
:10DC8000FFF744FF04B010BD30B587B01C460B9DB4
:10DC900003950A9D00920123CDE9014505AA05934C
:10DCA000FFF734FF07B030BDF8B50546044655F818
:10DCB000047B28460E46FFF705FB874216D12368F2
:10DCC000B3F5806F12D800212846FFF7BEFB00286D
:10DCD0000CDD00212846FFF7E1FA38B14EB90021EA
:10DCE00004F10C00FFF7B1FB00281FDC6FF0860089
:10DCF0001EE004F11C0500212846FFF7A6FB0028C2
:10DD0000F4DD00212846FFF7C9FA0028EED004F11F
:10DD1000240500212846FFF798FB0028E6DD0021B6
:10DD20002846FFF7BBFA0028D9D1DFE70EB900205B
:10DD3000F8BD002104F12C00FFF787FB0028D5DD9A
:10DD4000002104F13400FFF780FB0028CEDD002124
:10DD500004F13C00FFF779FB0028E8DCC6E77422F9
:10DD6000002100F0B9B9012938B50546144602D0A2
:10DD70006FF0950038BD22B90123C5E91B3400209E
:10DD8000F8E71046FBF7B6FF0028F5D1F0E700688A
:10DD90007047F0B50C4685B0002105461646FFF7E2
:10DDA00083FF58BB02A8FFF7A3F921462A6802A8FF
:10DDB000FFF78EFA0446C0B92C1D214602A8FFF7D2
:10DDC000FCFA002817DA2A4602A9443552F80C7BDF
:10DDD000009523460846FFF76BFD044628B93A46EE
:10DDE000314602A8FFF78CFA044602A8FFF785F92E
:10DDF000204605B0F0BD6FF08604F6E76FF08604AC
:10DE0000F6E710B5044698B35C30FFF776F904F1F5
:10DE10006400FFF772F904F14400FFF76EF904F1B2
:10DE20001400FFF76AF904F12400FFF766F904F122
:10DE30001C00FFF762F904F10C00FFF75EF9201DEA
:10DE4000FFF75BF904F15400FFF757F904F14C00B8
:10DE5000FFF753F904F13C00FFF74FF904F13400E8
:10DE6000FFF74BF904F12C00BDE81040FFF745B96E
:10DE700010BD6822002100F02FB910B16821FCF715
:10DE8000E3B870472DE9F04105460E46144612B33B
:10DE9000036C03F03F079B18036422BF436C0133FC
:10DEA00043647FB1C7F1400842450FD3424638442E
:10DEB00000F0EBF829462846FBF754FE2744464479
:10DEC000A7F140043F2C09D82CB100272246314647
:10DED000E81900F0DAF80020BDE8F081374606EBDB
:10DEE0000408394628464037FBF73CFEA8EB0703F9
:10DEF0003F2BF6D8A4F1400323F03F0340331E44E8
:10DF0000E41ADFE738B5036C03F03F035A1C0D46F3
:10DF1000382A4FF08001C154044610442FD8C2F172
:10DF20003802002100F0D8F8D4E910315A0F42EA43
:10DF3000C102DB0012BA1BBAA263E363214620468A
:10DF4000FBF710FEA36C1BBA2B60E36C1BBA6B6073
:10DF5000236D1BBAAB60636D1BBAEB60A36D1BBA7C
:10DF60002B61E36D1BBA6B61236E1BBAAB61636EF1
:10DF70001BBA2046EB61FFF780FF002038BDC2F1DD
:10DF80004002002100F0A8F821462046FBF7EAFDF8
:10DF9000382200212046C5E710B5044608B1FCF739
:10DFA00053F82046BDE81040FCF73EB870B5046851
:10DFB0000D1B002D02DC6FF05F0070BD94F9006056
:10DFC0002378002E0ADB631C036023781360036848
:10DFD000C91A13688B42EED80020EEE703F07F03E6
:10DFE0005C1E032C0ED89D42E5DD002414600468FD
:10DFF000013B013404605E1C1568E8D0247844EAD3
:10E000000524F3E76FF06300D7E770B404680E1BD4
:10E01000002E07DD26789E4208D10134046070BCD2
:10E02000FFF7C4BF6FF05F0070BC70476FF0610016
:10E03000FAE710B5D0F83032044623B14FF404713A
:10E040002030FCF701F80020C4F8300210BD38B5CC
:10E050000446FFF7EEFF237E012B10D0023B012B7D
:10E0600010D8E369012B14BF6FF0960500254FF41B
:10E070000D720021204600F02FF8284638BDE369D4
:10E08000002BF0E76FF09605F1E70A44914200F1AA
:10E09000FF3300D1704710B511F8014B03F8014F61
:10E0A0009142F9D110BD884210B501EB020402D9AA
:10E0B0008442234607D8431EA14207D011F8012B02
:10E0C00003F8012FF8E70244824200D110BD13F893
:10E0D000011D02F8011DF7E702440346934200D1F7
:10E0E000704703F8011BF9E7044608B5FCF7E4F9AB
:10E0F0002046F5F71FFA10B501390244904201D1CC
:10E10000002005E0037811F8014FA34201D0181B4D
:10E1100010BD0130F2E7F0B5C2F137050446EDB2AB
:10E1200002F01F020846B4FBF2F602FB1641CBB226
:10E13000092988BF5B19274688BFDBB23033BA4252
:10E1400000F8013B3446EED9F0BDD1E904329342E8
:10E150001EBF5A1C0A611870704700008820FF7F9C
:10E1600001000000E13500000000000089350000DA
:10E17000000000000000000004E20000657F0000D5
:10E1800000000000C5920000000000000000000038
:10E190003CE200000000000020E20000000000005F
:10E1A00074E200000000000090E2000000000000A7
:10E1B00058E200004567000000000000051E000056
:10E1C000000000002DC3000000000000E9920000E4
:10E1D0000000000000000000ACE2000000000000B1
:10E1E000C8E20000753600000000000000000000DA
:10E1F00000E3000000000000E4E20000A1060000CF
:10E200000000000078EB000094E6000024E5000028
:10E2100098020020982000200D540000000000000B
:10E22000BDEB0000B4E60000C8E400009E02002040
:10E2300068210020615E000000000000CBEB0000C0
:10E24000C8E60000C8E40000A002002074210020FD
:10E25000615E0000000000004AEA0000EC030020BC
:10E2600040E500009402002000000020C91B0000CF
:10E270000000000093EB000000000000A8E4000094
:10E280009A0200200C210020D95900000000000053
:10E29000EDEB000008E7000084E50000A602002086
:10E2A0004C02002013BA0000000000006BEB0000DD
:10E2B000000000009CE40000960200200000000026
:10E2C0007551000000000000A3EB000000000000FA
:10E2D000B0E400009C02002000000000D15A0000C1
:10E2E00000000000D9EB000000000000ECE400009A
:10E2F000A202002080210020F16100000000000047
:10E30000E7EB0000DCE6000008E50000A4020020C6
:10E3100050050020F962000000000000C5C20000A6
:10E32000A7BB000000000000C7B2000090E20000A0
:10E330006DB9000000000000C7B20000000000003E
:10E34000C7B2000000000000C7B20000AC0100200E
:10E350004FB70000997A0000A7BB00000000000042
:10E36000C7B2000000000000C7B2000000000000BB
:10E37000C7B2000000000000C7B20000E4E20000E5
:10E38000616100000C210020455A000000000000DF
:10E39000C7B2000000000000C7B20000000000008B
:10E3A000C7B2000000000000D567000000000000B8
:10E3B000C7B2000000000000C7B20000000000006B
:10E3C000C7B2000000000000C7B20000000000005B
:10E3D000C7B2000000000000C7B20000000000004B
:10E3E000C7B2000000000000C7B20000000000003B
:10E3F000C7B2000000000000C7B20000000000002B
:10E40000C7B2000000000000C7B20000000000001A
:10E41000C7B2000000000000C7B20000000000000A
:10E42000C7B2000000000000C7B2000000000000FA
:10E43000C7B2000000000000C7B2000000000000EA
:10E44000C7B2000000000000C7B2000000000000DA
:10E45000C7B200005D450000A7BB0000000000003F
:10E46000C7B2000000000000C7B2000000000000BA
:10E47000C7B2000000000000C7B2000000000000AA
:10E48000C7B2000000000000C7B20000000000009A
:10E49000C7B2000000000000C7B20000394E000003
:10E4A000B95100005802000085590000D5580000FD
:10E4B0007BB60000055C00007D5B0000C95A0000CF
:10E4C00047B60000B95A0000915C0000A3B60000F6
:10E4D000B1B60000C9B60000D5B60000E1B6000034
:10E4E0009D5E0000FBB60000000000000000000080
:10E4F00000000000000000007961000035610000AC
:10E50000000000000000000000000000000000000B
:10E5100000000000B7B700003162000000000000FA
:10E520000000000069540000E5B4000049B5000097
:10E530000000000081B400000000000000000000A6
:10E54000D5AE0000111C000000000000811A000080
:10E550008DAE0000611A00002BAE000035AE000049
:10E56000411A000055AE0000000000005FAE000040
:10E5700000000000000000006DAE0000E7AE0000EB
:10E5800085AE000005B8000019640000F7B7000070
:10E59000E3BA00002BB8000053B8000089B80000AF
:10E5A0009DB80000CBB80000DFB800009DB80000A7
:10E5B000BBB80000F3B8000001B900000FB90000BB
:10E5C0000000000041B900007FE9000003000000E6
:08E5D0008FEA000003000000C7
:10E5E00000C2010000000800000000000000000060
:10E5F0000338FDD870470000D1230000D5B10000DA
:10E60000010000009BEC00000CE600000E01000081
:10E6100004000000000000000000000000400100B5
:10E62000C8E20000010000000040010000400700B7
:10E63000C8E200000200000000800800004007005F
:10E64000C8E200000300000000C00F00004000000E
:10E65000C8E20000000000200000000000000B06DF
:10E660000200000068E600000000000043EB00002C
:10E6700026000202000000204BEB000022000B11DC
:10E680009C0100200D380000C95300009953000080
:10E69000000000004D5500009954000087EB000079
:10E6A0007DB500006FB500008DEB00000400000098
:10E6B00000FF0000FFFF000000030050AC0100203D
:10E6C0000000000001000000FFFFFFFF00000050FD
:10E6D000AC0100200000000000000000ACE20000DF
:10E6E0000200000000000000000000000000000028
:10E6F000400D0300A08601000000000000000000A3
:10E700006400000000000000002000400100000044
:10E710000000000028E700000000D6010000000013
:10E720009B6700209A6700200020004034E700002B
:10E73000010000003CE700000200000011000000A2
:10E740000F060001080000000300000064E1000063
:10E750006CE10000B4E10000BCE10000FCE100005D
:10E7600004E200008BEC000000010000000000004B
:10E77000982F8A4291443771CFFBC0B5A5DBB5E92C
:10E780005BC25639F111F159A4823F92D55E1CABA0
:10E7900098AA07D8015B8312BE853124C37D0C552E
:10E7A000745DBE72FEB1DE80A706DC9B74F19BC176
:10E7B000C1699BE48647BEEFC69DC10FCCA10C2466
:10E7C0006F2CE92DAA84744ADCA9B05CDA88F9764A
:10E7D00052513E986DC631A8C82703B0C77F59BFB4
:10E7E000F30BE0C64791A7D55163CA0667292914E0
:10E7F000850AB72738211B2EFC6D2C4D130D38537D
:10E8000054730A65BB0A6A762EC9C281852C72923E
:10E81000A1E8BFA24B661AA8708B4BC2A3516CC76C
:10E8200019E892D1240699D685350EF470A06A10A5
:10E8300016C1A419086C371E4C774827B5BCB034F4
:10E84000B30C1C394AAAD84E4FCA9C5BF36F2E6892
:10E85000EE828F746F63A5781478C8840802C78C21
:10E86000FAFFBE90EB6C50A4F7A3F9BEF27871C624
:10E87000D9E0000001000200100011001200200089
:10E880002100220023002400300031003200330038
:10E89000FFFF25633A205374617274696E672062CA
:10E8A0006F6F746C6F616465720A0025633A20456E
:10E8B0006E746572207468652073657269616C207E
:10E8C0007265636F76657279206D6F64650A0025E5
:10E8D000633A20556E61626C6520746F2066696EC4
:10E8E0006420626F6F7461626C6520696D61676539
:10E8F0000A0025633A20426F6F746C6F6164657221
:10E9000020636861696E6C6F616420616464726524
:10E910007373206F66667365743A20307825780AC1
:10E920000025633A20496D616765207665727369D9
:10E930006F6E3A207625642E25642E25640A002504
:10E94000633A204A756D70696E6720746F20746831
:10E950006520666972737420696D61676520736CE8
:10E960006F740A0025633A204E65766572207368DD
:10E970006F756C642067657420686572650A006D48
:10E980006375626F6F740025633A204469646E2773
:10E99000742066696E64204C454420646576696322
:10E9A000652072656665727265642062792074689C
:10E9B00065204C4544305F4E4F44450A0A002563AC
:10E9C0003A20696E76616C696420666C61736820B8
:10E9D00049442025640A002A2A2A205573696E6753
:10E9E000205A6570687972204F53206275696C6493
:10E9F0002076342E342E302D333433332D6732329B
:10EA000063386264393733623436202A2A2A0A008E
:10EA10004661696C656420746F207265626F6F7403
:10EA20003A207370696E6E696E6720656E646C65FE
:10EA300073736C792E2E2E0A003031323334353612
:10EA4000373839414243444546006364635F61633C
:10EA50006D5F7561727400757362776F726B7100B0
:10EA600025633A204E6F7420656E6F756768206D60
:10EA7000656D6F727920746F2073746F7265206991
:10EA80006E636F6D696E672064617461210A007343
:10EA9000657269616C5F6164617074657200726354
:10EAA00000696D6167650064617461006C656E008A
:10EAB0006F66660025633A204572726F7220256486
:10EAC000207768696C652065726173696E67207272
:10EAD000616E67650A0025633A204661696C65646A
:10EAE00020746F206F70656E20666C6173682061A2
:10EAF000726561733A2025640A0025633A204661F5
:10EB0000696C656420746F2072656164207365634D
:10EB1000746F72733A2025640A00696D61676573CA
:10EB200000736C6F74006861736800766572736956
:10EB30006F6E002568752E2568752E256875002E68
:10EB4000257500464C4153485F30005352414D5F9C
:10EB50003000657869740061626F727428290A0058
:10EB6000757362645F776F726B71006164634034C8
:10EB70003030303730303000636C6F636B4034308E
:10EB8000303030303030006866636C6B006C666328
:10EB90006C6B0072616E646F6D4034303030643085
:10EBA000303000666C6173682D636F6E74726F6CC9
:10EBB0006C657240343030316530303000677069D8
:10EBC0006F403530303030333030006770696F401F
:10EBD00035303030303030300074656D7040343056
:10EBE0003030633030300076626174740075617269
:10EBF000744034303030323030300025633A2046B3
:10EC000061696C65642072656164696E6720696D15
:10EC1000616765206865616465720A0025633A2052
:10EC200042616420696D616765206D616769632079
:10EC30003078256C780A0025633A20496D61676554
:10EC4000206E6F7420626F6F7461626C650A0025BC
:10EC5000633A20496D6167652073697A652062694E
:10EC600067676572207468616E2064657369676E9A
:10EC70006174656420617265613A20256C75203E7F
:10EC800020256C750A006D61696E00737973776F6A
:10EC9000726B7100286E756C6C29003082010A025B
:10ECA00082010100CFF0A97B52474EBADAEAABF0FD
:10ECB0002C0B3EA6B815C07A04D3390D6212379ECC
:10ECC0007E460E1289CD5D05789A8314CFCC79A249
:10ECD000F810562BD1EC240D2C601BAF0EFDF28EDC
:10ECE00077547329DAAA984F3DE3BBB3BC510BB6F6
:10ECF000F385460216EA0F17D0083B7844D83C9BB0
:10ED00009ADEC9B0E651F9E4DF38D11090623C9048
:10ED10005A49CC95801178AA546AB71C5D245CFBD3
:10ED20006E5E037A30A6D6672DD8BFD9CA17F348CE
:10ED30007C8AC5AC482768ED40EA5D79EFCB3AD3D1
:10ED40004823E21F14A2746FD653606E71122CF622
:10ED500081323452673C7C41E64B3951563EC37A8E
:10ED6000F1407289892AF8F13AE17D29F2BF7E2DBE
:10ED700080C96F0592F94B1D7805EF055575346311
:10ED800036540977FDB812F7F73068F627290C7961
:10ED9000693B67F3A5BF334AA7A4E394AEAFBD7C3C
:10EDA0006E22CAD902030100017F7F7F7F7F7F7FB0
:10EDB0007F7F7F7F7F7F7F7F7F7F7F7F7F7F7F7F63
:10EDC0007F7F7F7F7F7F7F7F7F7F7F7F7F7F7F7F53
:10EDD0007F7F7F7F3E7F7F7F3F3435363738393ABC
:10EDE0003B3C3D7F7F7F407F7F7F00010203040526
:10EDF000060708090A0B0C0D0E0F1011121314153B
:10EE0000161718197F7F7F7F7F7F1A1B1C1D1E1FFF
:10EE1000202122232425262728292A2B2C2D2E2F7A
:10EE2000303132337F7F7F7F7F41424344454647C5
:10EE300048494A4B4C4D4E4F5051525354555657DA
:10EE400058595A6162636465666768696A6B6C6D7C
:10EE50006E6F707172737475767778797A3031323B
:10EE6000333435363738392B2F00000000000000CE
:10EE7000000100020006010501040107020301056B
:10EE80000202010302050401010102010301040160
:10EE9000060108010C011001180120014001800049
:10EEA00001020304050607002030303030303030D6
:10EEB000303030303030300001090000000D0102E8
:10EEC00003040506070801020203030303092040A7
:10EED0000000000000000000000000000000000032
:10EEE0000000000000000000000000000000000022
:10EEF0000000000000000000000000000000000012
:10EF00000000000000000000000000000000000001
:10EF100000000000000000000000000000000000F1
:10EF200000000000000000000000000000000000E1
:10EF300000000000000000000000000000000000D1
:10EF400000000000000000000000000000000000C1
:10EF50000000000000000000000000006C01002024
:10EF60005801002000C2010000000800000000005D
:10EF70000000000000000000000000000000000091
:10EF800000000000B4000020B400002000000000D9
:10EF900001000000C4000020C400002000000000A8
:10EFA0000100000000000000000000000000000060
:10EFB0000000000000000000000000000000000051
:10EFC0000000000000000000000000000000000041
:10EFD0000000000000000000000000000000000031
:10EFE0000000000000000000000000000000000021
:10EFF0000000000000000000000000000000000011
:10F000000000000000000000000000000000000000
:10F0100000000000000000000000000000000000F0
:10F0200085A8000014E6000080A700200000000072
:10F0300000000000000000000004000080AB002081
:10F0400000000000000000000000000000040000BC
:10F05000751B000080000000551800000000000033
:10F060005518000080000000FFFFFFFF00000000B7
:10F0700041B30000000000000000000000600040FC
:10F080000000000000000000000000000000000080
:10F090000000000000000000000000000000000070
:10F0A0000000000000000000000000000000000060
:10F0B0000000000000000000000000000000000050
:10F0C0000000000000000000000000000000000040
:10F0D0000000000000000000000000000000000030
:10F0E0000000000000000000000000000000000020
:10F0F0000000000000000000000000000000000010
:10F1000000000000000000000000000000000000FF
:10F110001557000000000000000000005C02002005
:10F1200000000000000000000000000000000000DF
:10F13000000000009C67002020000000000000008C
:10F140000090D003FF00000090020000FFFFFFFFCF
:10F150008002002080020020E9E000004BB30000A4
:10F1600071350000000000000000000000000000F9
:10F17000000000000000000000000000000000008F
:10F18000CD90000000000000000000000000000022
:10F19000C0020020C002002081B500000000000075
:10F1A000000000000000000000000000000000005F
:10F1B000E0020020E002002000A500200000000086
:10F1C000200000001400000000000000FC020020ED
:10F1D000FC02002000000000000000000E00000003
:10F1E00010030020100300200100000001000000B7
:10F1F0000000000000000000280300202803002079
:10F2000012010002EF02014015190053040401022B
:10F21000030109020000000100E032080B000202B5
:10F220000200000904000001020200000524001091
:10F23000010524010201042402020524060001073D
:10F2400005800310000A09040100020A00000007FB
:10F250000580024000000705000240000004030989
:10F26000040E035A4550485952000000000000287F
:10F270000353756C614A616C6D617269204D435531
:10F28000426F6F74000000000000000000000000EA
:10F2900000000000000000220330313233343536E4
:10F2A0003738394142434445460000000000000021
:0BF2B000000000000000000000000053
:10F2BC0000000000530300200DAE0000811D000073
:10F2CC00111B000000000000000000000300000003
:08F2DC008001002015E015E09F
:020000040001F9
:104000003DB8F3960000000000020000F4EF01004C
:1040100000000000000000000000000000000000A0
:104020000000000000000000000000000000000090
:104030000000000000000000000000000000000080
:104040000000000000000000000000000000000070
:104050000000000000000000000000000000000060
:104060000000000000000000000000000000000050
:104070000000000000000000000000000000000040
:104080000000000000000000000000000000000030
:104090000000000000000000000000000000000020
:1040A0000000000000000000000000000000000010
:1040B0000000000000000000000000000000000000
:1040C00000000000000000000000000000000000F0
:1040D00000000000000000000000000000000000E0
:1040E00000000000000000000000000000000000D0
:1040F00000000000000000000000000000000000C0
:1041000000000000000000000000000000000000AF
:10411000000000000000000000000000000000009F
:10412000000000000000000000000000000000008F
:10413000000000000000000000000000000000007F
:10414000000000000000000000000000000000006F
:10415000000000000000000000000000000000005F
:10416000000000000000000000000000000000004F
:10417000000000000000000000000000000000003F
:10418000000000000000000000000000000000002F
:10419000000000000000000000000000000000001F
:1041A000000000000000000000000000000000000F
:1041B00000000000000000000000000000000000FF
:1041C00000000000000000000000000000000000EF
:1041D00000000000000000000000000000000000DF
:1041E00000000000000000000000000000000000CF
:1041F00000000000000000000000000000000000BF
:10420000003E002041AC0100FD8B02002DAC0100FE
:104210002DAC01002DAC01002DAC01000000000010
:104220000000000000000000000000002DAD0100B3
:104230002DAC010000000000F1AE01002DAC01002A
:1042400061AF010061AF010061AF010061AF01002A
:1042500061AF010061AF010061AF010061AF01001A
:1042600061AF010061AF010061AF010061AF01000A
:1042700061AF010061AF010061AF010061AF0100FA
:1042800061AF010061AF010061AF010061AF0100EA
:1042900061AF010061AF010061AF010061AF0100DA
:1042A00061AF010061AF010061AF010061AF0100CA
:1042B00061AF010061AF010061AF010061AF0100BA
:1042C00061AF010061AF010061AF010061AF0100AA
:1042D00061AF010061AF010061AF010061AF01009A
:1042E00061AF010061AF010061AF010061AF01008A
:1042F00061AF010061AF010061AF010061AF01007A
:1043000080F0004002E000BF81F0004142001FBF8A
:104310005FEA410392EA030F7FEA226C7FEA236C93
:104320006AD04FEA1262D2EB1363C1BFD218414088
:1043300048404140B8BF5B42192B88BF704710F01E
:10434000004F40F4000020F07F4018BF404211F0C1
:10435000004F41F4000121F07F4118BF494292EA29
:10436000030F3FD0A2F1010241FA03FC10EB0C0055
:10437000C3F1200301FA03F100F0004302D54942E2
:1043800060EB4000B0F5000F13D3B0F1807F06D38F
:1043900040084FEA310102F10102FE2A51D2B1F187
:1043A000004F40EBC25008BF20F0010040EA03007C
:1043B0007047490040EB0000013A28BFB0F5000FFC
:1043C000EDD2B0FA80FCACF1080CB2EB0C0200FAB2
:1043D0000CF0AABF00EBC25052421843BCBFD04001
:1043E0001843704792F0000F81F4000106BF80F47B
:1043F00000000132013BB5E74FEA41037FEA226C3E
:1044000018BF7FEA236C21D092EA030F04D092F008
:10441000000F08BF0846704790EA010F1CBF00203C
:10442000704712F07F4F04D1400028BF40F0004099
:10443000704712F100723CBF00F50000704700F0B9
:10444000004343F0FE4040F4000070477FEA2262E0
:1044500016BF08467FEA23630146420206BF5FEAB1
:10446000412390EA010F40F4800070474FF00003B1
:1044700004E000BF10F0004348BF40425FEA000C78
:1044800008BF704743F0964301464FF000001CE020
:1044900050EA010208BF70474FF000030AE000BF76
:1044A00050EA010208BF704711F0004302D54042B4
:1044B00061EB41015FEA010C02BF84460146002026
:1044C00043F0B64308BFA3F18053A3F50003BCFA41
:1044D0008CF2083AA3EBC25310DB01FA02FC6344EE
:1044E00000FA02FCC2F12002BCF1004F20FA02F2F5
:1044F00043EB020008BF20F00100704702F12002E8
:1045000001FA02FCC2F1200250EA4C0021FA02F248
:1045100043EB020008BF20EADC7070474FF0FF0C4D
:104520001CEAD0521EBF1CEAD15392EA0C0F93EA48
:104530000C0F6FD01A4480EA010C400218BF5FEAEA
:1045400041211ED04FF0006343EA501043EA51115D
:10455000A0FB01310CF00040B1F5000F3EBF490057
:1045600041EAD3715B0040EA010062F17F02FD2A5B
:104570001DD8B3F1004F40EBC25008BF20F001003E
:10458000704790F0000F0CF0004C08BF49024CEA55
:10459000502040EA51207F3AC2BFD2F1FF0340EAE7
:1045A000C250704740F400004FF00003013A5DDC58
:1045B00012F1190FDCBF00F000407047C2F1000299
:1045C000410021FA02F1C2F1200200FA02FC5FEA86
:1045D000310040F1000053EA4C0308BF20EADC70D0
:1045E000704792F0000F00F0004C02BF400010F442
:1045F000000F013AF9D040EA0C0093F0000F01F0EF
:10460000004C02BF490011F4000F013BF9D041EA10
:104610000C018FE70CEAD15392EA0C0F18BF93EA12
:104620000C0F0AD030F0004C18BF31F0004CD8D13C
:1046300080EA010000F00040704790F0000F17BFC3
:1046400090F0004F084691F0000F91F0004F14D009
:1046500092EA0C0F01D142020FD193EA0C0F03D161
:104660004B0218BF084608D180EA010000F0004064
:1046700040F0FE4040F40000704740F0FE4040F43F
:10468000400070474FF0FF0C1CEAD0521EBF1CEADE
:10469000D15392EA0C0F93EA0C0F69D0A2EB0302FC
:1046A00080EA010C49024FEA402037D04FF0805396
:1046B00043EA111143EA10130CF000408B4238BF5B
:1046C0005B0042F17D024FF4000C8B4224BF5B1A69
:1046D00040EA0C00B3EB510F24BFA3EB510340EAB7
:1046E0005C00B3EB910F24BFA3EB910340EA9C0065
:1046F000B3EBD10F24BFA3EBD10340EADC001B01D5
:1047000018BF5FEA1C1CE0D1FD2A3FF650AF8B4278
:1047100040EBC25008BF20F0010070470CF0004C85
:104720004CEA50207F32C2BFD2F1FF0340EAC250B0
:10473000704740F400004FF00003013A37E792F071
:10474000000F00F0004C02BF400010F4000F013ACF
:10475000F9D040EA0C0093F0000F01F0004C02BFCA
:10476000490011F4000F013BF9D041EA0C0195E733
:104770000CEAD15392EA0C0F08D142027FF47DAFCC
:1047800093EA0C0F7FF470AF084676E793EA0C0FBC
:1047900004D14B023FF44CAF08466EE730F0004CBA
:1047A00018BF31F0004CCAD130F000427FF45CAF4A
:1047B00031F000437FF43CAF5FE700BF4FF0FF3CB8
:1047C00006E000BF4FF0010C02E000BF4FF0010C0B
:1047D0004DF804CD4FEA40024FEA41037FEA226CD4
:1047E00018BF7FEA236C11D001B052EA530C18BFF6
:1047F00090EA010F58BFB2EB030088BFC81738BF5B
:104800006FEAE17018BF40F0010070477FEA226C48
:1048100002D15FEA402C05D17FEA236CE4D15FEA44
:10482000412CE1D05DF8040B704700BF8446084678
:104830006146FFE70FB5FFF7C9FF002848BF10F139
:10484000000F0FBD4DF808EDFFF7F4FF0CBF01207E
:1048500000205DF808FB00BF4DF808EDFFF7EAFF08
:1048600034BF012000205DF808FB00BF4DF808EDC3
:10487000FFF7E0FF94BF012000205DF808FB00BFB8
:104880004DF808EDFFF7D2FF94BF012000205DF83E
:1048900008FB00BF4DF808EDFFF7C8FF34BF01204B
:1048A00000205DF808FB00BF4FEA4002B2F1FE4F66
:1048B0000FD34FF09E03B3EB12620DD94FEA0023E2
:1048C00043F0004310F0004F23FA02F018BF4042BB
:1048D00070474FF00000704712F1610F01D14202A2
:1048E00005D110F0004008BF6FF0004070474FF056
:1048F0000000704742000ED2B2F1FE4F0BD34FF0D2
:104900009E03B3EB126209D44FEA002343F0004345
:1049100023FA02F070474FF00000704712F1610F68
:1049200001D1420202D14FF0FF3070474FF000003A
:10493000704700BF7BB972B90029BEBF00204FF09D
:10494000004106E008BF00281CBF6FF000414FF097
:10495000FF3000F057B8ADF1080C6DE904CE002926
:1049600009DB002B1ADB00F069F8DDF804E0DDE973
:10497000022304B07047404261EB4101002B1BDB76
:1049800000F05CF8DDF804E0DDE9022304B0404209
:1049900061EB4101524263EB43037047524263EBC8
:1049A000430300F04BF8DDF804E0DDE9022304B036
:1049B000404261EB41017047524263EB430300F018
:1049C0003DF8DDF804E0DDE9022304B0524263EB78
:1049D0004303704753B94AB9002908BF00281CBFD8
:1049E0004FF0FF314FF0FF3000F00CB8ADF1080C84
:1049F0006DE904CE00F022F8DDF804E0DDE90223E1
:104A000004B07047704700BF10F8012B11F8013B4C
:104A1000012A28BF9A42F7D0D01A7047034611F8EE
:104A2000012B03F8012B002AF9D17047034613F834
:104A3000012B002AFBD1181A013870472DE9F047E5
:104A40008C468E46089E154604461946002B40F0BB
:104A5000D080724547D9B2FA82F74FB1C7F120032F
:104A60000EFA07FC20FA03F3BD4043EA0C0CBC40ED
:104A70004FEA154EA8B2BCFBFEF8230C0EFB18CC77
:104A800008FB00F943EA0C43994528D9EB1808F1D3
:104A9000FF3204D2994502D9A8F102022B44A3EBBC
:104AA0000903A4B2B3FBFEFC0EFB1C330CFB00F0AD
:104AB00044EA0344A04214D92C190CF1FF3304D268
:104AC000A04202D9ACF102032C44241A43EA02406A
:104AD0001EB1FC40002334607360BDE8F08742469D
:104AE000DDE76346F1E7002A79D0B2FA82F3002BC2
:104AF0003FD01946C1F1200302FA01F52EFA03F264
:104B00000EFA01FE20FA03F343EA0E034FEA154EB4
:104B100000FA01F4B2FBFEFCAFB20EFB1C201A0C33
:104B20000CFB07F842EA004290455AD9AA180CF14A
:104B3000FF3004D2904502D9ACF102002A44A2EB26
:104B400008029BB2B2FBFEFC0EFB1C220CFB07F71B
:104B500043EA02439F4246D9EB180CF1FF3204D2DC
:104B60009F4202D9ACF102022B44DB1B42EA004215
:104B700002E0AEEB020301224FEA154EAFB2B3FBE7
:104B8000FEFC200C0EFB1C330CFB07F840EA034331
:104B900098452AD9EB180CF1FF3004D2984502D978
:104BA000ACF102002B44A3EB0803A4B2B3FBFEFC60
:104BB0000EFB1C330CFB07F744EA0344A74216D94B
:104BC0002C190CF1FF3304D2A74202D9ACF1020335
:104BD0002C44E41B43EA00400F46114678E71F21AE
:104BE00088E76046ABE76246BFE76046DBE76346BF
:104BF000EFE7734506D916B9002108466DE7C6E907
:104C0000000EF9E7B3FA83F787B9734501D38242FF
:104C100007D8841A6EEB030301209C461EB90021BD
:104C20005BE73846FAE7C6E9004CF8E7C7F1200C25
:104C3000BB4022FA0CF51D4320FA0CF12EFA0CF3BE
:104C40000EFA07FE41EA0E014FEA154900FA07F491
:104C5000B3FBF9F81FFA85FE09FB18300B0C08FBB3
:104C60000EFA43EA00439A4502FA07F240D9EB18DC
:104C700008F1FF3004D29A4502D9A8F102002B4472
:104C8000A3EB0A0389B2B3FBF9F809FB183308FB5D
:104C90000EFE41EA03418E452CD9691808F1FF3315
:104CA00004D28E4502D9A8F10203294443EA004008
:104CB000A0FB0298A1EB0E014145CE46434602D32C
:104CC00006D14C4504D2B9EB020E68EB050301385E
:104CD000002EA4D0B4EB0E0261EB030101FA0CFC30
:104CE00022FA07F34CEA0303F940C6E9003196E7DC
:104CF0004046C5E74346D9E72DE9F04FFF2989B083
:104D0000884646D8D0E90063029383898568059375
:104D1000B36802995B6806AA30469847002838DBDA
:104D2000DDE90649A5FB042305FB0933049203933F
:104D3000DDE9031018A3D3E90023FFF74BFE049B22
:104D4000DFF85CA04FF0FF3B9B45039B7AEB03032E
:104D500007461ED3FF23B5FBF3F508FB05F5A5FBBE
:104D6000048405FB09440CA3D3E9002321464046F3
:104D7000FFF730FEC3457AEB0404034609D38742AC
:104D800007D3B26805990091146802993A463046F3
:104D9000A04709B0BDE8F08F00CA9A3B00000000B0
:104DA000FFC99A3B000000002DE9F04706468AB093
:104DB0000F46904617F016FC4FF47A73A0FB03459C
:104DC00003FB0155E40B012F44EA45444FEAD53576
:104DD00008D1CDE900452A4A0821304612F016FFD5
:104DE000002013E0D8F8047026483946FFF70CFE7F
:104DF00078B125483946FFF707FE50B13046234ABF
:104E00003B46012112F002FF6FF004000AB0BDE83A
:104E1000F0872046294618A3D3E90023FFF78AFD2F
:104E200005460C4610461946194A0023FFF782FD35
:104E300080460F46104619464EF660220023FFF7C3
:104E400079FD82468946104619464FF47A7200234E
:104E5000FFF770FDCDE904A9CDE90601CDE90823EE
:104E6000CDE90287CDE900540A4A0821304612F004
:104E7000CDFEB5E7AFF30080005C26050000000022
:104E8000ECF40200FDF4020000F5020009F5020056
:104E900080EE360021F502007FB51E4D1E4C01AAA2
:104EA0004FF47C21284615F0A2FC029AA5624FF42B
:104EB0007C2320462360E2604FF48043B3FBF2F38F
:104EC000238202F011F8064600BB144D28232A461F
:104ED0000121204612F028FB282806D12A68104B11
:104EE0009A4202D1AB88072B10D00E4D0B4C0FCD40
:104EF0000FC40FCD0FC495E80300282384E80300F6
:104F0000A4F120020448012102F08CF9304604B0DB
:104F100070BD00BF94CB0200A013002078130020C6
:104F2000EFBEADDE58D3020030B404460FCC084DBE
:104F30000FC50FCC0FC594E8030085E80300A5F169
:104F40002002044830BC2823012102F06BB900BFC5
:104F500078130020A013002030B5054D04460FCD76
:104F60000FC40FCD0FC495E8030084E8030030BDE3
:104F70007813002013B5044601A800F039FE20463E
:104F8000BDF80430034A082112F040FE002002B0B0
:104F900010BD00BFB4E602001FB5044602A800F031
:104FA00067FABDF90C300193BDF90A300093204631
:104FB000BDF90830034A082112F028FE002004B091
:104FC00010BD00BFBEE60200042970B5144622D110
:104FD000506817F02BFCFFF74DFA1249FFF752FB10
:104FE0000546A06817F022FCFFF744FA0D49FFF7C9
:104FF00049FB0646E06817F019FCFFF73BFA094940
:10500000FFF740FB31460246284600F075FBBDE83D
:10501000704000F0B3BB044A012112F0F7FD6FF0BD
:10502000150070BD00007F43CEE6020005292DE982
:10503000F04114463AD1506817F0F8FB0746A068D3
:1050400017F0F4FB00282BDBA06817F0EFFBFFF74D
:1050500011FA1A49FFF716FB0546E06817F0E6FB60
:1050600000281FDBE06817F0E1FBFFF703FA1349A4
:10507000FFF708FB0646206917F0D8FB002813DB72
:10508000206917F0D3FBFFF7F5F90C49FFF7FAFA9F
:105090000346324629463846BDE8F04100F0BABC26
:1050A000074DDAE7064EE6E7054BF2E7054A012130
:1050B00012F0ACFD6FF01500BDE8F08100007F43F9
:1050C000000080BFFAE6020005292DE9F0411446F0
:1050D00025D1506817F0AAFB0546A06817F0A6FB7B
:1050E000FFF7C8F91249FFF7CDFA0646E06817F056
:1050F0009DFBFFF7BFF90E49FFF7C4FA0746206989
:1051000017F094FBFFF7B6F90949FFF7BBFA3A46E7
:10511000034631462846BDE8F04100F0FFBB054A92
:10512000012112F073FD6FF01500BDE8F08100BFA2
:1051300000007F433BE702007FB5064601A95068A7
:10514000154600F007FA044650B16B68084A012181
:10515000304612F05BFD6FF01504204604B070BDC0
:10516000039A0299019800F0C7FA00F007FBF4E7F0
:105170006DE70200022908B50BD1506817F056FB05
:10518000FFF778F90649FFF77DFABDE8084000F01F
:105190008BBA044A012112F039FD6FF0150008BDE9
:1051A0000000C84280E70200022908B506D1506815
:1051B00017F03CFBBDE8084000F022BA034A012189
:1051C00012F024FD6FF0150008BD00BFA3E7020038
:1051D00010B5064817F059F838B9BDE81040034833
:1051E00040F6CD4200230FF001BC10BD00000020AE
:1051F0001FB50223019002938DF80C309DF80C30FE
:10520000064843F002038DF80C30836801229C6845
:1052100001A96923A04704B010BD00BFB4CB0200B0
:1052200070B52E4886B00469836805A95B68984705
:10523000002839D12368059C5C4014F4000433D164
:1052400017F0D0F94FF47A720D46A0FB020302FB6F
:105250000533234D2349C20B28680E6842EA4342B6
:10526000121A4FEAD33340F2F51063F10003824281
:1052700073F1000306F0070618DB022E08D91A4B5B
:105280000094CDE9014303222346204611F0B0F9F2
:1052900017F0A8F94FF47A72A0FB020302FB013168
:1052A000C00B40EA4140286006B070BD022E08D90C
:1052B0000E4B0094CDE9014303222346204611F012
:1052C00097F940F20223ADF814300022002305A91B
:1052D000074809F065F811F009FAD9E7F4CA0200A5
:1052E000D013002098070020B2E90200B6E90200BE
:1052F0001CD10200F0B58FB0564C204616F077FD59
:10530000034680B954490A68520708D022680392BC
:10531000524A0090CDE90102012211F069F96FF0C3
:1053200012000FB0F0BD6B23ADF814306C23ADF854
:10533000183041F61C03ADF81C301D23ADF82030A9
:1053400042F23803ADF824304FF62273ADF828301E
:105350004CF26903ADF82C301923ADF8303005A8B4
:1053600042F26B03ADF83430FFF742FF00212120F9
:1053700011F04DF906A8FFF73BFF0021212011F0A5
:1053800046F907A8FFF734FF0021212011F03FF96B
:1053900008A8FFF72DFF0021212011F038F909A8F6
:1053A000FFF726FF0021212011F031F90AA8FFF7AD
:1053B0001FFF0021212011F02AF90BA8FFF718FF89
:1053C0000021212011F023F90CA8FFF711FF002183
:1053D000212011F01CF90DA8FFF70AFF40F6CD407F
:1053E000002111F014F91E4C2669A568336823F4D6
:1053F000000333602B684FF4803217212046984712
:10540000AF6967B1336813F4000F14BF4FF0007336
:105410004FF080634FF0A07217212046B847114A21
:10542000114B53604FF400039360EB691BB10D49BE
:105430000B480122984717F0D5F84FF47A72A0FB79
:10544000020302FB0131C00B084A40EA41401060F0
:10545000002066E7B4CB020098070020C1E90200F3
:10546000F4CA0200D4130020D1510100D01300204F
:1054700070B58EB03B23ADF816300DF116030893CE
:1054800006AB0B930623022200250C930723044648
:1054900009928DF828508DF834309DF83430124838
:1054A00013438DF83430836808A99E686923B04798
:1054B00078B10E490B685B0709D00D4B0390CDE91D
:1054C000015300952B460122284611F091F80EB0A9
:1054D00070BDBDF818302380BDF81A306380BDF868
:1054E0001C30A380F3E700BFB4CB02009807002074
:1054F000DCE902007FB503A800F07AFB134B1888A3
:10550000FEF7B4FF124B06461888FEF7AFFF4FF0C8
:105510007E550446BDF80C00FEF7A8FF2146009515
:105520000023324611F048F800210446FFF794F9B1
:1055300048B929462046FFF7ADF910B1284604B016
:1055400070BD2046FBE70020F9E700BFB006002051
:10555000FC1B00202DE9F843DFF8408007460D468C
:105560000024230108EB041658F803904846FFF77F
:105570005DFA3946421C484617F079F9034630B9BE
:10558000321D07CA85E807001846BDE8F8830134D4
:10559000282CE6D16FF01503F6E700BF78D502009E
:1055A0002DE9F0410F4D076806460024A8466868BB
:1055B0003946FFF747F970B17168A868FFF742F9FB
:1055C00048B1B168E868FFF73DF920B1240158F807
:1055D0000400BDE8F0810134282C05F11005E6D166
:1055E0000148F6E778D50200F7E9020027289ABFBC
:1055F000024B03EB00100020704700BF78D502007B
:105600002649274A2DE9F0474FF47A730C464FF4A8
:105610000045002158434FF4FF73B0FBF3F0E0FB6B
:10562000054120460023FFF7D5F91E4E07460D46DB
:105630000024FFF75FFFDFF86CA081464FF0000801
:105640005AF8040B4A46214608F1010810F0F0FF11
:10565000B8F1080FF4D138462946013410F0F9FFAB
:10566000FF2CE6D1FE24FFF745FFB24681464FF0FE
:1056700000085AF8040B4A46214608F1010810F0C8
:10568000D7FFB8F1080FF4D13846294610F0E1FFF2
:10569000013CE8D20020BDE8F08700BF3F420F0088
:1056A00040420F00F8D70200F8B50446FFF722FF8A
:1056B0004FF0824106462046FEF730FF0C490D4F61
:1056C000FEF72CFFFFF716F900250446FF2C94BFC8
:1056D0002146FF2157F8040B324605F101058CBF26
:1056E000FF3C002410F0A4FF082DEFD10020F8BDEE
:1056F00000007F43F8D702002DE9F84314460D4619
:105700000646FFF7F7FE31468146FEF707FF1649CA
:10571000FEF704FFFFF7EEF829465FFA80F84846E7
:10572000FEF7FCFE1049FEF7F9FEFFF7E3F821460D
:10573000C7B24846FEF7F2FE0B49FEF7EFFEFFF751
:10574000D9F80A4BC2B283F800805F709A7083F870
:1057500003801F715A71064B1E60064B1D60064B7D
:105760001C600020BDE8F88300007F431E1C002061
:10577000E8130020E4130020E01300201FB51148B7
:1057800084686368BBB923680F490E4802229847B2
:10579000044668B10D490B685B0709D00C4B0293B6
:1057A0000023CDE9003303940122184610F031FFA5
:1057B000204604B010BD98470128E4D86FF02104BA
:1057C000E8E700BF54CC02001E1C00209C0700200C
:1057D000FEE9020070B590B006A8FFF7BDFBBDF86A
:1057E0002830BDF82A20424D424E434C2B80934234
:1057F000328014D3216811F0060F0BD0CDE90332AB
:105800003E4B02930023CDE9003302222146184685
:1058100010F0FFFE00232B8040F2FF33338023681B
:1058200003F00703022B0DD9338804932B880393CD
:10583000334B02930023CDE900332F49032218464E
:1058400010F0E7FE2F4E002556F8043B186816F0BE
:10585000CEFA034678B92268520708D02A4A264968
:105860000395CDE901020090012210F0D2FE6FF005
:10587000120010B070BD56F8040C00210135FFF77E
:105880003BFA082DE0D1236803F00703022B09D966
:105890001E4B02930023CDE900331749032218461B
:1058A00010F0B7FE1A4816F0A2FA2268034602F07A
:1058B000070250B9002ADAD0164A0F490090CDE904
:1058C0000102012210F0A5FED1E7022A0BD9022322
:1058D0000393114B02930023CDE9003306490322C1
:1058E000184610F096FE10F0B8FE0020C1E700BF89
:1058F000FC1B0020B00600209C0700201DEA0200CF
:1059000051EA0200F8D702006DEA020082EA0200C2
:1059100054CC020097EA0200B2EA02002DE9F74FE8
:105920000F463649DFF8D8B00C464FF4004599468B
:1059300000214FF47A7358434FF4FF73B0FBF3F038
:10594000E0FB05412046904600232E4AFFF742F82F
:10595000002406460D462046FEF78CFD5946FEF70C
:1059600091FE824601464846FEF7D8FD5146019019
:105970004046FEF7D3FD514600903846FEF7CEFD77
:10598000019A0099FFF7B8FE0134FFF7F7FE3046A1
:10599000294610F05EFEFF2CDDD1DFF864B04FF039
:1059A000FE0A5046FEF766FD5946FEF76BFE494675
:1059B0000446FEF7B3FD414601902046FEF7AEFDDA
:1059C000394600902046FEF7A9FD019A0099FFF79D
:1059D00093FEFFF7D3FE3046294610F03AFEBAF1A7
:1059E000010ADED2084A00231360084A1360084AFD
:1059F0000020136003B0BDE8F08F00BF3F420F00EE
:105A000000007F4340420F00E8130020E413002011
:105A1000E01300202DE9F04F0E461C463A4B85B0AE
:105A2000074600213046D3F800901546FEF714FFD4
:105A300000B14E46354B00212846D3F800A0FEF7B2
:105A40000BFF00B15546324B00212046D3F800B081
:105A5000FEF702FF00B15C462E492F4A4FF47A73DD
:105A600003FB07F04FF4004C0F460021FF23B0FB6F
:105A7000F3F0E0FB0C7100233846FEF7ABFFCDE9F5
:105A800001014FF000084046FEF7F4FC2349FEF701
:105A9000F9FD594607462046FEF736FC3946FEF723
:105AA0003DFD5946FEF732FC514603902846FEF76D
:105AB0002BFC3946FEF732FD5146FEF727FC4946DE
:105AC00000903046FEF720FC3946FEF727FD494698
:105AD000FEF71CFC039A0099FFF70EFE08F101087F
:105AE000FFF74CFEDDE9010110F0B3FDB8F5807F52
:105AF000C9D1054B1E60054B1D60054B00201C6085
:105B000005B0BDE8F08F00BFE8130020E4130020CB
:105B1000E01300203F420F0040420F0000007F438F
:105B20001FB50223019002938DF80C309DF80C30C4
:105B3000064843F002038DF80C30836801229C680C
:105B400001A93823A04704B010BD00BFB4CB0200A8
:105B500010B592B0224C204616F049F9034680B9A0
:105B600020490A68520708D0226803921E4A009012
:105B7000CDE90102012210F07CFD6FF0120012B09D
:105B800010BD08A8FFF7E8F9184BBDF834200C98B1
:105B90009A8018604FF480721B79ADF814200421AC
:105BA00005A88DF818108DF81930ADF81C20FFF7F6
:105BB000B7FF002140F6CD4016F080FC06A8FFF7A5
:105BC000AFFF00214FF4A47016F078FC07A8FFF790
:105BD000A7FF40F6CD40002116F070FC0020CEE774
:105BE000B4CB0200A0070020C1E90200FE1B002088
:105BF00070B58CB01E23ADF816300DF116030222DD
:105C0000069305ABCDE90932002407230546079228
:105C10008DF820408DF82C309DF82C300E48134321
:105C20008DF82C30836806A99E683823B04778B178
:105C30000A490B685B0709D0094B0390CDE9014382
:105C4000009423460122204610F013FD0CB070BDD5
:105C5000BDF814302B80F9E7B4CB0200A007002078
:105C6000DCE902001FB5FFF717F9044680B11E49B1
:105C70000B685B0709D01D4B039002930023CDE90D
:105C800000330122184610F004FD204604B010BD78
:105C9000FFF7A0FD044630B113490B685807F4D054
:105CA000134B0394E9E7FFF725FB044630B10E4997
:105CB0000B685A07E9D00F4B0390DEE7FFF748FF68
:105CC000044630B108490B685B07DED00A4B0390ED
:105CD000D3E700F09DF800F0CDF800214FF400402C
:105CE00016F0ECFBF9E700BFAC070020DCEB02008C
:105CF000F6EB02000EEC020025EC02002DE9FF4756
:105D00003D4D0027BFF35B8F2B68BFF35B8F83B9DB
:105D10003A490A6802F00702022A07D9384A009372
:105D2000CDE901321846032210F0D1FC04B0BDE8E1
:105D3000F08710F0BEFCDFF8CC8004460E46BFF3BF
:105D40005B8F2B68BFF35B8F9BBB3846FFF7ACFCC8
:105D500010F0AFFCDFF8AC90DFF8AC8004460E46E4
:105D6000BFF35B8F2B68BFF35B8F002BCAD010F0A3
:105D7000A0FCD9F80420001B61EB0603D117904268
:105D800073EB0101BEDADFF884A0D8F80830BAF866
:105D90000000D8F80420D8F800104008FFF73AFEB9
:105DA000BAF8000000223B4611464008FFF732FED9
:105DB000D6E710F07EFCD8F80020001B61EB06034C
:105DC000D11790428B41C0DA10F073FC001B61EBDD
:105DD0000601FEF765FB8146D8F80000FEF74AFB96
:105DE00001464846FEF74EFCFFF75EFC002140F6F8
:105DF000CD4016F063FBA2E700140020B00700209E
:105E000052EC0200F8130020EC130020B206002030
:105E100010B590B006A8FFF79FF8DDE90801104B18
:105E2000104C0CAA83E8030007CA84E807000E4A56
:105E3000BDF83C1011800D490A6802F00702022AE1
:105E40000CD95A6804921B680393094B02930023F0
:105E5000CDE900330322184610F039FC10B010BD14
:105E6000F8130020EC130020B2060020B007002039
:105E700067EC020030B5224B012289B0BFF35B8F83
:105E800053E8001F002903D143E800200028F7D180
:105E9000BFF35B8F1B4D0CBF1346002326D100229E
:105EA0000023CDE9062300240523CDE90334CDE901
:105EB0000144154B154900944FF4806214480EF0CC
:105EC00079FF144912480EF031FE2B6803F00703E6
:105ED000022B09D9104B0094CDE90143032223463C
:105EE0002946184610F0F3FB09B030BD2A6812F0BD
:105EF000060FF9D0094A0093CDE901320222EFE7FB
:105F000000140020B0070020FD5C0100C01C002030
:105F1000600A0020420403008FEC02009DEC0200A6
:105F200030B51B4B002585B0BFF35B8F53E8002FC6
:105F3000012A03D143E800510029F7D1BFF35B8F59
:105F4000144C0CBF01232B4617D14FF0FF331248DE
:105F50004FF0FF320EF05AFF236803F00703022BC5
:105F600009D90E4B0095CDE9015303222B4621465A
:105F7000184610F0ACFB05B030BD226812F0060FD9
:105F8000F9D0074A0093CDE901320222EFE700BFC2
:105F900000140020B0070020600A0020B3EC0200CB
:105FA000C1EC0200F0B5164F85B00646002510F092
:105FB00052FBA84202DC002005B0F0BD2846FFF7E6
:105FC00015FB39460446C068FEF7A8FAFEF76CFCDC
:105FD0000290A0683946FEF7A1FAFEF765FC019031
:105FE00060683946FEF79AFAFEF75EFC0090236877
:105FF000044A0821304611F009FE0135D7E700BFF9
:1060000000007F43D3EC02007FB5054608460C46EE
:10601000FFF7C6FA0E490646A068FEF77FFAFEF7BC
:1060200043FC029060680A49FEF778FAFEF73CFCF0
:10603000019020680649FEF771FAFEF735FC054A23
:10604000009033460821284611F0E0FD04B070BDF1
:1060500000007F43EDEC020010B58EB0044604A8AA
:10606000FEF77AFF079B1E4A00930821069B2046F5
:1060700011F0CCFD0AA92046FFF7C6FFBDF8343069
:10608000184A0821204611F0C1FD9DF82430012B4B
:106090001BD0022B1BD0042B1BD0082B1BD0102B8A
:1060A0001BD10422104901EBC2025268CDE9013232
:1060B000BDF8223000932046BDF820300B4A08215D
:1060C00011F0A4FD00200EB010BD0022EAE701226D
:1060D000E8E70222E6E70322E4E7054AE6E700BF35
:1060E00012ED020030ED020090D9020042ED0200F4
:1060F0000AED020070B5134600228CB00546114629
:1061000058680FF09DFEC4B2012C16D0022C16D098
:10611000042C16D0082C16D0102C05D10423154AB7
:1061200002EBC3035E6886B92846134A012111F0C9
:106130006DFD6FF015000CB070BD0023EFE701237B
:10614000EDE70223EBE70323E9E702A8FEF704FFEC
:1061500002A88DF81C40FEF7E7FEFFF7F9FCFFF7F9
:1061600057FE2846054A00962346082111F04EFDA9
:106170000020E0E790D902006DED0200C4ED0200BE
:1061800030B505468DB0506816F050FBB0F5803F35
:1061900004460AD3154A4FF6FF730121284611F031
:1061A00035FD6FF015000DB030BD02A8FEF7D4FE2E
:1061B000BDF81820A3B2934207D8009223460C4A98
:1061C0000121284611F022FDEBE702A8ADF81A30B4
:1061D000FEF7AAFEFFF7BCFCFFF71AFE2846054AA9
:1061E0002346082111F012FD0020DCE7FAED020041
:1061F00013EE020043EE020030B505468DB0506844
:1062000016F014FBB0F5803F04460AD3154A4FF64A
:10621000FF730121284611F0F9FC6FF015000DB055
:1062200030BD02A8FEF798FEBDF81A20A3B2934233
:1062300007D3009223460C4A0121284611F0E6FCC0
:10624000EBE702A8ADF81830FEF76EFEFFF780FC12
:10625000FFF7DEFD2846054A2346082111F0D6FC4B
:106260000020DCE76FEE020088EE0200B5EE0200CF
:1062700030B514468DB0054602A8FEF76DFE606885
:1062800016F0D4FA0490A06816F0D0FA059002A88F
:10629000FEF74AFEFFF7BCFD10F028FAA368009352
:1062A00028466368034A082111F0B0FC00200DB0B5
:1062B00030BD00BFE1EE0200F0B58FB001AE054683
:1062C000314650681746FFF745F9044650B17B68E0
:1062D000114A0121284611F099FC6FF0150420465F
:1062E0000FB0F0BD04A8FEF737FE96E807000AAB32
:1062F00083E8070004A8FEF717FEFFF789FD10F0FA
:10630000F5F92846054A082111F080FC3146284657
:10631000FFF77AFEE3E700BF6DE702001AEF020025
:1063200030B504468BB0506816F080FA051E08DCC4
:1063300020460E4A012111F069FC6FF015000BB0E8
:1063400030BD6846FEF708FE6846ADF82450FEF7FB
:10635000EBFDFFF75DFD10F0C9F92046BDF82430D4
:10636000034A082111F052FC0020E8E737EF020051
:1063700061EF02002DE9FF410F46002972D0046849
:106380000E1F361BF50826F0070604EB0608B8F8C2
:10639000023013F0010314D134490A68520708D0BF
:1063A000334A0397CDE9013200930122184610F0D9
:1063B00032FA002383F31188BFF36F8F042318464A
:1063C00002DF2946204610F098F9284434F830308E
:1063D000C01A854215D025490B68580709D0254BAE
:1063E00002930023CDE9003303970122184610F0F1
:1063F00012FA002383F31188BFF36F8F042318462A
:1064000002DFB8F8023023F00103A8F80230294671
:10641000204610F072F92F1804EBC7035B88DA07E7
:1064200008D43946204610F0B1F93A4629462046AC
:1064300010F001FAA65BAE1B04EBC6035B88DB071A
:1064400009D43146204610F0A1F92A4631462046AB
:1064500010F0F1F935462946204604B0BDE8F04178
:1064600010F050B904B0BDE8F08100BFC8070020AB
:10647000E1F10200B8F1020008B5024810F053FB48
:10648000002008BD0EF202002DE9F04F91B0840704
:10649000009302F004030293C2F3C20303F1010369
:1064A000DDF868A0039205460E46059340F09D81F5
:1064B000041D00284AD101F00706341DC6F1080664
:1064C000009B00275A1E4FF004084FF0FF33019342
:1064D0000497B946BB4643460DB100992160059823
:1064E000002800F3D78090480099814203D38F4859
:1064F0008142C0F0CF80039911F0020CA4EB05009B
:1065000040F0D680B9F10F0F00F2CF80002D00F0DF
:10651000D68009F140010DEB010EC0F3870001990F
:106520000EF8200C0EF8101CBCF1000F00F0C38018
:1065300060F07F000EF8200C013709F10109C5F168
:106540000801043406914FF6DA7E8CE00729B7D8AB
:106550006FF01B0011B0BDE8F08F7A285BD84B2894
:106560000FD8472857D829282ED8252850D052D8B8
:10657000202818BF23280CBF4FF0010B4FF0000B51
:1065800071E04C382E2846D8DFE800F06D454545CF
:1065900045454545454545454845454545454545A8
:1065A00045564548485656566D486A456D45184803
:1065B0001845457F7C48454548457C0000204FF004
:1065C000000B4FF0040835E02A38C0B2012101FA6F
:1065D00000F010EA0E0F46D110F0625C2CD110EAE8
:1065E000010B40D06046013C4444B4FBF8F408FB86
:1065F00004F425B1A3EB050CA444B445A8D80028A5
:1066000070D00599013905915AF8041B009163E790
:106610000199013901914FF0000B24E012F8010CAF
:106620006C2834D112F8023C00206C2B8346C8D170
:106630004FF008084346D6E70AF1070A2AF0070A8E
:106640000734FAE802BC24F0070435B10698204468
:10665000B0423FF67DAFC4E900BC08344FF0000BF8
:106660004FF00808434612F8010F002853D0BBF141
:10667000000F7FF472AF2528F5D1019B0133019300
:106680004FF0010B4FF00408ECE7584697E7002065
:106690008346A8E7039988077FF551AF601B4FF049
:1066A000010CB0F5007FFFF42DAF6FF0150051E73E
:1066B0004FF0000CF5E70498013004903DE7BCF181
:1066C000000F01D0013638E70298023600287FF427
:1066D00034AF0098CDE90632FEF7A8F9DDE90632BD
:1066E00006442AE7042B08D10AF1040015B1DAF8B0
:1066F0000010216004348246B5E70AF1070323F055
:10670000070303F1080A1DB1D3E90001C4E9000140
:1067100008340823A7E7631BB3F5806FC5D23DB9E2
:10672000A6F10804E01815E7C4C902009427030085
:10673000029A28609B082B709DF81030AAB1EB706C
:10674000AF702FB108A80022C5F1010C91450ED100
:10675000C5F101030DF120084FF0000A01930DF17E
:10676000300BD14512D1601BF4E66B70E8E710F8EE
:10677000013B190608D50CEB040EB64503F07F0368
:106780003FF6E6AE04F8013B0132DFE71FB198F9AE
:106790000020002A17DB029BD3B11AF80B2004F863
:1067A000012B0022019B18191044B0423FF6D0AED5
:1067B00098F8000004F8010B00990392204616F0A7
:1067C00006F8039A14440AF1010A08F10108C8E71F
:1067D00098F8002055F822300093029B45F82230AB
:1067E0000098FEF723F9421CDCE76FF00D00B1E6DC
:1067F00030B50446EFF31185202383F31288BFF3ED
:106800006F8F044B0FCB84E80F0085F31188BFF323
:106810006F8F30BD180B002001281FB50C4605D026
:10682000042822D06FF0150004B010BD15F0DAFE78
:10683000174AC30BC0F30E00A0FB0202C00B43EAD1
:10684000414340EA4240C90BC4E90031A0606846B8
:10685000FFF7CEFF6946204610F033F918B90D4B0B
:106860000FCB84E80F000020DEE715F0BBFE084ADE
:10687000C30BC0F30E00A0FB0202C00B43EA41436E
:1068800040EA4240C90BC4E90031A060EBE700BF19
:1068900000CA9A3BF0D2020001287FB50C4633D1E2
:1068A0008A681B4B9A422FD815F09CFEC20B42EA15
:1068B000414252424FEAD13363EB4303CDE9002317
:1068C000144AC0F30E00A0FB0202C30B43EA42438A
:1068D0005B426846029300F0AFF82146684610F02C
:1068E000F0F8EFF31186202383F31288BFF36F8F44
:1068F0009DE80F00084C84E80F0086F31188BFF371
:106900006F8F002004B070BD6FF01500FAE700BF74
:10691000FFC99A3B00CA9A3B180B0020014B186034
